:100000000C948C080C94AB080C94AB080C9440092D
:100010000C9476090C94AB080C94AB080C94AB08C8
:100020000C94AB080C94AB080C94AB080C94AB0884
:100030000C94AB080C94AB080C94AB080C947E0C9D
:100040000C94AB080C94AB080C94AB080C94AB0864
:100050000C94FE610C940A590C94AB080C94AB08F8
:100060000C94AB080C94E0590C94AB080C94D45944
:100070000C94AB080C94AB080C94AB080C94AB0834
:100080000C94C16D0C94AB080C94AB080C94AB08A9
:100090000C941E5A0C94AB080C94125A0C94AB0896
:1000A0000C94AB080C94AB080C94AB080C94AB0804
:1000B0000C94AB080C94AB080C94AB080C94AB08F4
:1000C0000C94AB080C94AB080C94AB080C94AB08E4
:1000D0000C94AB080C94AB080C94AB080C94AB08D4
:1000E0000C94AB080C94B7610C94C1610C94AD6195
:1000F0000C9467610C94F2610C94E3610C94D761E9
:100100000C94CB610C94AB080C94AB080C94AB082A
:100110000C94AB080C94AB080C94AB080C94AB0893
:10012000084AD73B3BCE016E84BCBFFDC12F3D6C5E
:1001300074319ABD56833DDA3D00C77F11BED9E4C4
:10014000BB4C3E916BAAAABE000000803F076342F1
:1001500036B79BD8A71A39685618AEBAAB558C1D5E
:100160003CB7CC5763BD6DEDFD753EF6177231BFE0
:10017000000000803F08000000BE922449123EAB00
:10018000AAAA2ABECDCCCC4C3E00000080BEABAAB1
:10019000AAAA3E00000000BF000000803F0000004F
:1001A0000000084178D3BB4387D1133D190E3CC3EF
:1001B000BD4282AD2B3E68EC8276BED98FE1A93E6E
:1001C0004C80EFFFBE01C4FF7F3F00000000002510
:1001D000730A005854414C5F5452494D3D25640008
:1001E00025730A0025730A00546573742036202590
:1001F000730A005465737420352025730A00546512
:10020000737420342025730A0054657374203320DE
:1002100025730A005465737420322025730A005434
:1002200065737420312025730A006368616E3D2573
:10023000640A0074787077723D25640A0025730A99
:100240000073656E743D252D75206475703D252DF8
:10025000752069676E6F7265643D252D7520747415
:100260006C5F7A65726F3D252D750A0025372E3338
:10027000662025372E33660025352E326620004550
:1002800072726F72203020566F6C74004E6F742043
:10029000737570706F727465640A004572726F7264
:1002A000203020566F6C74004572726F72203020BF
:1002B000566F6C740025630074746C3D252D6420AA
:1002C0000074746C3D252D6420004E657720747495
:1002D0006C3D252D6420002563004D5335363131AA
:1002E00020503D252D372E326620252D372E3266A3
:1002F0006D0A00424D5030383520256C6420506125
:100300002020252D372E32666D00256300545F486E
:100310004541545F4944583D252D352E3266200015
:10032000545F4445573D252D352E32662000414807
:100330003D252D352E32662000545F5348543258E7
:100340003D252D352E3266200052485F53485432E9
:10035000583D252D352E32662000545F52483D25EC
:100360002D342E3166200052483D252D342E316625
:100370002000256300256300256300256300437585
:100380007272656E74207265706F727420696E741B
:10039000657276616C3D252D64207365630A004E9D
:1003A0006577207265706F727420696E74657276FD
:1003B000616C3D252D64207365630A00256300721E
:1003C00065706F72745F616C6C3D007265706F7206
:1003D000743D00256300256300256300256300202C
:1003E0004F534343414C3D256420002046757365BF
:1003F0003A2065653D253032782068663D253032EB
:1004000078206C663D25303278206C623D25303294
:1004100078004D43553D2530366C78002563002526
:100420002D31306C7520252D31306C7520252D3106
:10043000306C7520252D31306C75200A00747820C1
:100440006C656E20202020207268206D69737320F7
:100450002020207268207374616C652020207268EF
:10046000206D6973630A002563004F4B0A00256302
:100470000025630025630025630025630064656231
:1004800075675F616C6C3D0064656275673D006413
:10049000656275673D0025730A00646565700A0032
:1004A000666F7263655F69646C650A006E6F6E6586
:1004B0000A00707772733D00696E74725F736563D2
:1004C0005F70313D252D372E33660A00696E7472D8
:1004D0005F70313D252D6C640A00696E74725F7324
:1004E00065635F70303D252D372E33660A00696ED7
:1004F00074725F70303D252D6C640A00765F6D6309
:10050000753D252D352E32660A00707077723D25B7
:10051000730A0064656275673D0025730A006175A2
:10052000746F0A006C6F675F6D6F64653D00757373
:10053000625F7077723D25730A007265706F727426
:100540003D007265706F72745F696E74657276617A
:100550006C3D252D640A0072656C61793D25730A36
:100560000074746C3D252D640A0052494D455F614D
:100570006464723D252D642E252D640A006E656924
:100580006768626F725F7461626C655F73697A65D8
:100590003D25640A00747870773D25640A0063681D
:1005A000616E3D25640A006932633D0069643D0067
:1005B0007478743D25730A0053797374656D205304
:1005C000756D6D6172790A00745F686561745F6949
:1005D000647800745F64657700616800705F6D73B4
:1005E000353631310072685F736874327800745F39
:1005F0007368743278007061007000616434006167
:10060000643300616432006164310061330061323F
:1006100000613100765F696E007268007570746900
:100620006D650070315F6C73740070315F740070C1
:10063000310070305F6C73740070305F7400703024
:1006400000765F6D637500745F6D637500743100D3
:1006500074006964006536340074787400617574E0
:100660006F006E6F6E650072656C61795F6C6564BA
:100670007900636F6D7061737300616363656C0013
:100680007072657300705F707772006165730070DF
:10069000315F6C6564790070305F6C656472006511
:1006A00076656E74006C6564006F7700706B740023
:1006B00074785F6C6564790072785F6C6564720051
:1006C0006F706572006E6F6E65002530327800764F
:1006D0005F6164343D252D382E3666002000765F3C
:1006E0006164333D252D382E3666002000765F612B
:1006F00064323D252D382E3666002000765F616419
:10070000313D252D382E3666002000765F6C6967F6
:1007100068743D252D382E3666002000765F6132E4
:100720003D252D372E3366002000765F61313D2553
:100730002D372E3366002000765F696E3D252D35FE
:100740002E326600204E657665722D7573656420C5
:10075000737461636B203E20256420627974657335
:100760000A00757074696D653D252D642D6461798D
:10077000732D253032643A253032643A25303264A4
:100780002D686F7572730A0074657374205B6F66F1
:10079000667C317C327C337C347C355D20202020AB
:1007A000202020202D2074657374206D6F64657384
:1007B0000A0D00263A205B545820504B5420434FDA
:1007C0004E54454E545D2020202020202020202DF6
:1007D0002073656E6420706B742066726F6D206389
:1007E0006D646C696E652F636861740A0D007764CF
:1007F00074205B6F6E7C6F66667C746573745D20BD
:10080000202020202020202020202D2077617463AC
:1008100068646F670A0D00757067722020202020C1
:1008200020202020202020202020202020202020C8
:100830002020202D207265626F6F74207669612000
:10084000626F6F746C6F616465720A0D00626F6F26
:100850007420202020202020202020202020202044
:100860002020202020202020202D207265626F6F04
:10087000740A0D0070777273205B646565707C6626
:100880006F7263655F69646C657C6E6F6E655D2019
:100890002D206D637520736C656570206D6F6465C8
:1008A0000A0D007265737420656570726F6D20208B
:1008B0002020202020202020202020202020202D2B
:1008C00020726573746F726520656570726F6D0A52
:1008D0000D0070707772205B6F6E7C6F66665D20B6
:1008E00020202020202020202020202020202D20FB
:1008F00070726F6772616D6D61626C652070777286
:100900000A0D00747874205B737472696E675D20E1
:100910002020202020202020202020202020202DCA
:1009200020536574207265706F72742074657874DA
:1009300020737472696E670A0D0074787077205B9B
:1009400031352D305D202020202020202020202027
:100950002020202020202D205458205077722E2037
:1009600048696768657374203020283364426D29B4
:100970000A0D0074746C205B302D31355D20202011
:100980002020202020202020202020202020202D5A
:100990002074696D652D746F2D6C69766520666FA6
:1009A00072207061636B6574730A0D00737320208D
:1009B0002020202020202020202020202020202037
:1009C00020202020202020202D2073797374656D35
:1009D0002073756D6D6172790A0D0072732020208D
:1009E0002020202020202020202020202020202007
:1009F000202020202020202D20726164696F207328
:100A0000746174730A0D007269205B696E745D20F5
:100A100020202020202020202020202020202020D6
:100A20002020202D207265706F727420696E7465AD
:100A30007276616C0A0D007265205B6D61736B7C70
:100A40006175746F2C6D61736B5D202020202020F8
:100A50002020202D206D6F7465207265706F727478
:100A60002073657474696E670A0D006F772020200B
:100A70002020202020202020202020202020202076
:100A8000202020202020202D206F6E652D77697278
:100A9000652073656E736F72730A0D006C6F67204B
:100AA0005B6175746F7C6F6E7C6F66665D20202065
:100AB00020202020202020202D206D6F74657320A1
:100AC00064617461206F6E205553420A0D006E659B
:100AD000205B666C7573685D20202020202020201C
:100AE000202020202020202020202D206E656967D6
:100AF00068626F72207461626C650A0D00657272C3
:100B000020202020202020202020202020202020E5
:100B10002020202020202020202D206572726F723E
:100B200020696E666F0A0D006D63752020202020FD
:100B300020202020202020202020202020202020B5
:100B4000202020202D206D637520696E666F0A0DB0
:100B5000006964205B72657365745D20202020202D
:100B6000202020202020202020202020202D20692F
:100B7000642068616E646C696E670A0D0068756D4B
:100B80002020202020202020202020202020202065
:100B90002020202020202020202D2068756D6964D1
:100BA0006974792073656E736F720A0D0072656CDB
:100BB0006179205B6F6E7C6F66667C7374617473A1
:100BC0005D20202020202020202D2072656C61795E
:100BD000206E6574776F726B207265706F727473BC
:100BE0000A0D006465205B6D61736B5D2020202021
:100BF0002020202020202020202020202020202DE8
:100C00002064656275670A0D006368616E205B3160
:100C1000312D32365D202020202020202020202051
:100C200020202020202D206368616E2031312D325C
:100C3000362028322E3430352D32343830204D686D
:100C40007A290A0D0063616C69205B5B765F696ECF
:100C50007C61317C61325D20766F6C747C7265736F
:100C600065747C6E6F6E655D202D2063616C6962BA
:100C7000726174650A0D00616463202020202020C9
:100C80002020202020202020202020202020202064
:100C90002020202D2073686F7720765F696E2C20CE
:100CA00061312C20613220766F6C74616765730A44
:100CB0000D00752020202020202020202020202012
:100CC00020202020202020202020202020202D2017
:100CD000757074696D650A0D007620202020202033
:100CE0002020202020202020202020202020202004
:100CF00020202020202D2076657273696F6E0A0DEA
:100D000000682020202020202020202020202020BB
:100D1000202020202020202020202020202D20687E
:100D2000656C700A0D00256300756E6B6E6F776ED3
:100D300020636D640A00484D43353838330025730D
:100D400000257300202573002025362E32662000F2
:100D5000253032780074656D705F65787465726EE9
:100D60003D252D362E326600202573002025362E97
:100D70003266204F6E2D426F6172640025303278EA
:100D80000074656D705F626F6172643D252D362E53
:100D90003266000A00503A20256C64205061202001
:100DA000252D372E3266206D0A002563002563004D
:100DB0004932433A2000452025642E256420636C87
:100DC0006F636B20256C752063707520256C752012
:100DD0006C706D20256C752069727120256C7520F2
:100DE000676C656420256C7520796C656420256CC2
:100DF0007520726C656420256C7520747820256CD4
:100E000075206C697374656E20256C752073656E32
:100E1000736F727320256C752073657269616C2025
:100E2000256C750A00532025642E256420636C6FA1
:100E3000636B20256C7520747820256C7520727882
:100E400020256C752072747820256C75207272785C
:100E500020256C75207265786D697420256C75206D
:100E600061636B747820256C75206E6F61636B74A1
:100E70007820256C752061636B727820256C752055
:100E800074696D65646F757420256C75206261648A
:100E900061636B727820256C7520746F6F6C6F6E58
:100EA0006720256C7520746F6F73686F72742025CE
:100EB0006C752062616473796E636820256C75209F
:100EC00062616463726320256C7520636F6E746564
:100ED0006E74696F6E64726F7020256C7520736517
:100EE0006E64696E6764726F7020256C75206C6C1F
:100EF000747820256C75206C6C727820256C750ACE
:100F000000257325730A004F6E6C696E650A000A2E
:100F1000002C20636865636B207261746520257501
:100F200020487A0025732025732C206368616E6E3B
:100F3000656C20257520706F776572202575000A15
:100F40000025783A004D41432061646472657373F3
:100F5000200052616E646F6D204555493634206122
:100F60006464726573732067656E6572617465642D
:100F70000A000A2A2A2A2A2A2A2A426F6F74696ECC
:100F8000672025732A2A2A2A2A2A2A0A0002000010
:100F9000FFFE00000141544D454741313238726631
:100FA0006131006C6F63616C686F7374004545500C
:100FB000524F4D20697320636F72727570742C20CC
:100FC000726577726974696E6720776974682064E6
:100FD000656661756C74732E0A006E616E00696ED1
:100FE000660000407A10F35A00A0724E18090010F3
:100FF000A5D4E80000E87648170000E40B5402008E
:1010000000CA9A3B000000E1F505000080969800B8
:10101000000040420F000000A086010000001027E1
:1010200000000000E8030000000064000000000071
:101030000A00000000000100000000002C76D888A3
:10104000DC674F0823DFC1DFAE59E1B1B796E5E3B6
:10105000E453C63AE651997696E8E6C28426EB89CF
:101060008C9B62ED407C6FFCEFBC9C9F40F2BAA56C
:101070006FA5F490055A2AF75C936B6CF9676DC104
:101080001BFCE0E40D47FEF520E6B500D0ED902E08
:101090000300943577050080841E080000204E0A66
:1010A000000000C80C333333330F986E12831141A4
:1010B000EF8D2114893BE65516CFFEE6DB18D1846F
:1010C0004B381BF77C1D901DA4BBE4242032847296
:1010D0005E228100C9F124ECA1E53D274E414E4935
:1010E0004E495459494E46CDCCCC3D0AD7233C17E6
:1010F000B7D13877CC2B329595E6241FB14F0A0033
:101100000020410000C84200401C4620BCBE4CCA22
:101110001B0E5AAEC59D740011241FBECFEFD1E443
:10112000DEBFCDBF19E0A0E0B2E0E0EDF7E101E005
:101130000BBF02C007900D92A632B107D9F710E39A
:10114000A6E2B9E001C01D92A93AB107E1F70E94F9
:10115000C4570C94E68B0C94000082EB94E09F93B0
:101160008F930E94EE8880914002909141020F90EF
:101170000F9093FF03C08CEA94E007C092FF03C076
:1011800080EA94E002C08AE994E09F938F930E94E2
:10119000EE880F900F900895E091BB1AEF71F0E088
:1011A000E05FF44E80838091BB1A8F5F8093BB1AFF
:1011B0008091E32788608093E3274AE252E061E16F
:1011C000CA010E941C4880E090E00895CF93DF930D
:1011D000EC0180912D0990912E0986FF1DC08E8112
:1011E0001F928F938D811F928F938C811F928F936B
:1011F0008B811F928F938A811F928F938DEF93E043
:101200009F938F930E94DC888DB79EB70C960FB684
:10121000F8949EBF0FBE8DBFBE0184E699E00E9488
:101220006149BE0184E092E0DF91CF910C94CD48FA
:1012300087EE93E08115910511F00197F1F708957C
:101240008823B9F052985A981DBA8091690080623B
:1012500080936900EA9A53985B98EB9A80916900B1
:101260008068809369008091680081608093680045
:101270000895109269005A9AEA985B9AEB9808953B
:101280001F920F920FB60F9211248F939F93AF93DB
:10129000BF938091680080FF20C08091C327909108
:1012A000C427A091C527B091C6270196A11DB11DE5
:1012B0008093C3279093C427A093C527B093C627D4
:1012C00080912D0990912E0987FF07C0749882E0C4
:1012D00090E09093700280936F02BF91AF919F91C5
:1012E0008F910F900FBE0F901F9018951F920F9225
:1012F0000FB60F9211248F939F93AF93BF9380915A
:10130000680080FF20C08091C7279091C827A091D6
:10131000C927B091CA270196A11DB11D8093C72787
:101320009093C827A093C927B093CA2780912D090D
:1013300090912E0990FF07C0739882E090E09093FF
:10134000700280936F02BF91AF919F918F910F9028
:101350000FBE0F901F90189580937C0080917B00AA
:10136000877F80937B0080917C00806C80937C00E1
:1013700085E080937A0080917A00806880937A007B
:1013800080917B0087FFFCCF80917B0085FFFCCFA5
:1013900080917A00806480937A0080917A0086FD43
:1013A000FCCF109279001092780084E090E060E029
:1013B00070E020917A00206420937A0020917A00D6
:1013C00026FDFCCF2091780030917900620F731FC9
:1013D0000197009771F710927C0080917A008F77C7
:1013E00080937A00769567957695679580E090E092
:1013F0000E94747F089580E00E94AC0920916B02E6
:1014000030916C0240916D0250916E020E945481A5
:1014100021EE3AE744E95EE30E940D7E089580E103
:101420008093510160E1609351018091510185FFEA
:1014300003C06F5F6F31B9F78BE4689FB00111246F
:10144000882777FD8095982F0E94767F20E030E6F0
:101450004FE954E40E940D7E20E030E04AE754E476
:101460000E94D77E089565FF4BC080917B00886005
:1014700080937B0089EC80937C0085E080937A00E8
:1014800080917A00806880937A0080917B0087FF4A
:10149000FCCF80917B0085FFFCCF80917A00806437
:1014A00080937A0080917A0086FDFCCF80917A004B
:1014B000806480937A0080917A0086FDFCCF6091F1
:1014C00078007091790080E090E00E94747F27EDB1
:1014D00033EA40E95FE30E94548126E636E648E8B5
:1014E00053E40E940C7E6093801A7093811A80935B
:1014F000821A9093831A80917A008F7780937A0072
:101500000895BF92CF92DF92EF92FF920F931F93B5
:10151000CF93DF93CDB7DEB729970FB6F894DEBF30
:101520000FBECDBF6C01109226098FEF89870CEC9E
:101530001AE1B12C7E0189E0E80EF11C898588232F
:10154000E9F1E8E0BE16E1F1BE016F5F7F4FC70130
:101550000E94D65189858F3F11F08E3F19F48093F8
:1015600026092CC0CE010196C114D10471F40E9449
:10157000F0518093E027FE013196A8EDB7E281910A
:101580008D93EE15FF05D9F71DC00E94F051F801AB
:101590008083FE01319620E030E0A80148505109D7
:1015A0008191DA01A20FB31F8C932F5F3F4F283038
:1015B0003105B1F7B394075F1F4FC0CF8B2D03C028
:1015C00088E001C081E029960FB6F894DEBF0FBE17
:1015D000CDBFDF91CF911F910F91FF90EF90DF90E2
:1015E000CF90BF90089583E99DE09F938F930E94D1
:1015F000EE880F900F9008952F923F924F925F9236
:101600006F927F928F929F92AF92BF92CF92DF9212
:10161000EF92FF920F931F93CF93DF93EC014B0157
:10162000009711F427E004C08130910549F426E0C9
:101630004AE250E06BE270E089E290E00E94B25032
:10164000CE010E94810A9E01295D364F5901D901C0
:101650008C93CD2B69F09CECC92E9AE1D92EC4EC69
:10166000DAE1E12CF12C24E4222E2DE0322EA6C06A
:1016700088ED97E20E942253BC01882777FD809570
:10168000982F0E94767F6B017C01892869F020E009
:1016900030E048EC52E40E94D77E9F938F937F9373
:1016A0006F9381E89DE0ACC0C8EDD7E20CE71DE088
:1016B00089911F928F931F930F930E94EE880F9032
:1016C0000F900F900F90B7E2C03EDB0789F720E044
:1016D00030E048EC52E4C701B6010E94D77E9F93E8
:1016E0008F937F936F938CE69DE09F938F930E94DF
:1016F000EE880F900F900F900F900F900F908091A9
:10170000E027882319F08CE294E002C080EA94E09C
:101710009F938F9388E69DE09F938F930E94EE881E
:101720000F900F900F900F9075C000E010E0FE0139
:10173000E00FF11F80811F928F93A0E5BDE0BF9362
:10174000AF930E94EE880F5F1F4F0F900F900F9086
:101750000F900830110559F720E030E048EC52E4D2
:10176000C301B2010E94D77E9F938F937F936F93A3
:10177000A8E4BDE0BF93AF930E94EE880F900F9056
:101780000F900F900F900F90D6018C91882309F441
:1017900055C08CE294E09F938F933F922F920E94CA
:1017A000EE880E94F30ABFEFEB1AFB0AE9E0CE0EC7
:1017B000D11C29960F900F900F900F90D5018C910E
:1017C00090E0E816F906ECF5CE010E942253BC0128
:1017D000882777FD8095982F0E94767F2B013C010A
:1017E0008114910409F4A1CF20E030E048EC52E4E8
:1017F0000E94D77E9F938F937F936F9385E59DE0A3
:101800009F938F930E94EE880F900F900F900F90F0
:101810000F900F90DF91CF911F910F91FF90EF905C
:10182000DF90CF90BF90AF909F908F907F906F9000
:101830005F904F903F902F900C94F30A80EA94E0D1
:10184000AACFDF91CF911F910F91FF90EF90DF9082
:10185000CF90BF90AF909F908F907F906F905F9050
:101860004F903F902F900895CF93DF9300D0CDB746
:10187000DEB78091D92789838091DF278A83CE01C3
:1018800001960E94FB450F900F90DF91CF91089534
:10189000CF93DF93EC012091D8273091D927409145
:1018A000DA275091DB276091DC277091DD2780914A
:1018B000DE279091DF27AFEF0E947784E1F427E0E5
:1018C0004AE250E06BE270E089E290E00E94B250A0
:1018D00080E090E00E94810AC95DD64F888349E08C
:1018E00050E06AE070E088ED97E20E94318ADF9173
:1018F000CF910C94340CDF91CF9108951F920F92E9
:101900000FB60F9211240BB60F922F933F934F9364
:101910005F936F937F938F939F93AF93BF93CF9377
:10192000EF93FF938091E32782608093E327809178
:10193000400286FD2B9A8091400287FD2B9A809170
:101940006F02909170021816190614F4749A739A23
:1019500080912D0990912E0985FF02C0749873988B
:101960008091020290910302019790930302809369
:101970000202892B09F01DC180913B0990913C091D
:101980009C012F5F3F4F30933C0920933B094091CE
:1019900063235091642360916523709166234F5FA8
:1019A0005F4F6F4F7F4F4093632350936423609347
:1019B00065237093662320E130E030930302209387
:1019C00002022091400220FD02C01D9B05C0109222
:1019D0002B0910922A0906C021E030E030932B0930
:1019E00020932A09609146027091470261157105A2
:1019F00099F002960E945582892B71F47798809114
:101A00002D0990912E0992FF07C0749884E090E010
:101A10009093700280936F0260914602709147022A
:101A200061157105B1F180913B0990913C090E94CB
:101A30005582892B71F581E080937823809148024B
:101A4000809379238091490280937A2380914A027E
:101A500080937B2380914B0280937C2380914C0266
:101A600080937D2380914D0280937E2380914E024E
:101A700080937F2380914F02809380231092822352
:101A80001092812348E753E262E180E292E00E94F3
:101A90001C48609144027091450261157105A1F1E5
:101AA00080913B0990913C090E945582892B61F5F8
:101AB0008091C3279091C427A091C527B091C627D4
:101AC0004091591B50915A1B60915B1B70915C1B9C
:101AD000841B950BA60BB70B8093931A9093941AC3
:101AE000A093951AB093961A8091C3279091C4271A
:101AF000A091C527B091C6278093591B90935A1B7C
:101B0000A0935B1BB0935C1B6091420270914302F7
:101B100061157105A1F180913B0990913C090E94EA
:101B20005582892B61F58091C7279091C827A09194
:101B3000C927B091CA2740915D1B50915E1B6091EF
:101B40005F1B7091601B841B950BA60BB70B8093DA
:101B5000971A9093981AA093991AB0939A1A809111
:101B6000C7279091C827A091C927B091CA27809311
:101B70005D1B90935E1BA0935F1BB093601B8091D5
:101B8000400286FD2B98809140029091410291FF86
:101B900010C00E94E95D8A3119F0C1E0C80F01C090
:101BA000CBE00E942D5C8C2F90E00E94015E0E9491
:101BB000CB5C40E050E060E089E892E00E941C4885
:101BC000FF91EF91CF91BF91AF919F918F917F91B5
:101BD0006F915F914F913F912F910F900BBE0F909E
:101BE0000FBE0F901F9018958091BB1A909177238C
:101BF000891B08950E94F40D882371F0E0917723EA
:101C0000EF71F0E0E05FF44E808190E02091772367
:101C10002F5F2093772308958FEF9FEF0895CF9341
:101C2000DF93EC011092580910925709888199812D
:101C30000097C1F08734934021F01982188283E025
:101C4000B6C0613109F0B2C0F89478940E94FA0DE0
:101C5000992790935309809352098D3009F441C01C
:101C60008F3F49F40E94F40D8111EECF87E493E099
:101C7000998388839BC08231910509F458C08F37BE
:101C8000910509F050C080915009909151091816A2
:101C900019060CF56091A3307091A43088E090E0B3
:101CA0000E94AA886091A3307091A43080E290E0F5
:101CB0000E94AA886091A3307091A43088E090E0DF
:101CC0000E94AA88809150099091510901979093A0
:101CD0005109809350098091500990915109CF97F3
:101CE00009F6109277231092BB1A809150099091B7
:101CF0005109FC01ED57FC4D1082909358098093D7
:101D0000570910925109109250098091E127909142
:101D1000E227009709F4A6CF40E050E060916611F9
:101D20000E941C489FCF8830910571F5ACCF60911F
:101D3000A3307091A4308DE090E00E94AA881092A8
:101D40004F0910924E0980914E0990914F092091B0
:101D5000500930915109821793070CF0BCCFFC0158
:101D6000ED57FC4D80816091A3307091A43090E0DC
:101D70000E94AA8880914E0990914F0901969093F4
:101D80004F0980934E09DFCF6091A3307091A4304A
:101D90000E94AA888091500990915109209152097E
:101DA000FC01ED57FC4D2083019691CF81E0DF913E
:101DB000CF910895789480912A0990912B09892BCD
:101DC000C9F0809140029091410293FD13C092FFAF
:101DD00003C083B7817F03C083B7817F866083BFE1
:101DE000F89483B7816083BF7894889583B78E7F9A
:101DF00083BF78940895CF93DF93EC018881998114
:101E0000009719F0803C9E4099F40E941B5B0E9451
:101E1000DA0E40E050E065E880916C1190916D1110
:101E20000E941C4880EC9EE09983888381E003C077
:101E30001982188283E0DF91CF910895CF93DF93C9
:101E400000D0CDB7DEB7892B81F05F934F9381E44B
:101E50009DE09F938F9369837A830E94EE880F9011
:101E60000F900F900F907A8169817F936F938EE32B
:101E70009DE09F938F930E94EE880F900F900F909C
:101E80000F900F900F90DF91CF910895FF920F93D5
:101E90001F93CF93DF930E941B5B80EB0E94A253A2
:101EA00081111CC00E9408548091611F9091621F93
:101EB00081609093621F8093611F85E394E09F93FC
:101EC0008F938EE39DE09F938F930E94EE880F90F7
:101ED0000F900F900F90C1E0D0E002C0C0E0D0E0C2
:101EE000FEB08F2D8470F82E729A0E941B5B8EE4D8
:101EF0000E94A253811116C00E9408548091611F54
:101F00009091621F82609093621F8093611F8E0187
:101F10000F5F1F4F43E259E06DE374E0CE010E9472
:101F20001E0FE801F11001C072980E941B5B8EEE3B
:101F30000E94A253811116C00E9408548091611F13
:101F40009091621F84609093621F8093611F8E0145
:101F50000F5F1F4F43E259E065E474E0CE010E9439
:101F60001E0FE8010E941B5B86EA0E94A2538111AA
:101F700016C00E9408548091611F9091621F886072
:101F80009093621F8093611F8E010F5F1F4F43E28A
:101F900059E06CE474E0CE010E941E0FE8010E943B
:101FA0001B5B8CE30E94A25381111EC00E94085447
:101FB0008091611F9091621F80619093621F809356
:101FC000611F8E010F5F1F4F43E259E064E574E02B
:101FD000CE010E941E0F86E39DE09F938F930E9487
:101FE000EE880F900F90E8010E941B5B82ED0E942B
:101FF000A253811116C00E9408548091611F9091D4
:10200000621F80629093621F8093611F8E010F5F39
:102010001F4F43E259E06CE574E0CE010E941E0FB1
:10202000E8010E941B5B80E80E94A253811116C048
:102030000E9408548091611F9091621F916090935B
:10204000621F8093611F8E010F5F1F4F43E259E0B3
:1020500065E674E0CE010E941E0FE8010E941B5B42
:1020600080ED0E94A253811116C00E9408548091F5
:10207000611F9091621F80689093621F8093611F1F
:102080008E010F5F1F4F43E259E06BE674E0CE0113
:102090000E941E0FE8010E941B5B8CEE0E94A2535F
:1020A000811116C00E9408548091611F9091621F97
:1020B00092609093621F8093611F8E010F5F1F4F8C
:1020C00043E259E063E774E0CE010E941E0FE8018D
:1020D00007E010E00E941B5B8CE70E94A253811175
:1020E00013C00E9408548091611F9091621F806408
:1020F0009093621F8093611F43E259E06AE774E0A6
:10210000CE010E941E0F05C00150110901151105D5
:1021100009F70E940854DF91CF911F910F91FF9012
:102120000C94F30ACF93DF9300D0CDB7DEB74A8388
:1021300069830E94DE536981862F0E9410544A8170
:10214000842F0E9410540F900F90DF91CF910C9428
:102150000854AF92BF92DF92EF92FF920F931F93BA
:10216000CF93DF9300D01F92CDB7DEB7182FD22EBA
:102170004A835B8369830E94DE536981862F0E94B4
:102180001054812F81600E9405544A81A42E5B81E6
:10219000B52E00E010E0ED2CF12C81E0E81AF108FA
:1021A0000D1580F40E151F0519F40E942B5402C062
:1021B0000E942154F50180830F5F1F4FFFEFAF1A7C
:1021C000BF0AEECF0F900F900F90DF91CF911F912C
:1021D0000F91FF90EF90DF90BF90AF900C94085458
:1021E000AF92BF92CF92DF92EF92FF920F931F9325
:1021F000CF93DF93CDB7DEB760970FB6F894DEBF0D
:102200000FBECDBFB82EA42E6623E9F18E010F5F5D
:102210001F4F80E1F80111928A95E9F728E0A801A3
:1022200068E980EB0E94A910BB2041F023E834E06C
:102230003F932F930E94DC880F900F906E01F8E07F
:10224000CF0ED11C4AE8E42E44E0F42EF80181912F
:102250008F011F928F93FF92EF920E94DC880F9064
:102260000F900F900F900C151D0581F788851F9218
:102270008F932FED34E03F932F930E94DC880F90D3
:102280000F900F900F90AA20E9F18E010F5F1F4F62
:1022900080E1F80111928A95E9F728E0A80160E849
:1022A00080EB0E94A910BB2041F08FE894E09F933F
:1022B0008F930E94DC880F900F906E01F0E1CF0E9B
:1022C000D11C3AE8E32E34E0F32EF80181918F011E
:1022D0001F928F93FF92EF920E94DC880F900F90D5
:1022E0000F900F900C151D0581F788851F928F9315
:1022F0008FED94E09F938F930E94DC880F900F9056
:102300000F900F9060960FB6F894DEBF0FBECDBF52
:10231000DF91CF911F910F91FF90EF90DF90CF90C1
:10232000BF90AF900895CF93DF9300D0CDB7DEB7C5
:102330001A82198222E0AE014F5F5F4F6AEA8EEE89
:102340000E94A910898190E0982F88272A81822BEA
:102350009093311B8093301B22E0AE014F5F5F4FA3
:102360006CEA8EEE0E94A910898190E0982F882750
:102370002A81822B9093331B8093321B22E0AE0183
:102380004F5F5F4F6EEA8EEE0E94A910898190E048
:10239000982F88272A81822B9093351B8093341B9A
:1023A00022E0AE014F5F5F4F60EB8EEE0E94A910FE
:1023B000898190E0982F88272A81822B9093431B54
:1023C0008093421B22E0AE014F5F5F4F62EB8EEEC7
:1023D0000E94A910898190E0982F88272A81822B5A
:1023E0009093451B8093441B22E0AE014F5F5F4FEB
:1023F00064EB8EEE0E94A910898190E0982F8827C7
:102400002A81822B9093471B8093461B22E0AE01CA
:102410004F5F5F4F66EB8EEE0E94A910898190E0BE
:10242000982F88272A81822B9093371B8093361B05
:1024300022E0AE014F5F5F4F68EB8EEE0E94A91065
:10244000898190E0982F88272A81822B9093391BCD
:102450008093381B22E0AE014F5F5F4F6AEB8EEE38
:102460000E94A910898190E0982F88272A81822BC9
:1024700090933D1B80933C1B22E0AE014F5F5F4F6A
:102480006CEB8EEE0E94A910898190E0982F88272E
:102490002A81822B90933F1B80933E1B22E0AE014A
:1024A0004F5F5F4F6EEB8EEE0E94A910898190E026
:1024B000982F88272A81822B9093411B8093401B61
:1024C0000F900F90DF91CF9108952F923F924F92EE
:1024D0005F926F927F928F929F92AF92BF92CF92B4
:1024E000DF92EF92FF920F931F93CF93DF93CDB7BD
:1024F000DEB76A970FB6F894DEBF0FBECDBF182FB8
:10250000488F298F19821A821B828091541B811156
:1025100007C06A8F0E94931181E08093541B6A8DDB
:10252000662309F46CC04EE264EF8EEE0E949210B6
:1025300069E07AE180E090E00E948F5322E0AE01F2
:102540004F5F5F4F66EF8EEE0E94A9102981822FA8
:1025500090E0A0E0B0E02227382F492F5A2F8A813F
:10256000282B8091461B9091471B281B390B410952
:102570005109A091441BB091451B0E9432826B010E
:102580007C018FE0F594E794D794C7948A95D1F7AE
:1025900060913E1B70913F1B882777FD8095982F97
:1025A0002BE0660F771F881F991F2A95D1F720917E
:1025B000401B3091411B442737FD4095542F2C0D73
:1025C0003D1D4E1D5F1D0E949F82C20ED31ED092E4
:1025D0003B1BC0923A1B88E0C80ED11C34E0D59456
:1025E000C7943A95E1F7EE24D7FCE094FE2CC09214
:1025F000481BD092491BE0924A1BF0924B1B012FC3
:102600000295000F000F007C0C5CA12FB0E0BD8B89
:10261000AC8BA3E0B0E0012E02C0AA0FBB1F0A944E
:10262000E2F725E335E00E942B82DC01CB01029624
:10263000A11DB11D8C879D87AE87BF8780E593EC78
:10264000A0E0B0E004C0B595A795979587951A9539
:10265000D2F7888B998BAA8BBB8B10E018861986D2
:102660001A861B86A8E02A2E312CAC89BD892A1A2D
:102670003B0A988D191709F436C1402F64EF8EEE8E
:102680000E9492106C857D858E859F850E948F5358
:1026900023E0AE014F5F5F4F66EF8EEE0E94A91000
:1026A000E0913A1BF0913B1BE05AFF409F01DF0194
:1026B0000E9414826B017C018091321B9091331B2C
:1026C0009F8B8E8BA090301BB090311B2091341BC0
:1026D0003091351B0E9414822B013C013DE0759422
:1026E0006794579447943A95D1F7A091361BB091CF
:1026F000371BA70196016CE05595479537952795AF
:102700006A95D1F70E943D82BB2797FDB095AB2F0C
:10271000480E591E6A1E7B1E92E0490E511C611C18
:10272000711CB2E07594679457944794BA95D1F7A9
:10273000A0E85A0E611C711CA091421BB091431B72
:10274000A30192010E943282DC01CB012FE0B695F9
:10275000A795979587952A95D1F78C839D83AE830E
:10276000BF8329818A8190E0A0E0B0E04424582E04
:10277000692E7A2E622A8B81482A022C04C0759415
:102780006794579447940A94D2F74501AA2497FC7A
:10279000A094BA2C42E0880C991CAA1CBB1C4A9538
:1027A000D1F7A091381BB091391BA70196010E9467
:1027B0003D826B017C0157E1F594E794D794C7946F
:1027C0005A95D1F72E893F89DF010E941482EBE0F0
:1027D0009595879577956795EA95D1F7C60ED71E9B
:1027E000E81EF91E8C0C9D1CAE1CBF1C0C8804C07E
:1027F000880C991CAA1CBB1C0A94D2F792E0890E83
:10280000911CA11CB11CF2E0B594A79497948794F5
:10281000FA95D1F7481859086A087B08A301920174
:10282000688979898A899B890E94458297FD0DC0B4
:10283000660F771F881F991F2C813D814E815F8114
:102840000E947D8249015A010CC02C813D814E813C
:102850005F810E947D8249015A01880C991CAA1C43
:10286000BB1C9927B7FC9A958B2D7A2D692D9B015E
:10287000AC010E9445829B01AC01AEEDBBE00E9421
:1028800032826C01FF24D7FCF094EF2CA3E4B3EE6A
:10289000A50194010E944082BB2797FDB095AB2F04
:1028A000C80ED91EEA1EFB1EAFECCA0EAEE0DA1E41
:1028B000E11CF11CA4E0F594E794D794C794AA9581
:1028C000D1F7C80CD91CEA1CFB1C88859985AA8500
:1028D000BB858C0D9D1DAE1DBF1D88879987AA875E
:1028E000BB871F5FC6CE112391F0212F30E040E05F
:1028F00050E0688579858A859B850E947D8220933A
:102900004C1B30934D1B40934E1B50934F1BA98D76
:10291000AA2389F160914C1B70914D1B80914E1B35
:1029200090914F1B611571058105910521F10E9460
:10293000767F20E836EE45EC57E40E94D77E21E012
:102940003EED42E45EE30E94B7819B01AC0160E092
:1029500070E080E89FE30E940C7E2BE43AE34DEBAD
:1029600057E30E94D77E6093501B7093511B809356
:10297000521B9093531B6A960FB6F894DEBF0FBE9E
:10298000CDBFDF91CF911F910F91FF90EF90DF901E
:10299000CF90BF90AF909F908F907F906F905F90FF
:1029A0004F903F902F9008950F931F93CF93DF93F5
:1029B00000D000D000D0CDB7DEB78E010F5F1F4F23
:1029C00086E0F80111928A95E9F780918A1A8111BF
:1029D00013C040E061E386EA0E9492104AE06CE294
:1029E00086EA0E94921081E080938A1A6CE77EE367
:1029F00080E090E00E948F5348E06DE286EA0E94FA
:102A000092106CE77EE380E090E00E948F5326E016
:102A1000A80162E386EA0E94A91047E06DE286EA17
:102A20000E9492108A8190E0982F88272981822B1A
:102A30009093851A8093841A2C8130E0322F2227BC
:102A40004B81242B3093871A2093861A4E8150E0B5
:102A5000542F44276D81462B5093891A4093881A2E
:102A60005F934F933F932F939F938F9383E994E0CA
:102A70009F938F930E94DC880FB6F894DEBF0FBE41
:102A8000CDBF26960FB6F894DEBF0FBECDBFDF9147
:102A9000CF911F910F910895CF92DF92EF92FF9205
:102AA0000F931F93CF93DF93CDB7DEB72A970FB65F
:102AB000F894DEBF0FBECDBF8E010F5F1F4F86E0C3
:102AC000F80111928A95E9F741E062E08CE30E94F7
:102AD000921048E560E08CE30E94921062E174E39A
:102AE00080E090E00E948F5326E0A80163E08CE331
:102AF0000E94A91043E062E08CE30E9492100981D9
:102B000010E0102F00278A81082B1093611A009380
:102B1000601AEB80F12CFE2CEE248C81E82AF092D6
:102B2000631AE092621ACD80D12CDC2CCC248E81E9
:102B3000C82AD092651AC092641AB801882777FD16
:102B40008095982F0E94767F9B01AC01B701882762
:102B500077FD8095982F2F83388749875A870E9461
:102B6000767F2F81388549855A850E94807E20EEA8
:102B70003EE245E652E40E94548120E030E044E326
:102B800053E40E940D7E9F938F937F936F93DF9208
:102B9000CF92FF92EF921F930F9381EA94E09F935D
:102BA0008F930E94DC880FB6F894DEBF0FBECDBFB6
:102BB0002A960FB6F894DEBF0FBECDBFDF91CF913E
:102BC0001F910F91FF90EF90DF90CF900895CF93DA
:102BD000DF93EC01888199810097F9F0893A9E4052
:102BE00021F01982188283E063C08DE399E00E948E
:102BF000FD4A892BE1F080912D0990912E0993FDDA
:102C000018C080912D0990912E0994FD43C08091A8
:102C10002D0990912E0995FD44C060E870E08DE388
:102C200099E00E94D24A89EA9EE09983888381E0F4
:102C30003FC08091611F82FFE4CF21E048E061E066
:102C400083E00E9465128091531B8F938091521BE9
:102C50008F938091511B8F938091501B8F93809104
:102C60004F1B8F9380914E1B8F9380914D1B8F93A1
:102C700080914C1B8F9385E99DE09F938F930E94D9
:102C8000EE888DB79EB70A960FB6F8949EBF0FBE1A
:102C90008DBFB7CF8091611F83FFB9CF0E94D4143D
:102CA000B6CF8091611F84FFB8CF0E944C15B5CF7D
:102CB000DF91CF910895CF93C82F8CEE0E940554D9
:102CC0008C2F0E94105465E375E080E090E00E9434
:102CD0008F538DEE0E9405540E942154C82F0E94EC
:102CE0002B542C2F30E0322F2227A901482BCA0168
:102CF000CF910895CF93DF93C82F8CEE0E94055497
:102D00008C2F0E94105462E174E380E090E00E94F6
:102D10008F538CEE0E94055480E00E94105465E3AE
:102D200075E080E090E00E948F538DEE0E94055484
:102D30000E942154C82F0E942154D82F0E942B5446
:102D40004D2F50E060E070E0762F652F542F442720
:102D50006C2B482BCB01BA01DF91CF9108952F92B4
:102D60003F924F925F926F927F928F929F92AF921B
:102D7000BF92CF92DF92EF92FF920F931F93CF9368
:102D8000DF93CDB7DEB7CD54D1090FB6F894DEBFCF
:102D90000FBECDBF8091000290910102892BD1F12D
:102DA00010920102109200028CEE0E9405548EE1F6
:102DB0000E9410546BE17EE480E090E00E948F530B
:102DC00082EA0E945B1690933A098093390984EA5B
:102DD0000E945B16909338098093370986EA0E9417
:102DE0005B16909336098093350988EA0E945B163A
:102DF00090933409809333098AEA0E945B1690937A
:102E00003209809331098CEA0E945B169093300955
:102E100080932F0988E40E947A166FAB78AF89AF50
:102E20009AAF88E50E947A164B015C0180913109C6
:102E30009091320920E030E040E050E0BA0126965F
:102E40002FAF269727963FAF279728964FAF289703
:102E500029965FAF29972A966FAF2A972B967FAF57
:102E60002B979C0140E050E060E070E080E090E053
:102E700008E00E9419840E94D2833901B42FA52F43
:102E8000F62FE72F8C019401A50160E070E080E04F
:102E900090E05301CB2EDA2EEF2EFE2E0E945084AE
:102EA00029833A832A011B014C01B101C40131502D
:102EB00041095F4F6F4F7F4F8F4F9F4FA1E0B0E0B1
:102EC0002596BFAFAEAF259721153F4F4F4F5140CD
:102ED000610571058105910509F020F425961FAE65
:102EE0001EAE259725966EAC7FAC259780912F0955
:102EF000909130095C01C12CD12CE12CF12C00E027
:102F000010E029813A81A201B101C4010E94F58239
:102F1000D22EE32EF42E052F162FB72FF82FE92FE0
:102F2000A0E00E94778484F42150310940485F4F2B
:102F30006F4F7F4F8F4F9F4FD22EE32EF42E052FD2
:102F4000162FB72FF82FE92F2D2D3E2D4F2D502F57
:102F5000612F7B2F8F2F9E2F07E10E9432842B8FB2
:102F60003C8F4D8F5E8F6F8F78A389A39AA32053D8
:102F7000384F4F4F5F4F6F4F7F4F8F4F9F4F2B8B70
:102F80003C8B4D8B5E8B6F8B788F898F9A8F205601
:102F9000304F4F4F5F4F6F4F7F4F8F4F9F4F243DAD
:102FA000304341055105610571058105910541F0E9
:102FB00038F025966EAC7FAC2597FFEF6F1A7F0A2D
:102FC00080913709909138099C0140E050E060E021
:102FD00070E080E090E000E10E9419842B833C8344
:102FE0004D835E836A8779878F8398874091330901
:102FF00050913409A980BA806201710184019A015B
:1030000040E050E060E070E080E090E00E94F582F7
:10301000D22EE32EF42E052F162FB72FF82FE92FDF
:10302000A0E00E9477845CF4AFE70E945984D22E1E
:10303000E32EF42E052F162FB72FF82FE92F2D2D65
:103040003E2D4F2D502F612F7B2F8F2F9E2F07E06E
:103050000E94328459016A017B018C012B813C81E1
:103060004D815E816A8579858F8198850E94508423
:103070002B833C834D835E836F8378878F87988B08
:103080002E5F3F4F434051096E4F7F4F8F4F9F4FF1
:1030900022303105494F5F4F64407105810591052C
:1030A00021F018F01FEF611A710A8091390990918F
:1030B0003A09BC0180E090E020E030E840E050E0D8
:1030C0000E944E8329873A874B875C876A8B798B6E
:1030D0008D879E874091350950913609A980BA8025
:1030E0006201710184019A0140E050E060E070E00B
:1030F00080E090E00E94F582D22EE32EF42E052F80
:10310000162FB72FF82FE92FA0E00E94778484F4C0
:1031100021503F4F4F4F5F4F6F4F7F4F8F4F9F4F0C
:10312000D22EE32EF42E052F162FB72FF82FE92FCE
:103130002D2D3E2D4F2D502F612F7B2F8F2F9E2F0A
:1031400008E00E94328459016A017B018C012985C3
:103150003A854B855C856A8979898D859E850E9433
:10316000508429873A874B875C876D877E87898B58
:103170009A8B2F5F3F4F41405109610971098109C5
:103180009109213030484C4F5F47614071058105FE
:10319000910521F018F0BFEF6B1A7B0A2B893C894F
:1031A0004D895E896F89788D898D9A8D2F3C374046
:1031B00041055105610571058105910511F00CF07E
:1031C000A5C1A980BA806201710184019501A201A3
:1031D000B101C4010E94F582A12CB12CC12C10E8D0
:1031E000D12EE12CF12C00E010E00E94B8822BAF30
:1031F0003CAF4DAF5EAF6FAF21967FAF2197229668
:103200008FAF229723969FAF2397AB8CBC8CCD8C2E
:10321000DE8CEF8CF8A009A11AA19501A601B701D7
:10322000C8010E94F58259016A017B01E82F192F1C
:1032300002E00E9419840E2F0E94508469017A01D5
:10324000162F272EF82FE92F322E8D2C942EAF2CEF
:10325000B62E072F582EB92FA0E00E9477845CF479
:10326000A1E00E945984322E832E942EA52EB62ED4
:10327000072F582EB92F232D382D492D5A2D6B2D60
:10328000702F852D9B2F01E00E9432842E962FAF48
:103290002E972D963FAF2D9749A75AA76BA77CA7CE
:1032A0008DA79EA7522E432E4BA35CA36DA37EA396
:1032B0008FA398A7B22D9601A701612F722D8F2F92
:1032C0009E2FA0E00E9477844CF4A3E00E945984D2
:1032D00069017A01162FB72FF82FE92F9601A70160
:1032E000612F7B2F8F2F9E2F02E00E9432842FA709
:1032F00038AB49AB5AAB6BAB7CAB8DAB9EAB19011A
:103300004A01B62FA72F24968FAF2497F92F2B8928
:103310003C894D895E896F89788D898D9A8D24329B
:103320003A4F4F4F5F4F6F4F7F4F8F4F9F4F0CF074
:103330008CC02B8D3C8D4D8D5E8D6F8D78A189A1BC
:103340009AA12455324F4F4F5F4F6F4F7F4F8F4F92
:103350009F4F59016A017B018C010E94F58219017E
:103360004A01B62FA72FFC0103E00E9419845101E6
:103370006401EB2EFA2E8F010E94658459016A01C7
:103380007B018C012E962FAD2E972D963FAD2D975C
:1033900049A55AA56BA57CA58DA59EA50E94508424
:1033A000522E432E4BA35CA36DA37EA38FA398A79D
:1033B0009101A4016B2F7A2FCF0102E00E941984A2
:1033C00051016401EB2EFA2E8F010E94658402E008
:1033D0000E9419840E2F0E946584F22E032F142F51
:1033E000D52EE62EB72FF82FE92FA0E00E94778484
:1033F0005CF4A1E00E945984F22E032F142FD52EE5
:10340000E62EB72FF82FE92F2F2D302F412F5D2DCE
:103410006E2D7B2F8F2F9E2F01E00E943284590149
:103420006A017B018C012FA538A949A95AA96BA96A
:103430007CA98DA99EA90E94508419014A01B62F2A
:10344000A72F24968FAF2497F92F2B813C814D8194
:103450005E816F8178858F859889A52CB42CCBA04F
:10346000DCA0EDA0FEA00FA118A50E9465842B830F
:103470003C834D835E836F8378878F87988B298504
:103480003A854B855C856D857E8589899A89510150
:103490006401EB2EFA2E24960FAD24971F2F0E9465
:1034A000658429873A874B875C876D877E87898B00
:1034B0009A8B2B893C894D895E896F89788D898D9E
:1034C0009A8DABACBCACCDACDEACEFAC2196FFAC16
:1034D000219722960FAD229723961FAD23970E9426
:1034E00065842056304F4F4F5F4F6F4F7F4F8F4F48
:1034F0009F4F243D3043410551056105710581050C
:10350000910521F018F02FEF621A720A6FA978ADB9
:1035100089AD9AADAB01BC0180E090E0DC0124965E
:103520004FAF249725965FAF259726966FAF2697C6
:1035300027967FAF279728968FAF289729969FAF1A
:1035400029972A96AFAF2A972B96BFAF2B97A984BE
:10355000BA84CB84DC84ED84FE8409891A899A01BB
:10356000AB0160E070E080E090E00E94F582F22E16
:10357000032F142FD52EE62EB72FF82FE92FA0E01A
:103580000E94778484F421503109404E5F4F6F4F81
:103590007F4F8F4F9F4FF22E032F142FD52EE62EE5
:1035A000B72FF82FE92F2F2D302F412F5D2D6E2DA6
:1035B0007B2F8F2F9E2F05E10E943284AB80BC8031
:1035C000CD80DE80EF80F8840F8518890E946584A5
:1035D000F22E032F142FD52EE62EB72FF82FE92F1A
:1035E000A0E00E94778484F4215030484F4F5F4F11
:1035F0006F4F7F4F8F4F9F4FF22E032F142FD52EDB
:10360000E62EB72FF82FE92F2F2D302F412F5D2DCC
:103610006E2D7B2F8F2F9E2F0FE00E943284690129
:103620007A018B018A83998329011A014B015C017C
:10363000285E3340410951096109710981099109E5
:10364000283D304D414051056105710581059105C9
:1036500021F018F0BFEF6B1A7B0A0E94085467280C
:1036600059F09601A701B8018A8199810E94D283FD
:1036700029011A014B015C019201A101B401C501AC
:103680000E94707F20E030E048EC52E40E94D77E38
:10369000C35BDF4F0FB6F894DEBF0FBECDBFDF9127
:1036A000CF911F910F91FF90EF90DF90CF90BF903F
:1036B000AF909F908F907F906F905F904F903F90D2
:1036C0002F9008954F925F926F927F928F929F9268
:1036D000AF92BF92CF92DF92EF92FF922B013C010B
:1036E00069017A0123EC35EF4CE851E4C701B601DA
:1036F0000E9454814B015C0128EB3EE143E753E417
:10370000C701B6010E940D7E9B01AC01C501B40149
:103710000E94D77E0E94447F4B015C0120E030E094
:1037200048EC52E4C301B2010E94D77E21E835E99A
:1037300043EC50E40E945481A50194010E945481FD
:103740004B015C0123E333E948E853E4C701B601C8
:103750000E940D7E9B01AC01C501B4010E94D77E81
:1037600023E333EB48E553E40E945481FF90EF904C
:10377000DF90CF90BF90AF909F908F907F906F9091
:103780005F904F9008954F925F926F927F928F92C9
:103790009F92AF92BF92CF92DF92EF92FF92690118
:1037A0007A010E94D68020E030E040E050E40E94A0
:1037B0000C7E22E93CE54EED5EE30E94D77E4B0194
:1037C0005C0123EC35EF4CE851E4C701B6010E94DF
:1037D00054812B013C0128EB3EE143E753E4C70150
:1037E000B6010E940D7E9B01AC01C301B2010E9493
:1037F000D77E9B01AC01C501B4010E940D7E6B0117
:103800007C0128EB3EE143E753E40E9454814B01E5
:103810005C01A701960163EC75EF8CE891E40E94CE
:103820000C7E9B01AC01C501B4010E94D77EFF90C4
:10383000EF90DF90CF90BF90AF909F908F907F9050
:103840006F905F904F9008954F925F926F927F922A
:103850008F929F92AF92BF92CF92DF92EF92FF92A0
:103860002B013C0169017A0123EC35EF4CE851E46E
:10387000C701B6010E9454814B015C0128EB3EE177
:1038800043E753E4C701B6010E940D7E9B01AC01E2
:10389000C501B4010E94D77E0E94447F4B015C01A8
:1038A00020E030E048EC52E4C301B2010E94D77E30
:1038B000A50194010E94548120E030E040E251E4EF
:1038C0000E940C7E24EE38E34EE05FE30E945481B8
:1038D0009B01AC01C701B6010E940D7EFF90EF90E5
:1038E000DF90CF90BF90AF909F908F907F906F9020
:1038F0005F904F900895CF92DF92EF92FF920F93D7
:103900001F93CF93DF9380E80E9405548AEF0E94B3
:1039100010548FE00E94105465E375E080E090E061
:103920000E948F5381E80E9405540E942154C82FA1
:103930000E9421540E942154D82F0E9421540E9499
:103940002154182F0E9421540E942B54082F0E94AA
:103950002B5480E80E9405548CEF0E94105489EC8F
:103960000E94105465E375E080E090E00E948F5360
:1039700081E80E9405540E942154D82E0E942154AF
:10398000C82E0E9421540E942154F82E0E942154D6
:10399000E82E0E942B541F92CF921F92DF921F920B
:1039A0000F931F921F931F92DF931F92CF931F922B
:1039B000EF921F92FF9286EB94E09F938F930E9469
:1039C000DC880E9408548DB79EB742960FB6F894D3
:1039D0009EBF0FBE8DBF20E030E040E050E060E0D1
:1039E00070E080E090E0DF91CF911F910F91FF9008
:1039F000EF90DF90CF9008950F931F93CF93DF93B5
:103A0000EC0180E80E940554209741F085EE0E9469
:103A1000105461E077E980E090E007C083EE0E94F7
:103A2000105469E97AEB81E090E00E948F5381E8BD
:103A30000E9405540E942154182F0E942154082FDF
:103A40000E942B540E940854602F70E0712B6C7FF1
:103A500080E090E0CD2B69F00E94747F20E030E0A0
:103A60004AEF5AE30E94548120E030E040EC50E4F9
:103A70000CC00E94747F22E538EB4FE25BE30E94AA
:103A8000548126E636E64BE352E40E940C7EDF9139
:103A9000CF911F910F9108950F931F93CF93DF93B1
:103AA000729A8091400283FF08C08EE40E94A25364
:103AB000811195C0C0E5D0E008C0C0E5D0E00E940B
:103AC000180921972097D9F7F0CF0E94180921975C
:103AD0002097D9F78FE40E94A2530E942154982F77
:103AE00092959695969593709130A9F440916B2399
:103AF00050916C2360916D2370916E234F5F5F4FE7
:103B00006F4F7F4F40936B2350936C2360936D23D3
:103B100070936E2316C09230A0F040916F235091A5
:103B2000702360917123709172234F5F5F4F6F4FCD
:103B30007F4F40936F235093702360937123709352
:103B40007223082F0F730E942154182F0E942154B2
:103B5000D82F0E942B54C82F0E94085480914002F5
:103B600083FF7298602F70E0762F6627610F711DBA
:103B700080E090E00E94747F20E134E048EC5BE359
:103B80000E9454816093551B7093561B8093571B62
:103B90009093581B6D2F70E0762F66276C0F711D68
:103BA000769567957695679580E090E00E94747FA2
:103BB00024EA3CEF44E25CE30E94548120E030E0E0
:103BC00040E252E40E940C7E6093E4277093E52764
:103BD0008093E6279093E72780E090E015C08091DE
:103BE000672390916823A0916923B0916A2301967D
:103BF000A11DB11D8093672390936823A09369232F
:103C0000B0936A2381E090E0DF91CF911F910F91F3
:103C100008957298729A8EE40E94A25380EA0E94DC
:103C2000105480E00E94105480E00E9410548FE4F1
:103C30000E94A2530E942154829586958695837096
:103C40008130A9F440916B2350916C2360916D23D6
:103C500070916E234F5F5F4F6F4F7F4F40936B2389
:103C600050936C2360936D2370936E2316C0823043
:103C7000A0F040916F235091702360917123709157
:103C800072234F5F5F4F6F4F7F4F40936F2350936F
:103C9000702360937123709372231F928F9385EE2C
:103CA00094E09F938F930E94DC888EE40E94A2533D
:103CB00080E80E94105480E00E94105480E00E942E
:103CC00010540E9408540F900F900F900F9080E0B6
:103CD00090E0089589E29DE09F938F930E94EE8883
:103CE000809162020F900F90882361F01F928F9352
:103CF00086E29DE09F938F930E94EE880F900F9035
:103D00000F900F90089581E09DE09F938F930E9404
:103D1000EE8889ED9CE09F938F930E94EE8882EB62
:103D20009CE09F938F930E94EE8887E79CE09F938F
:103D30008F930E94EE8885E49CE09F938F930E946E
:103D4000EE8889E09CE09F938F930E94EE8883EE3B
:103D50009BE09F938F930E94EE888DEA9BE09F9358
:103D60008F930E94EE888091611F9091621F8270F4
:103D700091702DB73EB7205F3F4F0FB6F8943EBF0E
:103D80000FBE2DBF892B41F08DE79BE09F938F9352
:103D90000E94EE880F900F9081E59BE09F938F9398
:103DA0000E94EE8888E29BE09F938F930E94EE88AA
:103DB0008DEF9AE09F938F930E94EE888EEC9AE0AD
:103DC0009F938F930E94EE888CE99AE09F938F9344
:103DD0000E94EE888BE69AE09F938F930E94EE8874
:103DE00087E39AE09F938F930E94EE8887E09AE0A2
:103DF0009F938F930E94EE888BED99E09F938F9312
:103E00000E94EE888CEA99E09F938F930E94EE883F
:103E100083E799E09F938F930E94EE888AE399E06D
:103E20009F938F930E94EE8883E099E09F938F93F6
:103E30000E94EE8882ED98E09F938F930E94EE8817
:103E400083EA98E09F938F930E94EE8884E798E03E
:103E50009F938F930E94EE888DB79EB780960FB682
:103E6000F8949EBF0FBE8DBF8DE498E09F938F9313
:103E70000E94EE8887E198E09F938F930E94EE88DE
:103E80008EEE97E09F938F930E94EE8883EB97E0EE
:103E90009F938F930E94EE8888E897E09F938F937B
:103EA0000E94EE882DB73EB7265F3F4F0FB6F894BD
:103EB0003EBF0FBE2DBF089585EF94E00C9412898C
:103EC0004F925F926F927F928F929F92AF92BF922A
:103ED000CF92DF92EF92FF92CF93DF93CDB7DEB711
:103EE00028970FB6F894DEBF0FBECDBF8091632335
:103EF00090916423A0916523B091662389839A836E
:103F0000AB83BC834090632350906423609065230F
:103F1000709066238091632390916423A091652320
:103F2000B09166238D839E83AF83B88760916323AE
:103F30007091642380916523909166232CE3822EF7
:103F4000912CA12CB12CA50194010E947D827F931C
:103F50006F9330E1C32E3EE0D32EE12CF12C6D8126
:103F60007E818F819885A70196010E947D82A5019F
:103F700094010E947D823F932F9340E8842E41E577
:103F8000942EAA24A394B12CC301B201A5019401DB
:103F90000E947D82A70196010E947D823F932F930C
:103FA00069817A818B819C81A50194010E947D8227
:103FB0003F932F9382E697E09F938F930E94EE8822
:103FC0000FB6F894DEBF0FBECDBF28960FB6F8949B
:103FD000DEBF0FBECDBFDF91CF91FF90EF90DF909E
:103FE000CF90BF90AF909F908F907F906F905F9099
:103FF0004F900895E9EAF0E3808191818234924400
:1040000079F0E95AF043FF93EF9384E497E09F93AC
:104010008F930E94EE880F900F900F900F9008954D
:104020003A96E53F81E4F80738F30895CF93DF939C
:10403000EC018C9A0E94FB099F938F937F936F935F
:1040400088E397E09F938F930E94EE880F900F90E4
:104050000F900F900F900F90209719F00E94F30A85
:1040600008C086E397E09F938F930E94EE880F909D
:104070000F9081E00E94AC092091670230916802A4
:104080004091690250916A020E9454819F938F93DC
:104090007F936F938AE297E09F938F930E94EE88BD
:1040A0000F900F900F900F900F900F90209719F096
:1040B0000E94F30A08C088E297E09F938F930E94C2
:1040C000EE880F900F9082E00E94AC09209163026D
:1040D0003091640240916502509166020E945481C1
:1040E0009F938F937F936F938CE197E09F938F9330
:1040F0000E94EE880F900F900F900F900F900F90EE
:10410000209719F00E94F30A08C08AE197E09F9374
:104110008F930E94EE880F900F9083E00E94AC096D
:104120009F938F937F936F938BE097E09F938F93F1
:104130000E94EE888C980F900F900F900F900F9028
:104140000F90209719F00E94F30A08C089E097E0C9
:104150009F938F930E94EE880F900F908091611F24
:1041600087FF7FC021E042E161E080ED0E94785549
:104170009F938F937F936F938CEF96E09F938F9392
:104180000E94EE880F900F900F900F900F900F905D
:10419000209719F00E94F30A08C08AEF96E09F93D7
:1041A0008F930E94EE880F900F9021E042E162E031
:1041B00080ED0E9478559F938F937F936F938DEE40
:1041C00096E09F938F930E94EE880F900F900F9030
:1041D0000F900F900F90209719F00E94F30A08C0DB
:1041E0008BEE96E09F938F930E94EE880F900F9036
:1041F00021E042E163E080ED0E9478559F938F9328
:104200007F936F938EED96E09F938F930E94EE883D
:104210000F900F900F900F900F900F90209719F024
:104220000E94F30A08C08CED96E09F938F930E9442
:10423000EE880F900F9021E042E164E080ED0E9453
:1042400078559F938F937F936F938FEC96E09F9316
:104250008F930E94EE880F900F900F900F900F9009
:104260000F90CD2B21F4DF91CF910C94F30ADF91C5
:10427000CF9108950F931F93CF93DF93882389F0F5
:1042800049E050E06FEF70E088ED97E20E944A88C5
:1042900049E050E06AE070E088ED97E20E94318AE0
:1042A00013C0C8EDD7E20AEC16E089911F928F93F4
:1042B0001F930F930E94EE880F900F900F900F9016
:1042C00087E2C03ED80789F7DF91CF911F910F9108
:1042D0000C94F30ACF92DF92EF92FF92CF93DF9389
:1042E0006B017C0160FF11C080E195E09F938F938B
:1042F0008EE39DE09F938F930E94EE880F900F9026
:104300000F900F9081E090E002C080E090E0C1FE4D
:1043100009C0EC01219643E259E065E175E00E9495
:104320001E0FCE01C2FE09C0EC01219643E259E006
:104330006DE175E00E941E0FCE01C3FE09C0EC01C5
:10434000219643E259E065E275E00E941E0FCE011E
:10435000C4FE09C0EC01219643E259E069E275E030
:104360000E941E0FCE01C5FE09C0EC01219643E25A
:1043700059E06CE275E00E941E0FCE01C6FE09C036
:10438000EC01219643E259E060E375E00E941E0FC4
:10439000CE01C7FE09C0EC01219643E259E066E375
:1043A00075E00E941E0FCE01D0FE09C0EC012196DF
:1043B00043E259E06EE375E00E941E0FCE01D1FE8C
:1043C00009C0EC01219643E259E066E475E00E94E1
:1043D0001E0FCE01D2FE09C0EC01219643E259E046
:1043E0006AE475E00E941E0FCE012091611F30919A
:1043F000621F24703270232B59F0D3FE09C0EC01E8
:10440000219643E259E060E575E00E941E0FCE015F
:104410002091611F23FF0BC0D4FE09C0EC0121963F
:1044200043E259E065E575E00E941E0FCE01209140
:10443000611F24FF0BC0D5FE09C0EC01219643E2A9
:1044400059E06BE575E00E941E0FCE01D6FE0CC050
:1044500043E259E063E675E0DF91CF91FF90EF9082
:10446000DF90CF900C941E0FCD28CE28CF2841F49A
:1044700085EC96E09F938F930E94EE880F900F90AB
:10448000DF91CF91FF90EF90DF90CF9008950F9341
:104490001F93CF93DF938C01C0E0D0E0011511058D
:1044A00009F482C060EC76E0C8010E942988892B5B
:1044B00009F4C16068EB76E0C8010E942988892B65
:1044C00009F4C26060EB76E0C8010E942988892B5C
:1044D00009F4C4606CEA76E0C8010E942988892B3F
:1044E00009F4C86069EA76E0C8010E942988892B2E
:1044F00009F4C06165EA76E0C8010E942988892B29
:1045000009F4C0626FE976E0C8010E942988892B0E
:1045100009F4C06467E976E0C8010E942988892B04
:1045200009F4C0686FE876E0C8010E942988892BE9
:1045300009F4D1606BE876E0C8010E942988892BD4
:1045400009F4D26065E876E0C8010E942988892BC9
:1045500009F4D46060E876E0C8010E942988892BBC
:1045600009F4D8606AE776E0C8010E942988892B9F
:1045700009F4D06162E776E0C8010E942988892B9E
:1045800009F4D06267E676E0C8010E942988892B89
:1045900009F4D064609160027091610280E090E063
:1045A0000E943D888C017ACFCE01DF91CF911F917F
:1045B0000F910895CF92DF92EF92FF92CF93DF9306
:1045C0006B017C0160FF11C08EE695E09F938F9395
:1045D0008EE39DE09F938F930E94EE880F900F9043
:1045E0000F900F9081E090E002C080E090E0209179
:1045F000611F20FF0BC0C2FE09C0EC01219643E2FF
:1046000059E062E775E00E941E0FCE01C1FE09C0AD
:10461000EC01219643E259E066E775E00E941E0F27
:10462000CE01C3FE09C0EC01219643E259E06EE8D9
:1046300075E00E941E0FCE01C4FE09C0EC01219658
:1046400043E259E069E775E00E941E0FCE01C5FE06
:1046500009C0EC01219643E259E06CE775E00E9445
:104660001E0FCE01C6FE09C0EC01219643E259E0BF
:1046700062E875E00E941E0FCE01C7FE09C0EC0182
:10468000219643E259E068E875E00E941E0FCE01D2
:10469000D0FE09C0EC01219643E259E06BE875E0D9
:1046A0000E941E0FCE01D1FE09C0EC01219643E20B
:1046B00059E060E975E00E941E0FCE01D2FE09C0EC
:1046C000EC01219643E259E067E975E00E941E0F74
:1046D000CE01D3FE09C0EC01219643E259E06AE91C
:1046E00075E00E941E0FCE01D4FE09C0EC01219698
:1046F00043E259E06FE975E00E941E0FCE01D5FE3E
:1047000009C0EC01219643E259E066EA75E00E9497
:104710001E0FCE012091611F21FF0BC0D6FE09C0E4
:10472000EC01219643E259E06DEA75E00E941E0F0C
:10473000CE012091611F3091621F30FF0BC0F4FE4B
:1047400009C0EC01219643E259E060EB75E00E945C
:104750001E0FCE012091611F3091621F30FF0BC0F0
:10476000F5FE09C0EC01219643E259E063EB75E0E8
:104770000E941E0FCE012091611F3091621F30FFF9
:104780000BC0F6FE09C0EC01219643E259E069EB4B
:1047900075E00E941E0FCE01D7FE09C0EC012196E4
:1047A00043E259E064EC75E00E941E0FCE01E0FE8A
:1047B00009C0EC01219643E259E069EC75E00E94E2
:1047C0001E0FCE01E1FE09C0EC01219643E259E043
:1047D0006CEC75E00E941E0FCE01E2FE09C0EC01F8
:1047E000219643E259E06FEC75E00E941E0FCE0166
:1047F0002091611F27FF0BC0E3FE09C0EC01219649
:1048000043E259E062ED75E00E941E0FCE01209157
:10481000611F27FF0BC0E4FE09C0EC01219643E2B3
:1048200059E066ED75E00E941E0FCE012091611FD8
:1048300027FF0BC0E5FE09C0EC01219643E259E0D9
:104840006AED75E00E941E0FCE012091611F27FFC7
:104850000BC0E6FE09C0EC01219643E259E06EED83
:1048600075E00E941E0FCE012091611F22FF0BC038
:10487000E7FE09C0EC01219643E259E066E876E0E4
:104880000E941E0FCE012091611F22FF0BC0F0FE7F
:1048900009C0EC01219643E259E062EE75E00E9406
:1048A0001E0FCE012091611F3091621F30FF0BC09F
:1048B000F1FE09C0EC01219643E259E065EE75E096
:1048C0000E941E0FCE012091611F3091621F30FFA8
:1048D0000BC0F2FE09C0EC01219643E259E06DEEF7
:1048E00075E00E941E0FCE012091611F3091621F62
:1048F00031FF0EC0F3FE0CC043E259E066EF75E0F5
:10490000DF91CF91FF90EF90DF90CF900C941E0F2E
:10491000CD28CE28CF2841F482E696E09F938F934E
:104920000E94EE880F900F90DF91CF91FF90EF9053
:10493000DF90CF900895CF92DF92EF92FF92CF93C6
:10494000DF93EC016DE576E00E942988892BA9F5BB
:104950008091611F82FD08C06DE4C62E60E8D62EEE
:1049600064E0E62EF12C07C05DE4C52E50E8D52E9C
:1049700054E8E52EF12C81FF02C06894D6F826E0B9
:104980004AE250E06BE270E089E290E00E94B250AF
:1049900081E090E00E94810A882311F06894C4F8B5
:1049A0008091611F9091621F90FF02C026E0F22A61
:1049B00091FF27C16894F3F824C1C12CD12C760152
:1049C00020C169E576E0CE010E942988892B11F487
:1049D0006894C0F865E576E0CE010E942988892BAD
:1049E00011F46894C2F862E576E0CE010E9429884D
:1049F000892B11F46894C1F860E576E0CE010E943D
:104A00002988892B11F46894C3F86DE476E0CE010F
:104A10000E942988892B11F46894C4F867E476E031
:104A2000CE010E942988892B11F46894C5F861E4AD
:104A300076E0CE010E942988892B11F46894C6F88B
:104A40006EE376E0CE010E942988892B11F46894E8
:104A5000C7F869E376E0CE010E942988892B11F41A
:104A60006894D0F862E376E0CE010E942988892B11
:104A700011F46894D1F86FE276E0CE010E942988A3
:104A8000892B11F46894D2F86AE276E0CE010E9494
:104A90002988892B11F46894D3F863E276E0CE017B
:104AA0000E942988892B11F46894D4F86CE176E08F
:104AB000CE010E942988892B11F46894D5F869E108
:104AC00076E0CE010E942988892B11F46894D6F8EB
:104AD00064E176E0CE010E942988892B11F4689464
:104AE000D7F861E176E0CE010E942988892B11F484
:104AF0006894E0F86EE076E0CE010E942988892B68
:104B000011F46894E1F86BE076E0CE010E94298808
:104B1000892B11F46894E2F867E076E0CE010E94F8
:104B20002988892B11F46894E3F863E076E0CE01DC
:104B30000E942988892B11F46894E4F86FEF75E0DE
:104B4000CE010E942988892B11F46894E5F86BEF57
:104B500075E0CE010E942988892B11F46894E6F84B
:104B600069EF75E0CE010E942988892B11F46894C1
:104B7000E7F866EF75E0CE010E942988892B11F4D1
:104B80006894F0F86EEE75E0CE010E942988892BBA
:104B900011F46894F1F865EE75E0CE010E94298861
:104BA000892B11F46894F2F86CED75E0CE010E9447
:104BB0002988892B11F46894F3F869ED75E0CE012A
:104BC0000E942988892B11F46894F4F863ED75E04C
:104BD000CE010E942988892B11F46894F5F868ECBD
:104BE00075E0CE010E942988892B11F46894F6F8AB
:104BF000609160027091610280E090E00E943D88C7
:104C0000EC01209709F0DDCEC701B601DF91CF910D
:104C1000FF90EF90DF90CF90089588EB95E09F9301
:104C20008F930E94EE880E945C1F86E79AE19F9313
:104C30008F9380EB95E09F938F930E94EE888CEA90
:104C400095E09F938F930E94EE8880E00E943A2126
:104C500087EA95E09F938F930E94EE880E94460F0B
:104C60008091611F2DB73EB7265F3F4F0FB6F89476
:104C70003EBF0FBE2DBF80FF05C041E061E081E077
:104C80000E94F0100E94601F80913F021F928F933C
:104C90008EE995E09F938F930E94EE888091290979
:104CA0001F928F9385E995E09F938F930E94EE88E2
:104CB0001F9280E48F938DE795E09F938F930E94DE
:104CC000EE888091E9271F928F938091E8271F92A9
:104CD0008F938AE695E09F938F930E94EE88809150
:104CE0003E021F928F9381E695E09F938F930E94DF
:104CF000EE8880914002909141022DB73EB72A5E26
:104D00003F4F0FB6F8943EBF0FBE2DBF96FF03C0B6
:104D10008FEF95E002C082E096E09F938F9387E546
:104D200095E09F938F930E94EE88809147028F9326
:104D3000809146028F9382E495E09F938F930E9427
:104D4000EE888AE395E09F938F930E94EE886091AE
:104D500048027091490280914A0290914B020E9450
:104D6000DA220E94F30A8DB79EB70A960FB6F8941E
:104D70009EBF0FBE8DBF1D9B03C08FEF95E002C08D
:104D800082E096E09F938F938EE295E09F938F93BE
:104D90000E94EE8884E295E09F938F930E94EE88B4
:104DA000809140020F900F900F900F900F900F90F6
:104DB00081FF09C08EE195E09F938F930E94EE885A
:104DC0000F900F9013C080FF03C08FEF95E002C0DB
:104DD00082E096E09F938F938AE195E09F938F9373
:104DE0000E94EE880F900F900F900F9083E195E056
:104DF0009F938F930E94EE8860912D0970912E09E8
:104E000080E090E00E946A210E94F30A0F900F90C8
:104E1000779903C08FEF95E002C082E096E09F9300
:104E20008F938AE095E09F938F930E94EE880E9473
:104E3000AD08609148027091490280914A029091B8
:104E40004B020E94330A0E940F0A9F938F937F9315
:104E50006F938CEF94E09F938F930E94EE8881E094
:104E600090E00E9416208091C3279091C427A091C2
:104E7000C527B091C627BF93AF939F938F938EEEB4
:104E800094E09F938F930E94EE888091D3278F9315
:104E90008091D2278F938091D1278F938091D027B3
:104EA0008F938AED94E09F938F930E94EE88809178
:104EB000C7279091C827A091C927B091CA27BF934F
:104EC000AF939F938F938CEC94E09F938F930E946A
:104ED000EE888091D7278F938091D6278F938091EA
:104EE000D5278F938091D4278F9388EB94E09F935D
:104EF0008F930E94EE882DB73EB72E5D3F4F0FB6C1
:104F0000F8943EBF0FBE2DBF61E070E080E090E0FE
:104F10000E94FC0A61E070E081E090E00C94FC0AE1
:104F2000F894E0E0F0E081E2809357008491E2E0C1
:104F3000F0E041E2409357004491E4E0F0E091E278
:104F400090935700E49190E0A0E0B0E0DC01992755
:104F5000882750E060E070E0762F652F542F4427BB
:104F6000840F951FA61FB71F8E0F911DA11DB11D88
:104F700080930C1B90930D1BA0930E1BB0930F1BE3
:104F8000789408950F931F93CF93DF93CDB7DEB737
:104F900061970FB6F894DEBF0FBECDBF44E050E07E
:104FA0006AE170E0CE010B960E94138A0B851C8586
:104FB0002D853E850F3F8FEF18072807380749F4E6
:104FC00044E050E06AE170E088E492E00E94318AB7
:104FD00010C0009348021093490220934A02309374
:104FE0004B0210924C0210924D0210924E021092FF
:104FF0004F0242E050E068E170E0CE010F960E945F
:10500000138A8F8598898F3F2FEF920779F48CE36D
:1050100090E0909347028093460242E050E068E1BE
:1050200070E086E492E00E94318A04C090934702C7
:105030008093460242E050E066E170E0CE010F96B8
:105040000E94138A8F8598898F3F2FEF920779F4FA
:105050008AE090E4909341028093400242E050E065
:1050600066E170E080E492E00E94318A04C090938F
:1050700041028093400242E050E06EE270E0CE01D7
:105080000F960E94138A8F8598898F3F2FEF920782
:1050900069F410922E0910922D0942E050E06EE260
:1050A00070E08DE299E00E94318A04C090932E094D
:1050B00080932D0949E050E06AE070E088ED97E2C6
:1050C0000E94138A0E94340C44E050E066E270E0D3
:1050D000CE010B960E94138A8B859C85AD85BE857B
:1050E00044E050E066E270E08F3F9F4FAF4FBF4F0C
:1050F00029F487E692E00E94318A04C087E692E0B4
:105100000E94138A44E050E062E270E0CE010B9608
:105110000E94138A8B859C85AD85BE8544E050E056
:1051200062E270E08F3F9F4FAF4FBF4F29F483E69D
:1051300092E00E94318A04C083E692E00E94138AC2
:1051400044E050E06AE270E0CE010B960E94138AC0
:105150008B859C85AD85BE8544E050E06AE270E0B9
:105160008F3F9F4FAF4FBF4F29F48BE692E00E94D5
:10517000318A04C08BE692E00E94138A41E050E03D
:1051800065E170E0CE0141960E94138A898941E071
:1051900050E065E170E08F3F29F489E299E00E94D8
:1051A000318A04C089E299E00E94138A41E050E00C
:1051B00064E170E0CE0141960E94138A898941E042
:1051C00050E064E170E08F3F29F48FE392E00E94A9
:1051D000318A04C08FE392E00E94138A41E050E0DC
:1051E00063E170E0CE0141960E94138A898941E013
:1051F00050E063E170E08F3F29F48EE392E00E947B
:10520000318A04C08EE392E00E94138A4AE050E0A3
:1052100060E070E0CE0101960E94138A89814AE025
:1052200050E060E070E08F3F29F486E79AE10E9449
:10523000318A04C086E79AE10E94138A61960FB60C
:10524000F894DEBF0FBECDBFDF91CF911F910F91BC
:105250000895CF92DF92EF92FF9260916002709179
:10526000610280E090E00E943D8866E076E00E9466
:105270005188892B09F0C0C08DE48093480280E8F2
:105280008093490284E080934A0210924B0210926C
:105290004C0210924D0210924E0210924F0244E0C6
:1052A00050E06AE170E088E492E00E94318A8CE389
:1052B00090E0909347028093460242E050E068E11C
:1052C00070E086E492E00E94318A8AE090E4909354
:1052D00041028093400242E050E066E170E080E4E9
:1052E00092E00E94318A10922E0910922D0942E01C
:1052F00050E06EE270E08DE299E00E94318AA2E215
:10530000CA2EDD24DA94ACECEA2EABE3FA2EC0927E
:105310006702D0926802E0926902F0926A0244E069
:1053200050E066E270E087E692E00E94318AC09227
:105330006302D0926402E0926502F092660244E059
:1053400050E062E270E083E692E00E94318A87EDED
:1053500094E3AFEEBCE380936B0290936C02A09356
:105360006D02B0936E0244E050E06AE270E08BE6BA
:1053700092E00E94318A1092290980E090E00E9418
:10538000745F41E050E065E170E089E299E00E94DD
:10539000318A8AE180933F028AE190E00E94EC5DCD
:1053A00041E050E064E170E08FE392E00E94318AD6
:1053B0008FE080933E0241E050E063E170E08EE3D5
:1053C00092E00E94318A8AE0E6E7FAE1DF011D926D
:1053D0008A95E9F74AE050E060E070E0CF010E9472
:1053E000318A81E00E943A2180E090E0FF90EF90C6
:1053F000DF90CF900C94480CFF90EF90DF90CF900F
:1054000008952F923F924F925F926F927F928F9268
:105410009F92AF92BF92CF92DF92EF92FF920F9343
:105420001F93CF93DF9300D0CDB7DEB79A838983E4
:10543000FC0180819181892B11F00C949837609147
:1054400060027091610283E893E20E943D8860E40B
:1054500070E083E893E20E947088009759F46091AD
:10546000A3307091A4308AE090E00E94AA8881E085
:105470000C949D378130910549F440908323512C41
:10548000612C712C812C912C5401BDC0823091056E
:10549000A1F4809183232091842390E0982F882782
:1054A000820F911D2C01892F880F880B682E782E72
:1054B000882E982EA82EB82EA6C083309105D1F53F
:1054C0002091832310918423E091852330E040E0F4
:1054D00050E060E070E080E090E000E10E9419841C
:1054E000522E632E742E852E962EB72FA82FF92FAD
:1054F000212F30E040E050E060E070E080E090E09C
:1055000008E00E94198459016A017B018C01252D54
:10551000362D472D582D692D7B2F8A2F9F2F0E94C6
:105520005084AE2EB12CC12CD12CE12CF12C00E0FA
:1055300010E059C004970CF45DC0209183231091B2
:105540008423E0918523F091862330E040E050E011
:1055500060E070E080E090E008E10E941984290199
:105560003A014B01B82FA92F212F30E040E050E045
:1055700060E070E080E090E000E10E941984590151
:105580006A017B018C019201A301B4018B2F9A2F38
:105590000E945084AF2EB12CC12CD12CE12CF12CC7
:1055A00000E010E00E945084522E632E742E852E4F
:1055B000962EB72FA82FF92F2E2F30E040E050E085
:1055C00060E070E080E090E008E00E9419845901FA
:1055D0006A017B018C01252D362D472D582D692D13
:1055E0007B2F8A2F9F2F0E94508429013A014B0163
:1055F0005C0109C09AE0492E512C612C712C812C40
:10560000912CA12CB12C0E94F30A9201A301B401A8
:10561000C5012436F3E63F07FCE64F075105610557
:1056200071058105910509F4D4C72436E3E63E07E8
:10563000ECE64E075105610571058105910511F0F4
:1056400008F076C12536F2E73F07410551056105AF
:1056500071058105910511F40C94BA342536E2E701
:105660003E0741055105610571058105910511F060
:1056700008F0A0C02436F1E63F0741055105610559
:1056800071058105910511F40C948B352436E1E602
:105690003E0741055105610571058105910509F038
:1056A000D0F5A5E70E94778409F485C50E94778428
:1056B00009F038F4A8E60E94778409F4CAC40C946F
:1056C00096379201A301B401C501A6E70E94778431
:1056D00009F47DC52A33364241055105610571053E
:1056E0008105910511F00C94963784E0809378231E
:1056F00085E08093792310927A2310927B23109275
:105700007C2381E080937D2310927E2310927F235F
:105710001092802350C69201A301B401C501253621
:10572000EEE63E07410551056105710581059105CC
:1057300011F40C9411342536FEE63F07410551055E
:10574000610571058105910509F0B8F42536E4E697
:105750003E0741055105610571058105910509F473
:1057600033C424363946410551056105710581056B
:10577000910509F403C50C9496379201A301B40175
:10578000C5012737EFE63E07410551056105710563
:105790008105910511F40C94ED3323333147410514
:1057A0005105610571058105910511F40C948B3546
:1057B0000C9496379201A301B401C5012837E4E6A1
:1057C0003E07E1E64E07510561057105810591052A
:1057D00009F446C22837F4E63F07F1E64F075105C2
:1057E000610571058105910511F008F04DC0233761
:1057F000E3E73E0741055105610571058105910506
:1058000011F40C947F352337F3E73F074105510529
:10581000610571058105910509F0C8F42936E2E7B3
:105820003E0741055105610571058105910511F49A
:105830000C94343523373247410551056105710514
:105840008105910511F40C9473350C9496379201EF
:10585000A301B401C5012133E4E63E07E1E64E07AA
:105860005105610571058105910509F4FDC12336D6
:10587000344641465105610571058105910511F4D4
:105880000C948B350C9496379201A301B401C50199
:105890002336EDE63E07E8E64E0751056105710542
:1058A0008105910509F400C22336FDE63F07F8E6BD
:1058B0004F075105610571058105910509F0C0F497
:1058C0002236E5E63E07E4E64E075105610571051F
:1058D0008105910509F478C32237324745465105C1
:1058E000610571058105910509F4CEC60C949637C2
:1058F0009201A301B401C5012D36E5E73E07E8E6B4
:105900004E075105610571058105910511F40C944F
:1059100099352336324349465105610571058105A4
:10592000910511F00C9496370E94460F0C9498370D
:105930009201A301B401C5012633E9E63E07E5E77C
:105940004E07E5E65E07610571058105910509F4DD
:1059500083C32633F9E63F07F5E74F07F5E65F0710
:10596000610571058105910511F008F0B6C02C366E
:10597000E4E73E074E075105610571058105910574
:1059800011F40C94F3362C36F4E73F074F0751051A
:10599000610571058105910511F008F04CC02033B7
:1059A000E1E33E07E1E74E07510561057105810519
:1059B000910509F469C62033F1E33F07F1E74F078A
:1059C0005105610571058105910509F0C0F427367F
:1059D000EFE63E07ECE64E075105610571058105CE
:1059E000910509F4F9C5253733464D465105610542
:1059F00071058105910509F492C60C9496379201C0
:105A0000A301B401C5012133E1E33E07E1E74E07FD
:105A10005105610571058105910509F480C620379E
:105A2000354642475105610571058105910509F427
:105A3000A1C70C9496379201A301B401C501243784
:105A4000EFE63E074E07E2E65E0761057105810558
:105A5000910509F40AC42437FFE63F074F07F2E631
:105A60005F07610571058105910509F0C8F42437C8
:105A7000E8E73E07E4E74E0751056105710581053A
:105A8000910509F4F5C324373446474751056105AC
:105A900071058105910511F40C9439370C949637F2
:105AA0009201A301B401C5012936ECE63E07E1E607
:105AB0004E07E3E65E07610571058105910509F46E
:105AC00020C12E3631464846534661057105810591
:105AD000910509F4A7C30C9496379201A301B40170
:105AE000C5012136ECE63E07E5E64E07E2E75E0734
:105AF000610571058105910509F4C1C22136FCE6F5
:105B00003F07F5E64F07F2E75F076105710581057D
:105B1000910511F008F04FC02237E7E73E07E0E7B4
:105B20004E075E07610571058105910509F4C0C046
:105B30002237F7E73F07F0E74F075F076105710579
:105B40008105910509F0C8F42037ECE63E07E5E64B
:105B50004E07E8E65E07610571058105910509F4C8
:105B600078C221363D464547584661057105810595
:105B7000910509F448C60C9496379201A301B4012B
:105B8000C5012337E5E63E07E2E74E07E0E75E079B
:105B9000610571058105910511F40C944136233797
:105BA000324747475047610571058105910509F462
:105BB000ADC60C9496379201A301B401C5012737F5
:105BC000E0E73E07E8E74E07E4E75E076105710599
:105BD0008105910509F407C32737F0E73F07F8E788
:105BE0004F07F4E75F07610571058105910509F02D
:105BF000C8F42437E3E73E07E5E64E07E2E75E0731
:105C0000610571058105910509F47DC62437334787
:105C100045465447610571058105910509F44BC35B
:105C20000C9496379201A301B401C5012237E7E62F
:105C30003E07E0E74E07E5E75E0761057105810570
:105C4000910509F4A3C42C363146444758476105F1
:105C500071058105910511F40C94C1360C949637A9
:105C60000E94D4140C94983721E04CE061E080ED60
:105C70000E94785521E04EE061E080ED0E94785569
:105C800021E040E161E080ED0E94785521E042E1B1
:105C900061E080ED0E94785522E040E161E080ED16
:105CA0000E9478550C9498370E944C150C949837A4
:105CB000609160027091610280E090E00E943D88F6
:105CC0008C016FEF75E00E945188892B19F4779849
:105CD0000C94983762E076E0C8010E945188892BC5
:105CE00019F4779A0C949837779903C08FEF95E061
:105CF00002C082E096E09F938F9386E994E00C9433
:105D00008D37609160027091610280E090E00E94A6
:105D10003D888C0169EC75E00E945188892B09F05F
:105D200053C0609160027091610280E090E00E9437
:105D30003D888C01009711F40C9498376DE076E063
:105D40000E945188892B29F482E29FEFACECBBE3DF
:105D50000BC063E176E0C8010E945188892B69F489
:105D600082E29FEFACECBAE3809367029093680203
:105D7000A0936902B0936A021DC0C8010E942787E0
:105D80004B015C0120E030E0A9010E94D37E882312
:105D9000C1F081E00E94AC099B01AC01C501B401D6
:105DA0000E94D77E609367027093680280936902B5
:105DB00090936A0244E050E066E270E087E692E089
:105DC0004AC288EA92E05AC06CEC75E0C8010E94B1
:105DD0005188892B09F057C060916002709161026F
:105DE00080E090E00E943D888C01009711F40C94B3
:105DF00098376DE076E00E945188892B29F482E281
:105E00009FEFACECBBE30BC063E176E0C8010E94FE
:105E10005188892B69F482E29FEFACECBAE380935E
:105E2000630290936402A0936502B09366021DC062
:105E3000C8010E9427874B015C0120E030E0A901E6
:105E40000E94D37E8823C1F082E00E94AC099B01AE
:105E5000AC01C501B4010E94D77E609363027093C8
:105E60006402809365029093660244E050E062E22F
:105E700070E083E692E0EFC18BE992E09F938F930D
:105E80000E94EE88E3C064EC75E0C8010E9451886E
:105E9000892B09F059C0609160027091610280E025
:105EA00090E00E943D888C01009711F40C94983783
:105EB0006DE076E00E945188892B69F487ED94E3C8
:105EC000AFEEBCE380936B0290936C02A0936D02E3
:105ED000B0936E022FC063E176E0C8010E94518842
:105EE000892B19F48CE892E0C9CFC8010E9427875A
:105EF0004B015C0120E030E0A9010E94D37E8823A1
:105F000001F180E00E94AC092B013C0121EE3AE74F
:105F100044E95EE3C501B4010E940C7EA301920135
:105F20000E94D77E60936B0270936C0280936D0227
:105F300090936E0244E050E06AE270E08BE692E0FB
:105F40008AC18FE792E09ACF0E94FB099F938F93BB
:105F50007F936F9388E792E09F938F930E94EE88E0
:105F600082E00E94AC09209163023091640240916A
:105F70006502509166020E945481162F072FF82E59
:105F8000E92E81E00E94AC09EF92FF920F931F93DC
:105F900020916702309168024091690250916A0233
:105FA0000E9454819F938F937F936F938CE692E02E
:105FB0009F938F930E94EE880E94F30A0FB6F89485
:105FC000DEBF0FBECDBFB4C76091600270916102A9
:105FD00080E090E00E943D880097C1F00E94472237
:105FE00020912D0930912E098217930709F1909382
:105FF0002E0980932D0942E050E06EE270E08DE2C0
:1060000099E00E94318A8FE894E002C088E894E029
:106010009F938F930E94EE8860912D0970912E09B5
:1060200080E090E00E946A210E94F30A0F900F9096
:106030008DE794E09F938F930E94EE886FEF7FEF40
:1060400080E090E00E946A210E94F30A0F900F9076
:106050006FC70E94831E6CC780918723843329F405
:1060600040E061E080E00E94F010809162028823AD
:1060700009F45EC71F928F938AE794E04EC7809120
:106080008723893709F070C06091600270916102C6
:1060900080E090E00E943D888C016FEF75E00E94E7
:1060A0005188892B31F48091400290914102906493
:1060B0000CC062E076E0C8010E945188892B91F4FF
:1060C00080914002909141029F7B90934102809386
:1060D000400242E050E066E170E080E492E00E941D
:1060E000318A42C068E176E0C8010E945188892B5C
:1060F00021F58091921A8F938091911A8F938091BC
:10610000901A8F9380918F1A8F9380918E1A8F930C
:1061100080918D1A8F9380918C1A8F9380918B1A16
:106120008F9381E492E09F938F930E94EE880FB645
:10613000F894DEBF0FBECDBF17C080914002909192
:10614000410296FF03C08FEF95E002C082E096E027
:106150009F938F938DE392E09F938F930E94EE889D
:106160000F900F900F900F9080916202882309F496
:10617000DFC61F928F9387E794E0CFC660916002DD
:106180007091610280E090E00E943D886DE076E0D1
:106190000E945188892B11F481E001C080E00E94A7
:1061A0003A2180916202882309F4C2C61F928F931C
:1061B00084E794E0B2C60E94601F80916202882347
:1061C00009F4B6C61F928F9381E794E0A6C60E9499
:1061D0005C1F80916202882309F4AAC61F928F93E4
:1061E0008EE694E09AC6609160027091610280E050
:1061F00090E00E943D880E942B87803160F480935C
:10620000290999270E94745F41E050E065E170E040
:1062100089E299E020C0809129091F928F9383E33E
:1062200092E07BC6609160027091610280E090E034
:106230000E943D880E942B8725EF280F203170F4A3
:1062400080933F0299270E94EC5D41E050E064E1B9
:1062500070E08FE392E00E94318A6AC680913F022B
:106260001F928F938AE292E058C60C94000060C699
:10627000609160027091610280E090E00E943D8830
:10628000009771F04AE050E0BC0186E79AE10E9475
:1062900061884AE050E060E070E086E79AE1DBCF99
:1062A00086E79AE19F938F938EE196E09F938F9379
:1062B0000E94DC8836C6609160027091610280E0C5
:1062C00090E00E943D885C0168E774E00E9451887C
:1062D000892B39F4219A809140029091410280618A
:1062E00092C16DEC75E0C5010E945188892B39F48B
:1062F000229A8091400290914102806284C16AE5B5
:1063000074E0C5010E945188892B39F4239A809149
:10631000400290914102806476C16EE075E0C50153
:106320000E945188892B39F4239A809140029091E0
:106330004102806868C162E574E0C5010E9451882D
:10634000892B09F040C081E0809378238091480236
:10635000809379238091490280937A2380914A0225
:1063600080937B2380914B0280937C2380914C020D
:1063700080937D2380914D0280937E2380914E02F5
:1063800080937F2380914F028093802310928223F9
:1063900010928123809140029091410291609093EC
:1063A00041028093400242E050E066E170E080E408
:1063B00092E00E94318A48E753E262E180E292E093
:1063C0000E941C48B5C561E874E0C5010E9451886F
:1063D000892B71F4EBE9FAE1119211929AE1EB3B0E
:1063E000F907D1F7809140029091410292600BC170
:1063F00062E076E0C5010E94518820914002309110
:106400004102892BA9F42F703C7F309341022093E5
:1064100040022B9A42E050E066E170E080E492E0B6
:106420000E94318A8091CF2790E00E94015E80C552
:1064300024FF03C08FEF95E002C082E096E09F93B7
:106440008F938FE192E09F938F930E94EE888091CB
:1064500040020F900F900F900F9085FF03C08FEFB9
:1064600095E002C082E096E09F938F9384E192E0F2
:106470009F938F930E94EE88809140020F900F901F
:106480000F900F9086FF03C08FEF95E002C082E06F
:1064900096E09F938F9389E092E09F938F930E9461
:1064A000EE88809140020F900F900F900F9087FF21
:1064B00003C08FEF95E002C082E096E09F938F9338
:1064C0008EEF91E09F938F930E94EE88809140021F
:1064D000909141020F900F900F900F9090FF03C08A
:1064E0008FEF95E002C082E096E09F938F9383EF59
:1064F00091E09F938F930E94EE888091400290914B
:1065000041020F900F900F900F9091FF03C08FEFFB
:1065100095E002C082E096E09F938F9388EE91E031
:106520009F938F930E94EE88809140029091410248
:106530000F900F900F900F9091FFFAC486E296E0B3
:106540000E941289BBE9AB2EBAE1BB2E0BE010E032
:106550008EE2E82E86E0F82EF50180819181F2E04E
:10656000AF0EB11C9F938F931F930F93FF92EF92E7
:106570000E94DC880F5F1F4F0F900F900F900F90BD
:106580000F900F900B31110539F7D2C48AE694E0D1
:106590009F938F930E94EE88809162020F900F90DC
:1065A000882361F01F928F9387E694E09F938F93E7
:1065B0000E94EE880F900F900F900F9088E10FB619
:1065C000F89480936000109260000FBE0C94007CE1
:1065D000AFC40E942E55ACC46091600270916102FC
:1065E00080E090E00E943D888C016FEF75E00E9492
:1065F0005188892B99F40E94CB5C80914002909144
:1066000041028D7F8160909341028093400242E07D
:1066100050E066E170E080E492E01DCE62E076E05A
:10662000C8010E945188892B41F40E942D5C809101
:106630004002909141028C7FE6CF69E376E0C80189
:106640000E945188892B49F40E942D5C8091400260
:10665000909141028E7F8260D6CF8091400281FF6F
:1066600007C089E396E09F938F9384EE91E055C431
:1066700080FF03C08FEF95E002C082E096E09F9319
:106680008F9380EE91E049C48DE394E09F938F93C4
:106690000E94EE88809172238F93809171238F9353
:1066A000809170238F9380916F238F9380916E23BD
:1066B0008F9380916D238F9380916C238F93809122
:1066C0006B238F9380916A238F93809169238F939B
:1066D000809168238F93809167238F938091762395
:1066E0008F93809175238F93809174238F938091E2
:1066F00073238F938FE194E09F938F930E94EE8892
:10670000809162020FB6F894DEBF0FBECDBF882322
:1067100009F40EC41F928F938CE194E0FEC3F894A9
:1067200081E090E029E0FC0120935700C895E02C1F
:1067300080E090E0FC0120935700C895F02C7894FD
:10674000F89483E090E0FC0120935700C895002D59
:1067500082E090E0FC0120935700C895102D7894BA
:1067600080910F1B8F9380910E1B8F9380910D1B37
:106770008F9380910C1B8F9322E134E03F932F93F2
:106780000E94EE881F92EF921F92FF921F920F932A
:106790001F921F938BEE93E09F938F930E94EE883E
:1067A0000E94FA1F809166001F928F938FED93E0F5
:1067B0009F938F930E94EE880E94F30A8091620259
:1067C0000FB6F894DEBF0FBECDBF882309F4B0C367
:1067D0001F928F938CED93E0A0C360E070E080E0A7
:1067E00090E00E94FC0A60E070E081E090E00E948E
:1067F000FC0A80916202882309F49AC31F928F9346
:1068000089ED93E08AC30E94091E0E94F30A8091D9
:106810006202882309F48CC31F928F9386ED93E064
:106820007CC3609160027091610280E090E00E9400
:106830003D886EE376E00E945188892B31F5F8940B
:1068400084E699E00E9413495C01009769F0C50154
:106850000F960E945F4CB50184E092E00E94CD4803
:10686000C5010E94D949F0CF84E699E00E94B94958
:10687000892B29F084E699E00E945449F5CF84E6FB
:1068800099E00E940F49789434C084E699E00E9410
:1068900013497C0104E416E0E114F10451F1F7011D
:1068A00086811F928F9380851F928F9385811F927F
:1068B0008F9381851F928F9387811F928F938481FD
:1068C0001F928F9383811F928F9382811F928F9348
:1068D00082851F928F931F930F930E94DC88C701BC
:1068E0000E94D9497C010FB6F894DEBF0FBECDBF20
:1068F000D3CF80916202882309F41AC31F928F9329
:1069000083ED93E00AC30E94292912C360916002BB
:106910007091610280E090E00E943D888C0163E804
:1069200076E00E945188892B31F480914002909149
:106930004102937F68CE63E176E0C8010E945188EE
:10694000892B39F48091400290914102937F9860A5
:106950005ACE68E876E0C8010E945188892B39F444
:106960008091400290914102937F94604CCE0E94AE
:10697000AD08DEC2609160027091610280E090E03B
:106980000E943D88009709F44AC00E949B241B0185
:106990002C01A0904802B0904902C0904A02D090C9
:1069A0004B02E0904C02F0904D0200914E0210918B
:1069B0004F029B01A20160E070E080E090E00E9445
:1069C0006E84C9F1209248023092490240924A02F4
:1069D00050924B0210924C0210924D0210924E02B5
:1069E00010924F0248E050E06AE170E088E492E0E3
:1069F0000E94318A8BEC93E09F938F930E94EE88E4
:106A0000609148027091490280914A0290914B0234
:106A10000E94DA220E94F30A0F900F900CC060913E
:106A200048027091490280914A0290914B020E9463
:106A3000DA220E94F30A8FEB93E09F938F930E94D8
:106A4000EE886FEF7FEFCB010E94DA220E94F30AFB
:106A5000809162020F900F90882309F469C21F92FF
:106A60008F938CEB93E059C2609160027091610248
:106A700080E090E00E943D880097D9F04AE050E025
:106A800060E070E00E9413866093460270934702B4
:106A90007F936F938FE993E09F938F930E94EE888B
:106AA00042E050E068E170E086E492E00E94318AC2
:106AB0000CC0809147028F93809146028F938EE79E
:106AC00093E09F938F930E94EE880F900F900F900A
:106AD0000F9080916202882309F42AC21F928F933B
:106AE0008BE793E01AC20E949C4C8091620288233B
:106AF00009F41EC21F928F9388E793E00EC20E9492
:106B00000D2680916202882309F412C21F928F938E
:106B100085E793E002C280E090E00E941620809119
:106B20006202882309F404C21F928F9382E793E0E4
:106B3000F4C18091611F81FF2DC00E944C1D892BE3
:106B400049F58091581B8F938091571B8F938091AB
:106B5000561B8F938091551B8F9387E693E09F93ED
:106B60008F930E94EE888091E7278F938091E6278C
:106B70008F938091E5278F938091E4278F938AE507
:106B800093E09F938F930E94EE880FB6F894DEBF38
:106B90000FBECDBF0E94F30A8091611F9091621FCA
:106BA00090FF63C081E090E00E94FC1C4B015C01FF
:106BB00080E090E00E94FC1C2B013C010E947B1CA9
:106BC000BF92AF929F928F9289E493E09F938F93AD
:106BD0000E94EE887F926F925F924F9289E393E0DA
:106BE0009F938F930E94EE88242D352D462D572D8F
:106BF000682D792D8A2D9B2D0E94621B9F938F9368
:106C00007F936F938EE293E09F938F930E94EE8821
:106C1000242D352D462D572D682D792D8A2D9B2D10
:106C20000E94C31B9F938F937F936F9380E293E0A7
:106C30009F938F930E94EE88242D352D462D572D3E
:106C4000682D792D8A2D9B2D0E94241C9F938F9354
:106C50007F936F938DE093E09F938F930E94EE88D4
:106C60000FB6F894DEBF0FBECDBF0E94F30A80912D
:106C70006202882309F45CC11F928F938AE093E03B
:106C80004CC18091611F82FF2BC021E048E061E090
:106C900083E00E9465128091531B8F938091521B59
:106CA0008F938091511B8F938091501B8F93809174
:106CB0004F1B8F9380914E1B8F9380914D1B8F9311
:106CC00080914C1B8F9383EF92E09F938F930E9450
:106CD000EE880E94F30A0FB6F894DEBF0FBECDBF58
:106CE0008091611F9091621F91FF41C00E94AF1679
:106CF000B62EA72E982E892E20E030E048EC52E4E4
:106D0000D501F4016B2F7A2F8F2F9E2F0E94548173
:106D100020E836EE45EC57E40E94D77E21E03EEDB8
:106D200042E45EE30E94B7819B01AC0160E070E049
:106D300080E89FE30E940C7E2BE43AE34DEB57E39F
:106D40000E94D77E9F938F937F936F938F929F9292
:106D5000AF92BF928AED92E09F938F930E94EE884C
:106D60000E94F30A0FB6F894DEBF0FBECDBF80912C
:106D70006202882309F4DCC01F928F9387ED92E0B2
:106D8000CCC0609160027091610280E090E00E944E
:106D90003D8863E976E00E945188892BB1F46091C7
:106DA00060027091610280E090E00E943D8800974F
:106DB00009F4BEC00E942B87803108F0B9C09091C1
:106DC0005201982B90935201B3C0809152018F7061
:106DD0001F928F9383ED91E09F938F930E94EE8893
:106DE0000E94F30A9EC0609160027091610280E08F
:106DF00090E00E943D88009711F14AE050E060E089
:106E000070E00E94DF84603198F460933E021F922C
:106E10006F938AEC92E09F938F930E94EE8841E0FB
:106E200050E063E170E08EE392E00E94318A11C08D
:106E300080913E021F928F9381EC92E006C0809178
:106E40003E021F928F9388EB92E09F938F930E9454
:106E5000EE880F900F900F900F900E94F30A809190
:106E60006202882309F464C01F928F9385EB92E03D
:106E700054C0609160027091610280E090E00E94D5
:106E80003D888C016FEF75E00E945188892B41F499
:106E90000E940F5B80914002909141029061B3CBC0
:106EA00062E076E0C8010E945188892BE1F4F894F1
:106EB0000E941D5B88E10FB6F894809360001092E9
:106EC00060000FBE84B7877F84BF809160008861B7
:106ED00080936000109260007894809140029091BD
:106EE00041029F7E90CB68E976E0C8010E945188FC
:106EF0002091400230914102892B21F434FF18C0C7
:106F0000F894FFCF34FF03C08FEF95E002C082E01A
:106F100096E09F938F938FEC91E09F938F930E94C5
:106F2000EE880F900F900F900F9002C00E946A1E83
:106F3000E981FA811182108283E00F900F90DF9136
:106F4000CF911F910F91FF90EF90DF90CF90BF9066
:106F5000AF909F908F907F906F905F904F903F90F9
:106F60002F9008950E94035B6C9A6B9A6A9A6F9AAD
:106F7000729A749A739A779A809880B3897F80BB4B
:106F80008398849887E080937E00549A0E9490278B
:106F90000E94C22781E00E94200980E090E00E94C8
:106FA000480C0E949C538091400286FD239A0895CC
:106FB000CF93DF93EC0188819981009741F08A3962
:106FC0009E4009F47EC01982188283E083C00E942B
:106FD000B2378091400280FD05C081FF01C01D9B3A
:106FE0000E942D5C809170008C7F80937000809156
:106FF000B60080628093B6001092B20082E0809367
:10700000B1008091B6008770E1F7809170008160D7
:10701000809370006CEC78E080E090E00E94E65A8B
:107020000E945C1F80E00E943A2180EB9DE09F93CC
:107030008F930E94EE880E94460F8091611F0F90EF
:107040000F9086FD0E94D9548091290990E00E94FA
:10705000745F80913F0290E00E94EC5D0E94E95DC8
:107060008093540980913F0290E00E94EC5D8091F2
:1070700029091F928F93809154091F928F938DE954
:1070800096E09F938F930E94DC881092560910928D
:1070900055090F900F900F900F900F900F9084E371
:1070A00092E09093E2278093E12783E290E090932F
:1070B0006711809366118AE99EE09983888381E055
:1070C00009C06332E1F760E070E085E599E00E9475
:1070D000012AE5CFDF91CF9108958436910514F10F
:1070E0009F938F938FEA96E09F938F930E94DC8803
:1070F0008091732390917423A0917523B09176238E
:107100000196A11DB11D8093732390937423A093C6
:107110007523B09376230F900F900F900F9081E01E
:1071200090E0089580E090E008952F923F924F9272
:107130005F926F927F928F929F92AF92BF92CF9207
:10714000DF92EF92FF920F931F93CF93DF93CDB710
:10715000DEB7C559D1090FB6F894DEBF0FBECDBF5B
:10716000C457DF4F99838883CC58D040633871F47B
:1071700089E599E0CB56DF4F6883C559D0400E941E
:107180005346CB56DF4F6881C559D040C457DF4FB7
:10719000E881F981CC58D040208131812D34FEE046
:1071A0003F07F9F040F42115310581F02B3B3C40BD
:1071B00009F485C079C02E358EE0380709F455C032
:1071C00025363E4011F40C948D436EC04DEE53E0D5
:1071D00061E870E089E599E00E9438468BEB9CE01D
:1071E00058C000E010E0209140023091410230FF91
:1071F0001EC0739880914D098F5F80934D098A83DB
:10720000B8016F5F7F4FCE0101960E94B04F89E5B4
:1072100099E00E94564640E050E065E880916C118C
:1072200090916D110E941C488DE49EE032C08D2D1E
:1072300090E00E94015EF0924702E0924602739A4B
:1072400080912A0990912B09892B11F00E942D5CC5
:1072500080914D098F5F80934D0980912D09909108
:107260002E0982FFBBCF739AB9CF85E499E00E94C3
:10727000FD4A892BB1F00E94CB5C8091400287FDD2
:107280002B9860E470E085E499E00E94D24A85E69C
:107290009EE0C457DF4FE881F981CC58D0409183FC
:1072A000808381E00C94A043C457DF4FE881F981CB
:1072B000CC58D0401182108283E00C94A0436231FC
:1072C00081F7809140029091410291FD87CF80919A
:1072D0007823813039F58090792390907A23A0909B
:1072E0007B23B0907C23F0917D23C257DF4FF8833E
:1072F000CE58D04020917E23C157DF4F2883CF58EE
:10730000D04030917F23C057DF4F3883C059D040E1
:1073100040918023CF56DF4F4883C159D040212C64
:10732000312C2FC0823049F58090792390907A23B8
:10733000A0907B23B0907C2350917D23C257DF4FD8
:107340005883CE58D04080917E23C157DF4F888329
:10735000CF58D04090917F23C057DF4F9883C059BA
:10736000D040E0918023CF56DF4FE883C159D04011
:10737000209081233090822304C0843009F02ECFE6
:10738000AACFFA2DF470C657DF4FF883CA58D04001
:1073900020E030E04F2F50E060E070E080E090E0CF
:1073A000A0E00E94778409F08C9AB401C5010E9484
:1073B000330A292D2074C557DF4F2883CB58D0407E
:1073C00020E0C557DF4F3881CB58D04040E050E037
:1073D00060E070E080E090E0A0E00E94778411F02F
:1073E0000E944C1D392D3078CE56DF4F3883C2595C
:1073F000D04020E040E050E060E070E080E090E0CD
:10740000A0E00E94778451F00E94FB096093CB2793
:107410007093CC278093CD279093CE27282D217071
:1074200030E040E050E060E070E080E090E0A0E01C
:107430000E947784F1F086E79AE19F938F9383EC23
:1074400096E09F938F931F9287E78F93CE010396C9
:107450009F938F930E943F897C010E946D380FB6E5
:10746000F894DEBF0FBECDBF892B09F0B7CE8701E0
:1074700002C000E010E0282D227030E040E050E033
:1074800060E070E080E090E0A0E00E947784C9F1C5
:10749000C80102966BEC76E0E1E0F0E0EC0FFD1F36
:1074A0008E0F9F1F0E945A880D5F1F4F68EDC62EDA
:1074B00067E2D62E7AE8E72E74E0F72EE7E77E2E15
:1074C000F60181916F011F928F93FF92EF921F92AD
:1074D0007F92C801029621E030E02C0F3D1F820F01
:1074E000931F9F938F930E943F89080F191F0FB618
:1074F000F894DEBF0FBECDBF50EEC51657E2D506DD
:10750000F9F6282D247030E040E050E060E070E0B3
:1075100080E090E0A0E00E94778409F446C0C801B2
:1075200002966FEC76E0E1E0F0E0EC0FFD1F8E0FCD
:107530009F1F0E945A880C5F1F4F6E01FAE7CF0E03
:10754000D11C80E1F60111928A95E9F728E0A601A5
:1075500068E980EB0E94A9103601F8E06F0E711CFB
:107560004AE8E42E44E0F42E57E7552EF6018191C7
:107570006F011F928F93FF92EF921F925F92C8014B
:10758000029621E030E02C0F3D1F820F931F9F9346
:107590008F930E943F89080F191F0FB6F894DEBF22
:1075A0000FBECDBFC614D70409F75B2D5078CD565A
:1075B000DF4F5883C359D04020E030E040E060E026
:1075C00070E080E090E0A0E00E94778401F5809177
:1075D0002B098F9380912A098F9384ED96E09F93D6
:1075E0008F931F9287E78F93C8010296E1E0F0E046
:1075F000EC0FFD1F8E0F9F1F9F938F930E943F895B
:10760000080F191F0FB6F894DEBF0FBECDBF20E0E4
:1076100030E040E050E0C257DF4F6881CE58D040A4
:10762000617070E080E090E0A0E00E94778409F152
:10763000E3E0F0E0EC0FFD1FE00FF11F80E280833C
:10764000E6E8F3E280810F5F1F4F882359F08081C5
:10765000A1E0B0E0AC0FBD1FA00FB11F12968C933C
:107660003196F0CFE3E0F0E0EC0FFD1FE00FF11FEB
:107670001082282D287030E040E050E060E070E09B
:1076800080E090E0A0E00E947784C1F127E04AE228
:1076900050E06BE270E089E290E00E94B25088ED29
:1076A00097E20E942253BC01882777FD8095982F8E
:1076B0000E94767F20E030E048EC52E40E94D77EC2
:1076C0009F938F937F936F938BED96E09F938F9310
:1076D0001F9287E78F93C801029641E050E04C0F5C
:1076E0005D1F840F951F9F938F930E943F89080F02
:1076F000191F0FB6F894DEBF0FBECDBF282D207125
:1077000030E040E050E060E070E080E090E0A0E039
:107710000E947784F1F126E04AE250E06BE270E0EB
:1077200089E290E00E94B25081E090E00E94810ADC
:107730008093280984EC9AE10E942253BC01882797
:1077400077FD8095982F0E94767F20E030E048EC0E
:1077500052E40E94D77E9F938F937F936F9385EE21
:1077600096E09F938F931F9287E78F93C8010296AD
:10777000E1E0F0E0EC0FFD1F8E0F9F1F9F938F93B2
:107780000E943F89080F191F0FB6F894DEBF0FBE85
:10779000CDBF282D207230E040E050E060E070E086
:1077A00080E090E0A0E00E94778431F18091831A1C
:1077B0008F938091821A8F938091811A8F938091F9
:1077C000801A8F9380EF96E09F938F931F9287E7A5
:1077D0008F93C801029641E050E04C0F5D1F840F6B
:1077E000951F9F938F930E943F89080F191F0FB613
:1077F000F894DEBF0FBECDBF282D207430E040E0EE
:1078000050E060E070E080E090E0A0E00E947784CB
:1078100001F10E940F0A9F938F937F936F938EEFD6
:1078200096E09F938F931F9287E78F93C8010296EC
:10783000E1E0F0E0EC0FFD1F8E0F9F1F9F938F93F1
:107840000E943F89080F191F0FB6F894DEBF0FBEC4
:10785000CDBF282D207830E040E050E060E070E0BF
:1078600080E090E0A0E00E94778441F1F89480915C
:10787000C3279091C427A091C527B091C6277894BB
:10788000BF93AF939F938F938CE097E09F938F93D9
:107890001F9287E78F93C801029641E050E04C0F9A
:1078A0005D1F840F951F9F938F930E943F89080F40
:1078B000191F0FB6F894DEBF0FBECDBF20E0392DE3
:1078C000317040E050E060E070E080E090E0A0E0E7
:1078D0000E94778409F477C0809146029091470214
:1078E000892B09F470C0F894C090C327D090C427A6
:1078F000E090C527F090C62778948091BC1A9091AB
:10790000BD1AA091BE1AB091BF1AA7019601281BFB
:10791000390B4A0B5B0BCA01B9010E94747F2B0122
:107920003C01609146027091470280E090E00E9425
:10793000747F9B01AC01C301B2010E94D77E3C0160
:107940007F928F937F936F9387E197E09F938F93BD
:107950001F9287E78F939E01200F311F2D5F3F4FAE
:107960003F932F93CB56DF4F6883C559D040CC56F9
:10797000DF4F7883C459D0400E943F89080F191FF8
:10798000CB56DF4F6881C559D040CC56DF4F788148
:10799000C459D040862F972FA62DB72D8093D0277E
:1079A0009093D127A093D227B093D327C092BC1A2B
:1079B000D092BD1AE092BE1AF092BF1A0FB6F89498
:1079C000DEBF0FBECDBF20E0392D327040E050E069
:1079D00060E070E080E090E0A0E00E94778491F1A8
:1079E0008091460290914702892B61F1F894809131
:1079F000931A9091941AA091951AB091961A78942E
:107A00009F938F93809145028F93809144028F932F
:107A100084E297E09F938F931F9287E78F93C8012B
:107A20000296E1E0F0E0EC0FFD1F8E0F9F1F9F9389
:107A30008F930E943F89080F191F0FB6F894DEBF7D
:107A40000FBECDBF20E0392D347040E050E060E043
:107A500070E080E090E0A0E00E94778471F1F894FB
:107A60008091C7279091C827A091C927B091CA27B4
:107A70007894BF93AF939F938F9384E397E09F9302
:107A80008F931F9287E78F93C801029641E050E0E1
:107A90004C0F5D1F840F951F9F938F930E943F890A
:107AA000080F191FC8010E946D380FB6F894DEBF89
:107AB0000FBECDBF892B09F091CB20E0392D387056
:107AC00040E050E060E070E080E090E0A0E00E94E4
:107AD000778409F477C08091460290914702892B00
:107AE00009F470C0F894C090C727D090C827E090E0
:107AF000C927F090CA2778948091C01A9091C11A32
:107B0000A091C21AB091C31AA7019601281B390B84
:107B10004A0B5B0BCA01B9010E94747F2B013C0127
:107B2000609146027091470280E090E00E94747F6D
:107B30009B01AC01C301B2010E94D77E3C017F9240
:107B40008F937F936F938FE397E09F938F931F9211
:107B500087E78F939E01200F311F2D5F3F4F3F938B
:107B60002F93CB56DF4F6883C559D040CC56DF4F9B
:107B70007883C459D0400E943F89080F191FCB5603
:107B8000DF4F6881C559D040CC56DF4F7881C4594A
:107B9000D040862F972FA62DB72D8093D427909372
:107BA000D527A093D627B093D727C092C01AD092DA
:107BB000C11AE092C21AF092C31A0FB6F894DEBF4F
:107BC0000FBECDBF20E0392D307140E050E060E0C5
:107BD00070E080E090E0A0E00E94778491F18091D5
:107BE000460290914702892B61F1F8948091971A8F
:107BF0009091981AA091991AB0919A1A78949F939B
:107C00008F93809143028F93809142028F938CE4F3
:107C100097E09F938F931F9287E78F93C8010296F7
:107C2000E1E0F0E0EC0FFD1F8E0F9F1F9F938F93FD
:107C30000E943F89080F191F0FB6F894DEBF0FBED0
:107C4000CDBF20E0392D307240E050E060E070E0C0
:107C500080E090E0A0E00E94778461F1809163234E
:107C600090916423A0916523B0916623BF93AF9355
:107C70009F938F938CE597E09F938F931F9287E755
:107C80008F93C801029641E050E04C0F5D1F840FB6
:107C9000951F9F938F930E943F89080F191FC8015A
:107CA0000E946D380FB6F894DEBF0FBECDBF892B92
:107CB00009F094CA20E0C557DF4F3881CB58D04037
:107CC00040E050E060E070E080E090E0A0E00E94E2
:107CD000778461F18091581B8F938091571B8F930C
:107CE0008091561B8F938091551B8F9387E697E069
:107CF0009F938F931F9287E78F93C801029621E08D
:107D000030E02C0F3D1F820F931F9F938F930E9493
:107D10003F89080F191FC8010E946D380FB6F894EB
:107D2000DEBF0FBECDBF892B09F058CA20E0CE566A
:107D3000DF4F3881C259D04040E050E060E070E051
:107D400080E090E0A0E00E94778461F18091CE27EE
:107D50008F938091CD278F938091CC278F938091A3
:107D6000CB278F9382E797E09F938F931F9287E7AC
:107D70008F93C8010296E1E0F0E0EC0FFD1F8E0F3B
:107D80009F1F9F938F930E943F89080F191FC8015F
:107D90000E946D380FB6F894DEBF0FBECDBF892BA1
:107DA00009F01CCA20E030E04A2D417050E060E04C
:107DB00070E080E090E0A0E00E94778489F181E0AB
:107DC0000E94AC09209167023091680240916902DB
:107DD00050916A020E9454819F938F937F936F9377
:107DE0008FE797E09F938F931F9287E78F93C80148
:107DF000029641E050E04C0F5D1F840F951F9F934A
:107E00008F930E943F89080F191FC8010E946D3887
:107E10000FB6F894DEBF0FBECDBF892B09F0DEC9C7
:107E200020E030E04A2D427050E060E070E080E0F9
:107E300090E0A0E00E94778489F182E00E94AC0982
:107E40002091630230916402409165025091660274
:107E50000E9454819F938F937F936F938CE897E058
:107E60009F938F931F9287E78F93C801029621E01B
:107E700030E02C0F3D1F820F931F9F938F930E9422
:107E80003F89080F191FC8010E946D380FB6F8947A
:107E9000DEBF0FBECDBF892B09F0A0C920E030E0C6
:107EA000C657DF4F4881CA58D04050E060E070E0CC
:107EB00080E090E0A0E00E94778441F183E00E949E
:107EC000AC099F938F937F936F9389E997E09F937A
:107ED0008F931F9287E78F93C8010296E1E0F0E04D
:107EE000EC0FFD1F8E0F9F1F9F938F930E943F8962
:107EF000080F191F8C98C8010E946D380FB6F894AE
:107F0000DEBF0FBECDBF892B09F068C920E030E08D
:107F10004A2D487050E060E070E080E090E0A0E022
:107F20000E94778471F18091611F87FF2AC021E050
:107F300042E161E080ED0E9478559F938F937F939B
:107F40006F9386EA97E09F938F931F9287E78F93B3
:107F5000C801029641E050E04C0F5D1F840F951F51
:107F60009F938F930E943F89080F191FC8010E9499
:107F70006D380FB6F894DEBF0FBECDBF892B09F068
:107F80002DC920E030E04A2D407150E060E070E003
:107F900080E090E0A0E00E94778471F18091611F01
:107FA00087FF2AC021E042E162E080ED0E9478551F
:107FB0009F938F937F936F9384EB97E09F938F931F
:107FC0001F9287E78F93C801029621E030E02C0FC3
:107FD0003D1F820F931F9F938F930E943F89080F2D
:107FE000191FC8010E946D380FB6F894DEBF0FBE8E
:107FF000CDBF892B09F0F2C820E030E04A2D407255
:1080000050E060E070E080E090E0A0E00E947784C3
:1080100071F18091611F87FF2AC021E042E163E096
:1080200080ED0E9478559F938F937F936F9382EC9E
:1080300097E09F938F931F9287E78F93C8010296D3
:10804000E1E0F0E0EC0FFD1F8E0F9F1F9F938F93D9
:108050000E943F89080F191FC8010E946D380FB692
:10806000F894DEBF0FBECDBF892B09F0B7C820E062
:1080700030E04A2D407450E060E070E080E090E035
:10808000A0E00E94778471F18091611F87FF2AC070
:1080900021E042E164E080ED0E9478559F938F9348
:1080A0007F936F9380ED97E09F938F931F9287E765
:1080B0008F93C801029641E050E04C0F5D1F840F82
:1080C000951F9F938F930E943F89080F191FC80126
:1080D0000E946D380FB6F894DEBF0FBECDBF892B5E
:1080E00009F07CC8FA2DF078EF2E20E030E04F2F19
:1080F00050E060E070E080E090E0A0E00E947784D3
:1081000049F08091611F82FF05C046E061E083E095
:108110000E9465122B2D2170F22E20E030E040E00D
:108120005F2D60E070E080E090E0A0E00E94778446
:1081300051F08091611F82FF06C021E046E061E0BE
:1081400083E00E94651220E030E04E2D50E060E0B8
:1081500070E080E090E0A0E00E94778481F180915F
:10816000611F82FF2CC080914F1B8F9380914E1B0B
:108170008F9380914D1B8F9380914C1B8F938EED2D
:1081800097E09F938F931F9287E78F93C801029682
:1081900041E050E04C0F5D1F840F951F9F938F931C
:1081A0000E943F89080F191FC8010E946D380FB641
:1081B000F894DEBF0FBECDBF892B09F00FC820E0B9
:1081C00030E040E05F2D60E070E080E090E0A0E013
:1081D0000E94778489F18091611F82FF2DC0809178
:1081E000531B8F938091521B8F938091511B8F93C0
:1081F0008091501B8F9386EE97E09F938F931F92F1
:1082000087E78F93C801029621E030E02C0F3D1FD5
:10821000820F931F9F938F930E943F89080F191F0E
:10822000C8010E946D380FB6F894DEBF0FBECDBFF7
:10823000892B11F00C94EE3820E030E040E05B2D0B
:10824000527060E070E080E090E0A0E00E947784EF
:1082500079F18091611F9091621F90FF29C080E0A9
:1082600090E00E94FC1C9F938F937F936F9381EF0C
:1082700097E09F938F931F9287E78F93C801029691
:10828000E1E0F0E0EC0FFD1F8E0F9F1F9F938F9397
:108290000E943F89080F191FC8010E946D380FB650
:1082A000F894DEBF0FBECDBF892B11F00C94EE38D1
:1082B00020E030E040E05B2D547060E070E080E052
:1082C00090E0A0E00E94778479F18091611F909105
:1082D000621F90FF29C081E090E00E94FC1C9F93E8
:1082E0008F937F936F9381E098E09F938F931F927A
:1082F00087E78F93C801029641E050E04C0F5D1F65
:10830000840F951F9F938F930E943F89080F191F19
:10831000C8010E946D380FB6F894DEBF0FBECDBF06
:10832000892B11F00C94EE3820E030E040E05B2D1A
:10833000507160E070E080E090E0A0E00E947784FF
:10834000D9F18091611F9091621F90FF35C081E04B
:1083500090E00E94FC1C6B017C0180E090E00E9498
:10836000FC1C9B01AC01C701B6010E94621B9F93DC
:108370008F937F936F9382E198E09F938F931F92E7
:1083800087E78F93C801029621E030E02C0F3D1F54
:10839000820F931F9F938F930E943F89080F191F8D
:1083A000C8010E946D380FB6F894DEBF0FBECDBF76
:1083B000892B11F00C94EE3820E030E040E05B2D8A
:1083C000507260E070E080E090E0A0E00E9477846E
:1083D000D9F18091611F9091621F90FF35C081E0BB
:1083E00090E00E94FC1C6B017C0180E090E00E9408
:1083F000FC1C9B01AC01C701B6010E94C31B9F93EB
:108400008F937F936F938DE198E09F938F931F924B
:1084100087E78F93C8010296E1E0F0E0EC0FFD1FC3
:108420008E0F9F1F9F938F930E943F89080F191FE4
:10843000C8010E946D380FB6F894DEBF0FBECDBFE5
:10844000892B11F00C94EE3820E030E040E05B2DF9
:10845000507460E070E080E090E0A0E00E947784DB
:10846000D9F18091611F9091621F90FF35C081E02A
:1084700090E00E94FC1C6B017C0180E090E00E9477
:10848000FC1C9B01AC01C701B6010E94241C9F93F8
:108490008F937F936F938BE298E09F938F931F92BC
:1084A00087E78F93C801029641E050E04C0F5D1FB3
:1084B000840F951F9F938F930E943F89080F191F68
:1084C000C8010E946D380FB6F894DEBF0FBECDBF55
:1084D000892B11F00C94EE3820E030E040E05B2D69
:1084E000587060E070E080E090E0A0E00E94778447
:1084F00069F18091611F9091621F91FF27C00E94D6
:10850000AF169F938F937F936F938EE398E09F9323
:108510008F931F9287E78F93C801029621E030E086
:108520002C0F3D1F820F931F9F938F930E943F89B3
:10853000080F191FC8010E946D380FB6F894DEBFEE
:108540000FBECDBF892B11F00C94EE3820E030E047
:1085500040E0CD56DF4F5881C359D04060E070E015
:1085600080E090E0A0E00E94778471F1F1018681C3
:108570001F928F9385811F928F9383811F928F9378
:1085800082811F928F938FE498E09F938F931F9225
:1085900087E78F93C801029621E030E02C0F3D1F42
:1085A000820F931F9F938F930E943F89080F191F7B
:1085B000C8010E946D380FB6F894DEBF0FBECDBF64
:1085C000892B11F00C94EE38779A80912D099091B7
:1085D0002E0992FD749A9401A501C257DF4F68815C
:1085E000CE58D040C157DF4F7881CF58D040C057C8
:1085F000DF4F8881C059D040CF56DF4F9881C15995
:10860000D040A0E0FE0133967F010E94778451F1B3
:1086100080912D0990912E0982FD08C08091400221
:1086200080FD04C081FF1EC01D9B1CC0FF92EF9205
:1086300086E698E09F938F930E94DC888091620287
:108640000F900F900F900F90882361F01F928F93DF
:108650008DEA9DE09F938F930E94EE880F900F907C
:108660000F900F9080913E028061898380914D0927
:108670008A83F701E00FF11F108280912D099091FC
:108680002E0998012D5F3F4F790180FF0CC0FF92AA
:108690002F938DE698E09F938F930E94DC880F9034
:1086A0000F900F900F90B701CE0101960E94B04F2E
:1086B0008091400282FF0AC023EC33E2A701BE0191
:1086C0006F5F7F4F80E592E00E94355480912D09C5
:1086D00090912E0982FD73980E94CB5C89E599E008
:1086E0000E945646809140029091410290FD02C046
:1086F0000C9420390F5F1F4FE0904602F090470224
:108700000E94E95DD82E109247021092460289E13C
:1087100090E00E94015E0C94F33885E499E00E9499
:10872000FD4A892B11F40C9451390E942D5C8091E3
:10873000400287FD02C00C94EE382B9A0C94EE3860
:10874000CB56DF4F0FB6F894DEBF0FBECDBFDF9123
:10875000CF911F910F91FF90EF90DF90CF90BF903E
:10876000AF909F908F907F906F905F904F903F90D1
:108770002F9008950C9480464F925F926F927F9253
:108780008F929F92AF92BF92CF92DF92EF92FF9221
:108790000F931F93CF93DF93CDB7DEB760970FB6DC
:1087A000F894DEBF0FBECDBF6B010E94E95DFC01F6
:1087B000EE0FFF1FEE7FF170EB57F54E8081918138
:1087C00001969183808380912D0990912E0981FDDE
:1087D000749880904002909041020E94E44E7C0187
:1087E000FC018081982F92959F70913099F48F7041
:1087F00051F48091911A9091921A01969093921A45
:108800008093911A08C1B60188EE97E20E94E9456B
:10881000892B51F080918F1A9091901A0196909324
:10882000901A80938F1AF7C0C40184E0989F812D1D
:1088300099271124F82FF1708F2E84E699E00E9479
:1088400013498C01009709F448C0B601C80102968B
:108850000E94E945892BE9F1980146EE58E060E075
:1088600074E6C8010F960E94D84BF7019181F80178
:108870008481981321C082858F5F828780918D1AB1
:1088800090918E1A019690938E1A80938D1A84E09F
:108890000E941850F801208530E02817390708F0A9
:1088A00074C184E00E941850F8018087F70180812C
:1088B0008F70F8018187AFC0F801128684E00E94B2
:1088C0001850F8018087F70180818F70F801818747
:1088D0005DC1C8010E94D949B4CF84E092E00E94F2
:1088E000A7488C01009709F496C0B601C80102960A
:1088F0000E94E045F70181818150F801848380E086
:1089000091E0A0E0B0E083879487A587B6871286C0
:1089100084E00E941850F8018087F70180818F70F1
:10892000F8018187B80184E699E00E949A4998018C
:1089300046EE58E060E074E6C8010F960E94D84BFE
:1089400099249394F7018181F8018483F701808150
:108950008F70F801878384E00E941850F8018583A6
:1089600083E00E9418505C01F801868387818F3074
:1089700009F0912CF7014180F8018481481A512CAB
:10898000612C712CB6E0440C551C661C771CBA9502
:10899000D1F72385348545855685A0ECB0E00E944B
:1089A0003282BB27A92F982F872F480E591E6A1E87
:1089B0007B1E438654866586768680912D0990912C
:1089C0002E0981FD32C08091400280FD2EC081FDC4
:1089D0002AC0992001F182E08093782381E080937E
:1089E000792310927A2310927B2380E880937C2352
:1089F00010927D2310927E2310927F231092802369
:108A0000109382230093812348E753E262E180E2DE
:108A100092E00E941C4880912D0990912E0981FFBF
:108A2000B7C0749AB5C01D9BD4CFA4E6B0E0A30133
:108A300092010E943282672F782F892F992724E68E
:108A400030E040E050E00E947D827F936F93452CA0
:108A5000562C672C77245F924F92BB24BF92AF9223
:108A6000F80185811F928F93F70180818F701F928B
:108A70008F9381811F928F93F60181811F928F9333
:108A800080811F928F93C70102969F938F938EE7E9
:108A900098E09F938F930E94DC88809162020FB6CA
:108AA000F894DEBF0FBECDBF882361F01F928F9375
:108AB0008AEA9DE09F938F930E94EE880F900F901B
:108AC0000F900F90809140029091410296FF2DC02F
:108AD000882059F1F7012081322F3F70832F90E0D9
:108AE0000297D4F08FEF830F207F822B808389E55C
:108AF00099E00E94BA4380918B1A90918C1A01964A
:108B000090938C1A80938B1A80912D0990912E0945
:108B100096FF0BC0739809C08091911A9091921A98
:108B200001969093921A8093911A8091611F86FF0B
:108B300050CF0E94CA54C70105960E948954F7017C
:108B400081811F928F93F80186811F928F93858177
:108B50001F928F9382EC98E09F938F931F9280E1F6
:108B60008F939E012F5F3F4F7901FF922F930E94B9
:108B70003F8982E00E94A654C7010E9489540FB623
:108B8000F894DEBF0FBECDBF24CF812C912CDACE5E
:108B900060960FB6F894DEBF0FBECDBFDF91CF91C8
:108BA0001F910F91FF90EF90DF90CF90BF90AF900B
:108BB0009F908F907F906F905F904F900895089551
:108BC000FC01DB018C91808311968C91119781833C
:108BD0000895FC01DB0190818C91981741F421E00C
:108BE00030E0918111968C911197981711F020E047
:108BF00030E0C9010895FC0180818093E8278181DC
:108C00008093E9270895DC011996ED91FC911A975C
:108C10000280F381E02D309709F009950895EF92D5
:108C2000FF920F931F93DF93CF9300D0CDB7DEB7A2
:108C30008C0188E10E942B50BC017E010894E11C4C
:108C4000F11CC7010E94E045D8011996ED91FC91F5
:108C50001A970190F081E02DC801B70109950F9096
:108C60000F90CF91DF911F910F91FF90EF9008959A
:108C7000EF92FF920F931F93CF93DF93EC018B0141
:108C80007A0143E752E00E946446FA86E986C80109
:108C900067E772E00E94C346DF91CF911F910F9169
:108CA000FF90EF9008950E947D460895CF93DF9343
:108CB000EC0188E168EE77E20E942150CE010E942B
:108CC0008046DF91CF910895EF92FF920F931F930B
:108CD000CF93DF93EC018B017A010E949C46F886CA
:108CE000EF82C8016BE772E00E94C346DF91CF912B
:108CF0001F910F91FF90EF9008950E94A54608954F
:108D00000E94A2620895FC01A781B0852D913C913B
:108D1000F90109950895DC011796ED91FC911897DA
:108D20000280F381E02D309709F00995089588E6D7
:108D300091E10E940F490895FC017383628388E6E4
:108D400091E1BF010E949A490895BC0188E691E132
:108D50000E9461490895CF93DF93EC0188E691E189
:108D60000E94134908C0828193818C179D0739F0B6
:108D7000CF010E94D949E82FF92F3097A1F7CF01F1
:108D8000DF91CF9108950F931F93CF93DF938B01C2
:108D90000E94AB46EC01009731F01D830C83C801A3
:108DA0000E94FA648E83DF91CF911F910F910895F5
:108DB0001F93CF93DF93EC01162F888580FF1DC092
:108DC000EC81FD813097C9F0D0936D11C0936C1187
:108DD00082E08887CE0106960995992787FD9095B0
:108DE00002978230910510F0133829F4CE01BE01AC
:108DF0000E94014702C081E08887DF91CF911F91D7
:108E00000895CF92DF92EF92FF920F931F93CF932B
:108E1000DF93EC017B01C0906C11D0906D1100913B
:108E20006A1110916B11F80103C00190F081E02DDF
:108E3000EC17FD0719F03097C1F746C0209709F4E9
:108E400043C08885882309F118860BC0C017D10755
:108E500029F0C80167E8AE010E94D846F8010081F8
:108E600011810115110591F7EC81FD81309769F0B1
:108E7000CE15DF0551F0D0936D11C0936C11CE016A
:108E8000069663E840E050E00995E0916A11F091A0
:108E90006B11CE17DF0791F48881998190936B1144
:108EA00080936A110DC0808191818C179D0729F4F0
:108EB000888199819183808303C0FC01309799F761
:108EC000D0926D11C0926C11DF91CF911F910F91D3
:108ED000FF90EF90DF90CF9008951F93CF93DF9393
:108EE00010926E11C0916A11D0916B1111E00EC0F9
:108EF0008985882341F018871986CE0162E840E011
:108F000050E00E94D8460990D881C02D209781F763
:108F1000DF91CF911F91089580911912982F9F5F33
:108F200090931912089560916C1170916D110E94C7
:108F3000014708958AE880931912109270111092D7
:108F40006F1110926B1110926A1110926D111092A4
:108F50006C11089580916E11882311F00E946D4765
:108F600070916F11772309F455C02091701130E092
:108F7000F901EE0FFF1FEE0FFF1FE20FF31FEF5877
:108F8000FE4E6081609318124181528150931712F6
:108F9000409316128381948190931512809314123A
:108FA0002F5F3F4F2F71307020937011715070936D
:108FB0006F11009741F580916A1190916B1118C063
:108FC00080916E11882311F00E946D474091161216
:108FD00050911712809112129091131260911812F1
:108FE0000E94D846E0911212F09113128081918173
:108FF0009093131280931212809112129091131277
:109000000097F1F607C0613819F421E0FC012087D0
:109010000E94D84680916E1120916F1130E0280F88
:10902000311DC901089580916E1120916F1130E0BA
:10903000280F311DC901089570916F117032D9F058
:1090400020917011270F2F712093111230E0F90138
:10905000EE0FFF1FEE0FFF1FE20FF31FEF58FE4E44
:10906000608352834183948383837F5F70936F1106
:1090700020E030E002C021E030E0C9010895CF9344
:10908000DF93C0916C11D0916D110E94D846D0939E
:109090006D11C0936C11DF91CF910895FC01AB016C
:1090A00090916A1180916B119C01A32FB22F03C084
:1090B0000D90BC91A02DAE17BF0791F01097C1F78E
:1090C000309771F090838183F0936B11E0936A1174
:1090D00081E0808717821682CF0161E80E943F48B5
:1090E0000895FC01009741F080858150823020F482
:1090F00081E0818780936E11089521E030E0FC01CA
:109100008085882311F420E030E0C9010895CF93D1
:10911000DF93EC014A815B818C819D8160E070E08E
:109120000E944A884A815B8188819981489F900189
:10913000499F300D589F300D11248E819F8160E032
:1091400070E0A9010E944A88DF91CF910895FC0147
:109150008281938120E030E019C0A481B581A20F03
:10916000B31F4C91442381F481E08C934081518161
:10917000249FC001259F900D349F900D11242681BE
:109180003781280F391F07C02F5F3F4F2817390736
:1091900020F320E030E0C9010895FC0126813781E9
:1091A0004281538180E090E018C02617370781F490
:1091B000A481B581A80FB91F2C91121614F4215067
:1091C0002C930480F581E02DE80FF91F808108952C
:1091D000A081B1812A0F3B1F01968417950728F3C0
:1091E0008FEF0895FC01CB01268137816217730749
:1091F00090F0A081B18162817381A69FA001A79F99
:10920000500DB69F500D1124420F531F21E030E046
:109210008417950710F020E030E0C9010895FC01A3
:10922000118210820895FC01808191810895FB01D3
:1092300020813181FC01318320830895FC0120814C
:1092400031812115310511F407C09C01F90180819C
:1092500091810097D1F702C020E030E0C901089564
:10926000CF93DF93DC012D913C91119721153105AE
:10927000A9F0F90180819181009729F411961C923F
:109280001E920EC0F90120813181D9018D919C91EE
:1092900011970097B9F71182108202C020E030E0E8
:1092A000C901DF91CF910895DC01ED91FC911197F7
:1092B000309729F08081918111969C938E93CF01F4
:1092C0000895CF93DF93FC01A081B1811097D9F06D
:1092D000C0E0D0E016C0A617B70771F48D919C913D
:1092E0001197209719F49183808302C09983888312
:1092F00011961C921E9207C0ED0198818981A92FB9
:10930000B82F109741F7DF91CF9108950F931F93D6
:10931000CF93DF938C01EB010E946149F8018081BA
:10932000918199838883D183C083DF91CF911F91ED
:109330000F910895EF92FF920F931F93CF93DF93B6
:10934000EC017B010E946149F70111821082CE017C
:109350000E941E49FC01009719F4E882F98202C0BC
:10936000F182E082DF91CF911F910F91FF90EF90FA
:109370000895DC01ED91FC91119720E030E005C0EB
:109380002F5F3F4F0190F081E02D3097C9F7C90161
:109390000895FB01309721F4BA010E94864908958F
:1093A000DA018081918111969C938E935183408341
:1093B0000895009721F0FC012081318102C020E056
:1093C00030E0C901089580911A1290911B12009704
:1093D00029F410921D1210921C1208950E948F59A8
:1093E000E0911A12F0911B12228133814081518148
:1093F000240F351F281B390B0CC04281538160811B
:109400007181460F571F481B590B4217530708F429
:109410009A010480F581E02D309779F7280F391FE4
:1094200030931D1220931C12089589E892E00E9447
:1094300071480895CF92DF92EF92FF920F931F939E
:10944000CF93DF937C01FC0180819181009729F00B
:109450008A35910509F06EC00BC010921B12109254
:109460001A128AE590E0F7019183808381E066C05B
:10947000673849F5CA01E0911A12F0911B1203C036
:109480000480F581E02D309741F32681378128173C
:109490003907B1F3E0931A12F0931B120FC016961E
:1094A0002D913C9117972817390739F414962D916F
:1094B0003C91159735832483DF01FD01A481B5819B
:1094C000109769F7CECF623861F6C0911A12D09129
:1094D0001B1200E010E02BC0CE010E94F268009742
:1094E000F1F08E819F8168E8AE010E941C480097D0
:1094F000A1F41F821E828C819D810115110521F02E
:10950000F8019583848304C090931B1280931A12F0
:109510001D821C820E94E349D8CF0E94154A8E0109
:109520009C818D81C92EE6016E01D82EE60120971F
:1095300099F697CFF7011182108283E0DF91CF91E6
:109540001F910F91FF90EF90DF90CF900895CF93F0
:10955000DF93EC010E94154A8E819F81009769F08C
:10956000E0911A12F0911B1206C0EC17FD07A9F04A
:109570000480F581E02D3097C1F780916C119091B6
:109580006D119F838E8380911A1290911B129D837F
:109590008C83D0931B12C0931A120E94E349DF916F
:1095A000CF910895CF93DF93EC010E94D268CE0152
:1095B0000E94A74ADF91CF910895CF93DF93EC01EA
:1095C0000E94DE68CE010E94A74ADF91CF910895E4
:1095D000CF93DF93EC010E94E868CE010E94A74A76
:1095E000DF91CF910895FC0180819181860F971FB3
:1095F000918380830E94E349089521E030E0FC01DB
:1096000086819781009711F020E030E0C90108952C
:10961000FC012281338180819181280F391FC9018A
:109620000895FC0180819181089521E030E08091CE
:109630001A1290911B12009711F420E030E0C9013A
:10964000089580911A1290911B12009729F0209191
:109650001C1230911D1202C020E030E0C9010895B3
:10966000CF93DF93EC01E0911A12F0911B128E1749
:109670009F0741F48C819D8190931B1280931A1255
:1096800014C0FC01309731F0848195818C179D07BF
:10969000C1F707C01D821C821F821E82DF91CF91FD
:1096A00008958C819D81958384830E94E349F2CF44
:1096B000CF92DF92EF92FF920F931F93CF93DF939E
:1096C0008C017A01FC0180819181009729F08B3413
:1096D000910509F051C01EC08FE192E10E9413492B
:1096E000C82EE6017E01F92EE70109C06C817D815B
:1096F000CE0102960E94D24A0990D881C02D2097AF
:10970000A9F781E080931E128BE490E0F801918329
:10971000808337C06838A9F58FE192E10E94134930
:10972000C82EE6016E01D92EE60123C0CE010296B5
:10973000E816F906D9F48FE192E1BE010E94614971
:10974000E0906C11F0906D118A859B8590936D115E
:1097500080936C11EC85FD85309719F08E859F857F
:109760000995F0926D11E0926C11CECF0990D881DD
:10977000C02D2097D9F6C8CFF8011182108283E05E
:1097800001C081E0DF91CF911F910F91FF90EF9089
:10979000DF90CF90089510921E128FE192E10E9407
:1097A0000F4982EA92E060E070E00E944E4808951E
:1097B0000F931F93CF93DF93EC0100916C111091E5
:1097C0006D111B870A875D874C873F872E878091A5
:1097D0001E12882379F082EA92E090936D118093B3
:1097E0006C11CE0102960E94D24A10936D11009323
:1097F0006C1102C07D836C838FE192E1BE010E94F7
:1098000061498FE192E1BE010E949A49DF91CF91B7
:109810001F910F9108950F931F93CF93DF93EC0146
:1098200080911E12882391F000916C1110916D119E
:1098300082EA92E090936D1180936C11CE010296B2
:109840000E94DD4A10936D1100936C118FE192E13B
:10985000BE010E9461498FE192E1BE010E949A49D6
:10986000DF91CF911F910F9108950F931F93CF9385
:10987000DF93EC0180911E12882391F000916C110E
:1098800010916D1182EA92E090936D1180936C11AA
:10989000CE0102960E94E84A10936D1100936C115C
:1098A0008FE192E1BE010E9461498FE192E1BE0128
:1098B0000E949A49DF91CF911F910F910895CF9304
:1098C000DF93EC0180911E12882329F0CE010296CD
:1098D0000E94304B04C01F821E82198618868FE1B9
:1098E00092E1BE010E946149DF91CF910895CF932B
:1098F000DF93EC0180911E12882331F0CE01029695
:109900000E94FD4A9C0114C08FE192E10E9413491C
:10991000E82FF92F06C0EC17FD0741F00190F08108
:10992000E02D3097C1F721E030E002C020E030E0C8
:10993000C901DF91CF9108950F931F930091E827FC
:109940001091E9270E94BC592DB73EB722553040EF
:109950000FB6F8943EBF0FBE2DBFEDB7FEB73196E0
:1099600025E23EE0ADB7BEB712963C932E93119719
:10997000028313821483158266837783808791879D
:109980008091DB299091DC29A091DD29B091DE291D
:1099900082879387A487B5878091DF299091E029FA
:1099A000A091E129B091E22986879787A08BB18B9E
:1099B0008091E3299091E429A091E529B091E629CD
:1099C000828B938BA48BB58B8091E7299091E829AA
:1099D000A091E929B091EA29868B978BA08FB18F4E
:1099E0008091EB299091EC29A091ED29B091EE297D
:1099F000828F938FA48FB58F8091EF299091F0295A
:109A0000A091F129B091F229868F978FA0A3B1A3DD
:109A10008091F3299091F429A091F529B091F6292C
:109A200082A393A3A4A3B5A38091F7299091F829C9
:109A3000A091F929B091FA2986A397A3A0A7B1A76D
:109A40008091FB299091FC29A091FD29B091FE29DC
:109A500082A793A7A4A7B5A78091FF299091002A78
:109A6000A091012AB091022A86A797A7A0ABB1AB1B
:109A70008091032A9091042AA091052AB091062A88
:109A800082AB93ABA4ABB5AB8091072A9091082A27
:109A9000A091092AB0910A2A86AB97ABA0AFB1AFCB
:109AA00080910B2A90910C2AA0910D2AB0910E2A38
:109AB00082AF93AFA4AFB5AFEDB7FEB7FF9680917D
:109AC0000F2A9091102AA091112AB091122A808316
:109AD0009183A283B383EDB7FEB7ED5BFF4F809117
:109AE000132A9091142AA091152AB091162A8083E6
:109AF0009183A283B383EDB7FEB7E95BFF4F8091FB
:109B0000172A9091182AA091192AB0911A2A8083B5
:109B10009183A283B383EDB7FEB7E55BFF4F8091DE
:109B20001B2A90911C2AA0911D2AB0911E2A808385
:109B30009183A283B383EDB7FEB7E15BFF4F8091C2
:109B40001F2A9091202AA091212AB091222A808355
:109B50009183A283B3830E94EE880091E82710913D
:109B6000E9272DB73EB72E5A3F4F0FB6F8943EBFA8
:109B70000FBE2DBF0E94BC59ADB7BEB7D2970FB66E
:109B8000F894BEBF0FBEADBFEDB7FEB7319626EB62
:109B90003DE012963C932E93119702831382148317
:109BA000158266837783808791878091232A90919D
:109BB000242AA091252AB091262A82879387A487F8
:109BC000B5878091272A9091282AA091292AB091BF
:109BD0002A2A86879787A08BB18B80912B2A909118
:109BE0002C2AA0912D2AB0912E2A828B938BA48BA4
:109BF000B58B80912F2A9091302AA091312AB09173
:109C0000322A868B978BA08FB18F8091332A9091C7
:109C1000342AA091352AB091362A828F938FA48F4F
:109C2000B58F8091372A9091382AA091392AB09126
:109C30003A2A868F978FA0A3B1A380913B2A909157
:109C40003C2AA0913D2AB0913E2A82A393A3A4A3CB
:109C5000B5A380913F2A9091402AA091412AB091CA
:109C6000422A86A397A3A0A7B1A780914B2A9091DF
:109C70004C2AA0914D2AB0914E2A82A793A7A4A75F
:109C8000B5A780914F2A9091502AA091512AB09166
:109C9000522A86A797A7A0ABB1AB0E94EE882DB73A
:109CA0003EB72E5C3F4F0FB6F8943EBF0FBE2DBFA0
:109CB0001F910F91089580E3809321120895EF92F0
:109CC000FF92CF93DF932091211230E0C0E3D0E0E8
:109CD000C21BD30B2A5D3D4EB901AE010E944188E3
:109CE000CE01DF91CF91FF90EF900895AF92BF9298
:109CF000CF92DF92EF92FF920F931F93CF93DF9358
:109D00007C01C0902212D09023122091211230E0C9
:109D10008601005D1F4F021B130B01381105E0F493
:109D2000C0E3D0E0C21BD30B2A5D3D4EB901AE01AA
:109D30000E944188CE0DDF1D209124123091251202
:109D40008091D8129091D912280F391FCE01B901F4
:109D5000A6010E94418802C000E010E0C801DF9126
:109D6000CF911F910F91FF90EF90DF90CF90BF9018
:109D7000AF90089590912112980F90932112089519
:109D800040912212509123129C014817590798F0D4
:109D90008091D8129091D912820F931F9093D9126B
:109DA0008093D812421B530B5093231240932212DC
:109DB00021E030E002C020E030E0C9010895909336
:109DC00023128093221208952091D8123091D91233
:109DD0002A5A3D4EC90108952091211230E02A5D92
:109DE0003D4EC901089521E030E080912412909108
:109DF000251242E18635940711F420E030E0C901D4
:109E000008950E94F34E009771F026E532E16091CB
:109E10002412709125124091221250912312C901EF
:109E20000E9441880895A091D812B091D91210973C
:109E3000B9F02091221230912312205D3F4FAA5A8F
:109E4000BD4EE6E5F2E180E390E003C04D91419321
:109E5000019682179307D4F31092D9121092D81258
:109E600008958091241290912512089580912212D4
:109E70009091231208959091211280E3891B0895F7
:109E800080E390912112891B20912212309123129C
:109E9000280F311DC90108951F93CF93DF93EC0163
:109EA00010912112812F90E08C179D076CF00E9479
:109EB000404F8C0F9D1F8138910530F41C1B10936F
:109EC000211221E030E002C020E030E0C901DF9142
:109ED000CF911F910895CF93DF93E2EFF7E21192B4
:109EE000119288E2E232F807D1F7C0E0D0E0CE016B
:109EF000880F991F8651984D61E772E00E94E045F6
:109F00002196C430D10599F7DF91CF910895109231
:109F1000D9121092D812109223121092221280E3BA
:109F20008093211286E592E190932512809324126A
:109F30000E946B4F08950F931F93CF93DF93EC0113
:109F40008B010E94874FD0932512C0932412109347
:109F5000231200932212DF91CF911F910F91089548
:109F6000CF92DF92EF92FF920F931F93DF93CF93E5
:109F700000D0CDB7DEB78C0169837A830E94874F0A
:109F800069817A81C62ED72E21E8C216D10418F035
:109F900030E8C32ED12C8091241290912512B80163
:109FA000A6010E944188D0922312C0922212C601BB
:109FB0000F900F90CF91DF911F910F91FF90EF9035
:109FC000DF90CF900895282F392FD901E2EFF7E2E3
:109FD00080E301900D928150E1F7862F972FDC01ED
:109FE000EAEEF7E288E001900D928150E1F70895E2
:109FF000E2EFF7E2282F392FD90180E30D9001928B
:10A000008150E1F7AAEEB7E2862F972FFC0188E096
:10A0100001900D928150E1F70895E82FF0E0EE0FE6
:10A02000FF1FEE50F84D7183608381E090E008954A
:10A03000E82FF0E0EE0FFF1FEE50F84D8081918188
:10A04000089590E0880F991F8654984D0E94E0452E
:10A0500081E090E00895282F30E0220F331F26542E
:10A06000384DC90108958115910511F00197F1F757
:10A070000895E0912528F091262890818091242848
:10A0800089230895E0912228F091232880819091DE
:10A090002428892B8083E0912728F091282880812B
:10A0A00090912428892B80830895E0912228F091B3
:10A0B0002328908180912428809589238083E091B2
:10A0C0002728F09128289081809124288095892341
:10A0D00080830895FF920F931F93E0912228F091BF
:10A0E0002328908180912428809589238083E09182
:10A0F0002728F0912828808190912428892B80831B
:10A100008FEB93E00E943350FFB6F894E09127283C
:10A11000F09128289081809124288095892380833C
:10A1200083E890E00E943350E0912528F0912628A2
:10A13000008110912428FFBE78948BE393E00E9465
:10A140003350E0912528F091262880819091242891
:10A15000892319F0802F812301C081E01F910F9185
:10A16000FF90089550932828409327287093232820
:10A1700060932228909326288093252881E090E000
:10A1800002C0880F991F2A95E2F7809324280E9425
:10A190006A5008950F931F93182F0FB7F894E0910A
:10A1A0002728F0912828808190912428892B80836A
:10A1B00083E090E00E943350112351F0E091272872
:10A1C000F09128289081809124288095892380838C
:10A1D00087E190E00E943350E0912528F0912628F5
:10A1E000808190912428892309F410E089E590E08A
:10A1F0000E943350E0912728F09128289081809187
:10A2000024288095892380830FBF8BE390E00E94F0
:10A210003350812F1F910F9108950F931F93182F83
:10A2200008E0812F81700E94CA5016958111106834
:10A230000150B9F7812F1F910F9108958FEF0E9460
:10A240000D510895DF92EF92FF920F931F93CF93DA
:10A25000DF93182FEB010E946A50882389F580EF65
:10A260000E940D51EE2400E498EFD92ED00E81E02B
:10A270000E94CA50F82E81E00E94CA50882319F02B
:10A28000FF2069F020C0FF2051F4011728F08881D9
:10A2900080FF05C0101719F0E02EFF24F3948F2DD6
:10A2A0000E94CA50888186958883FF2011F08068BB
:10A2B000888301500D15D9F6002339F02196D4CFAB
:10A2C000EE24EA9402C08EEFE82E8E2DDF91CF911E
:10A2D0001F910F91FF90EF90DF9008950F931F93C0
:10A2E000CF93DF93182FEB010E946A50209751F013
:10A2F00085E50E940D5108E089910E940D510150A1
:10A30000D9F703C08CEC0E940D51812F0E940D5192
:10A31000DF91CF911F910F9108950F931F93CF93CA
:10A32000DF93FB01DA01E801408150E0718160E0D8
:10A33000462B572B803171F4BA016E7F13E0660F04
:10A34000771F1A95E1F796814CE050E0491B5109BF
:10A35000460F571F57FF06C091E09C9350954195BB
:10A360005F4F01C01C92883289F4848190E0BC0167
:10A37000607670706036710549F086FF02C04E7FCE
:10A3800005C085FF02C04C7F01C0487FCA0154E070
:10A39000969587955A95E1F7F90180834F70488328
:10A3A00080E0DF91CF911F910F9108950F931F933C
:10A3B000CF93DF938C01EB01F8018081BE010E94F5
:10A3C0002251F801808381508D3F28F488818832A2
:10A3D00011F0803189F7DF91CF911F910F9108958E
:10A3E0001F93CF93DF93EC010E946A5084EBBE0170
:10A3F0000E946E5181E00E94CA50182F0E946A503C
:10A4000081E0112309F480E0DF91CF911F9108953D
:10A410001F93CF93DF93182FEB010E946A500E9485
:10A420003950882349F084E4BE010E946E511130F6
:10A4300029F00E94425002C082E001C080E0DF911A
:10A44000CF911F9108956F927F928F929F92AF92BA
:10A45000BF92CF92DF92EF92FF920F931F93DF9301
:10A46000CF93CDB7DEB729970FB6F894DEBF0FBEF6
:10A47000CDBF7C014B013A0159010E946A508EEB1D
:10A48000B7010E946E518E010F5F1F4F8AE0C82EE8
:10A49000D12CCC0EDD1E0E941E51F80181938F013C
:10A4A000EC15FD05C1F78E010F5F1F4FC80169E074
:10A4B00070E00E94A36D882351F4F7018081B801F8
:10A4C000A401930185010E948D5180E001C083E0C9
:10A4D00029960FB6F894DEBF0FBECDBFCF91DF91A6
:10A4E0001F910F91FF90EF90DF90CF90BF90AF90B2
:10A4F0009F908F907F906F9008957F928F929F9200
:10A50000AF92BF92CF92DF92EF92FF920F931F9381
:10A51000DF93CF93CDB7DEB729970FB6F894DEBFA0
:10A520000FBECDBF782E5B014A0179018EEB60E052
:10A5300070E00E946E518E010F5F1F4F9AE0C92E8E
:10A54000D12CCC0EDD1E0E941E51F80181938F018B
:10A55000EC15FD05C1F78E010F5F1F4FC80169E0C3
:10A5600070E00E94A36D882349F4872DB801A501EE
:10A57000940187010E948D5180E001C083E02996FB
:10A580000FB6F894DEBF0FBECDBFCF91DF911F9104
:10A590000F91FF90EF90DF90CF90BF90AF909F9082
:10A5A0008F907F9008950F931F93DF93CF93CDB734
:10A5B000DEB728970FB6F894DEBF0FBECDBF182FB9
:10A5C000062FDE011196E4EBF2E088E001900D9297
:10A5D0008150E1F7242F332727FD309541E752E0E2
:10A5E000249FC001259F900D349F900D112464E697
:10A5F00070E00E946982AB0164E6069FB0011124FD
:10A60000460F571FFE013196CE010996619170E009
:10A610002617370719F44F5F5F4F03C0E817F90794
:10A62000A9F7112319F0509541955F4FCA0128965B
:10A630000FB6F894DEBF0FBECDBFCF91DF911F9153
:10A640000F9108950F931F93DF93CF93CDB7DEB78C
:10A650002B970FB6F894DEBF0FBECDBF182F092F72
:10A66000885F612F792F0E940852882309F049C022
:10A6700066E471E48FE090E00E948F53812F902F69
:10A68000BE016F5F7F4FAE014E5F5F4F9E012D5F3A
:10A690003F4F0E9423528823A1F5DE011496ECEA75
:10A6A000F2E088E001900D928150E1F74B81642F38
:10A6B00070E021E732E0629FC001639F900D729FBE
:10A6C000900D112464E670E00E9469829A8184E60C
:10A6D000989FC0011124680F791FFE013496CE01A6
:10A6E0000C962191421719F46F5F7F4F03C0E81752
:10A6F000F907B9F78981882331F0709561957F4F0B
:10A7000002C064E371E2CB012B960FB6F894DEBF72
:10A710000FBECDBFCF91DF911F910F910895DC0146
:10A72000CB0181159105A105B10529F0815090401B
:10A73000A040B040D9F708951092B90080E280930C
:10A74000B800089594EA9093BC0020EA36E841E00E
:10A7500050E005C02150304040405040F1F0909111
:10A76000BC0097FFF7CF1DC09031B9F48093BB00B8
:10A7700084E88093BC0080EA96E8A1E0B0E004C0E1
:10A780000197A109B10959F02091BC0027FFF8CF2A
:10A790000EC081E0903421F40FC081E0089581E083
:10A7A00008959091B900987F9830F1F6DFCF90919D
:10A7B000B900987F983169F780E0089544EA34E859
:10A7C00024E94093BC009091BC0097FFFCCF90918E
:10A7D000B900987F983011F0903199F78093BB00C1
:10A7E0003093BC009091BC0097FFFCCF9091B900D2
:10A7F000987F903211F0983539F42093BC009091F5
:10A80000BC0094FDFCCFDDCF08950E94A2530895B3
:10A8100084E98093BC008091BC0084FDFCCF089546
:10A820008093BB0084E88093BC008091BC0087FFCC
:10A83000FCCF9091B900987F81E0983209F480E0D4
:10A84000089584EC8093BC008091BC0087FFFCCF0E
:10A850008091BB00089584E88093BC008091BC0087
:10A8600087FFFCCF8091BB000895E82FF92F80E18E
:10A87000919190933F018150D9F780913C018F7D58
:10A8800080933C0180913C01877F80933C01862F1F
:10A89000972FFC0180E1919190933E018150D9F76F
:10A8A00080913C01806880933C0180913D0180FF54
:10A8B000FCCF4051504080913C01806280933C012C
:10A8C00080913C01877F80933C0114C0862F972F95
:10A8D000FC0180E1919190933E018150D9F78091E4
:10A8E0003C01806880933C0180913D0180FFFCCF5A
:10A8F00040515040141615064CF3822F932FFC0143
:10A9000080E190913E0191938150D9F781E090E0F0
:10A9100008950F931F93CF93DF938C018CE70E94D0
:10A92000DE538CE70E941054C0E0D0E0F801819122
:10A930008F010E9410542196C031D105B9F70E94B1
:10A940000854DF91CF911F910F910895813039F410
:10A950008CE790E060E070E040E050E006C08CE7FB
:10A9600090E060E070E040EC50E00E9492100895AA
:10A97000813039F48CE790E060E070E04EE050E028
:10A9800006C08CE790E060E070E048E050E00E9494
:10A99000921008958CE790E060E070E041E050E0B4
:10A9A0000E9492106AE67AE080E090E00E948F5365
:10A9B00008958CE790E060E070E048E350E00E948A
:10A9C00092108CE790E060E070E049E350E00E9474
:10A9D00092108CE790E060E070E044E150E00E946B
:10A9E00092108CE790E060E070E048E750E00E9451
:10A9F00092108CE790E060E070E04EE550E00E943D
:10AA000092108CE790E060E070E04DE650E00E942C
:10AA100092106CE17AE186E090E00E948F538CE71F
:10AA200090E060E070E04CE050E00E9492108CE713
:10AA300090E060E070E041E050E00E9492108CE70E
:10AA400090E060E070E046E050E00E9492106AE61C
:10AA50007AE080E090E00E948F530895DF93CF93D7
:10AA6000CDB7DEB7A2970FB6F894DEBF0FBECDBF4D
:10AA7000DE011196ECEBF2E081E101900D92815044
:10AA8000E1F7DE015296EDECF2E081E101900D92EA
:10AA90008150E1F70E94D954CE0101960E94895459
:10AAA00082E00E94A6546AE67AE080E090E00E948C
:10AAB0008F53CE0142960E94895460E17EEA88E27B
:10AAC00090E00E948F5380E00E94B85460E17EEADB
:10AAD00088E290E00E948F5381E00E94B854A296D1
:10AAE0000FB6F894DEBF0FBECDBFCF91DF910895B2
:10AAF000DF92EF92FF920F931F93DF93CF9300D0DB
:10AB00000F92CDB7DEB7F82E042F122F213031F07F
:10AB1000223031F0243031F0283031F080E005C0AF
:10AB200081E003C082E001C083E00C3059F00E30B8
:10AB300011F4846007C0003111F4886003C0023151
:10AB400009F48C60613059F0623011F4806207C002
:10AB5000633011F4806403C0643009F48066682FA8
:10AB600060688F2D90E070E0AE014F5F5F4F23E093
:10AB700030E00E94A91069E07AE180E090E00E9454
:10AB80008F5381E0F82A8F2D0E94A2530E942154F6
:10AB900089830E9421548A83023119F40E9421542E
:10ABA0008B830E94215487FDF1CF0E942B540E9479
:10ABB000085469E07AE180E090E00E948F538F2D85
:10ABC0000E94A2530E94215489830E9421548A83A7
:10ABD000023119F40E9421548B830E94215429814F
:10ABE000023181F5622F70E080E090E03B814A8184
:10ABF00021FF12C0CB0177276627630F711D811DCE
:10AC0000911D342F20E040E050E0620F731F841F3D
:10AC1000951F8C6F9F6F0FC0CB0177276627630F3F
:10AC2000711D811D911D342F20E040E050E0620F26
:10AC3000731F841F951F0E94767F20E83FEF4FEF20
:10AC400057E41FC0722F60E08A81680F711D88274A
:10AC500077FD8095982F0E94767F0C3029F420E0B4
:10AC600030EE4FEF54E40DC00E3029F420E038EF01
:10AC70004FEF55E406C0003131F420E03EEF4FEFD6
:10AC800056E40E94D77E2FE632E143E050E40E9472
:10AC90005481D62EE72EF82E092F612F70E08827D9
:10ACA00077FD8095982F0E94767F9B01AC016D2DDA
:10ACB0007E2D8F2D902F0E94D77E0F900F900F909A
:10ACC000CF91DF911F910F91FF90EF90DF9008954A
:10ACD000E6E4F1E080812081908130818295869543
:10ACE0008695837022952F70822B832B92959F706F
:10ACF000892B0895DF92EF92FF920F931F93DF93BA
:10AD0000CF9300D0CDB7DEB780E06CE046E00E9484
:10AD1000505A89E18093C4001092C50082E080936C
:10AD2000C00080E00E94FA5A0E947F5984B784B71D
:10AD300084B784B784B7E9EAF0E322E432E43183EC
:10AD400020833A968DB79EB70A97E817F907B8F3AC
:10AD500000D000D082E79FE0ADB7BEB712969C93BB
:10AD60008E9311978EED92E014969C938E93139789
:10AD70000E94EE880F900F900F900F900E94BC6978
:10AD80000E949A4789E892E060E070E00E944E4895
:10AD90000E94CB4BE0912903F0912A0309950E9470
:10ADA000685690E00E94FA69CE0101960E94AD5863
:10ADB000882359F000D082E59FE0EDB7FEB792837B
:10ADC00081830E94EE880F900F908E010F5F1F4FBE
:10ADD000C8010E94FB450E94B7587C010E94BC58E4
:10ADE000BC01C701A8010E94075E0E9415580E947D
:10ADF000EC5D0E94C1580E94745F00D085E49FE022
:10AE0000ADB7BEB712969C938E9311970E94EE88B1
:10AE100000D0EDB7FEB7319601E41FE0ADB7BEB785
:10AE200012961C930E9311978A81828313820E943B
:10AE3000EE88EDB7FEB73196ADB7BEB712961C934C
:10AE40000E9311978981828313820E94EE880F905E
:10AE50000F908FE39FE0EDB7FEB7928381830E944E
:10AE6000EE880F900F900E94006AE091AC03F09181
:10AE7000AD030995E0919303F09194030995E09156
:10AE80005503F09156030995E0909103F0909203D9
:10AE90000091AA031091AB030E94E95DD82E0E9495
:10AEA0007C5F2DB73EB72A5030400FB6F8943EBFB6
:10AEB0000FBE2DBFEDB7FEB7319624E23FE0ADB730
:10AEC000BEB712963C932E931197F382E2821583BC
:10AED0000483D6821782808711860E94EE88E091D3
:10AEE000B603F091B7032DB73EB7265F3F4F0FB6BD
:10AEF000F8943EBF0FBE2DBF3097D1F00995BC012D
:10AF000000D000D081E19FE0ADB7BEB712969C9310
:10AF10008E93119780E890E00E945582EDB7FEB7BE
:10AF2000748363830E94EE880F900F900F900F90B0
:10AF300000D08FE09FE0ADB7BEB712969C938E9382
:10AF400011970E94EE880F900F9085ED93E060E0DE
:10AF500070E00E944E4881EF93E00E94A66800D006
:10AF600087E09FE0EDB7FEB7928381830E94EE8871
:10AF70000F900F900F900F90CF91DF911F910F9135
:10AF8000FF90EF90DF900895EF92FF920F931F9341
:10AF900080E880936100109261000E947A560E94BE
:10AFA000AA470E941B5B8091292890912A2800972C
:10AFB00029F0019790932A2880932928E0902B2844
:10AFC000F0902C2800912D2810912E280E94BC5919
:10AFD000E616F7060807190711F30E94BC5960939B
:10AFE0002B2870932C2880932D2890932E28D7CF30
:10AFF00000D000D000D0EDB7FEB7319621E03FE0A1
:10B00000ADB7BEB712963C932E931197938382836C
:10B01000758364830E94EE888DB79EB706960FB63F
:10B02000F8949EBF0FBE8DBF08950F931F93DF93BB
:10B03000CF93CDB7DEB7A2970FB6F894DEBF0FBEA1
:10B04000CDBF82E590E00E942B8A89839A83982F56
:10B050009B50903108F08A839A819095891709F462
:10B0600070C000D08DEA9FE0ADB7BEB712969C933A
:10B070008E9311970E94EE888E010D5F1F4F0F90E7
:10B080000F90D80180E090E0FC01E357F04FE4918D
:10B09000ED93019688309105B9F7F894CE010396A7
:10B0A00060E370E048E050E00E94318AD80180E01F
:10B0B00090E0FC01EB56F04FE491ED9301968E3059
:10B0C0009105B9F7CE01039668E370E04EE050E0D9
:10B0D0000E94318A80E090E0FC01ED55F04FE49150
:10B0E000D801ED938D0101968A309105A9F7CE0123
:10B0F000039666E470E04AE050E00E94318A84E5FD
:10B1000090E06DEC7BEA0E94498A86E590E060E081
:10B1100070E00E94498A88E590E060E00E943B8AE6
:10B1200080E590E060E070E00E94498A8AE18983CE
:10B1300085EE8A8369817A8182E590E00E94498A5E
:10B1400078948981A2960FB6F894DEBF0FBECDBF6A
:10B15000CF91DF911F910F910895F89460E370E013
:10B1600042E050E00E94138A789480E0089584E5DC
:10B1700090E00E942B8A089586E590E00E942B8A39
:10B18000089588E590E00E94238A08952091372849
:10B19000309138284091392850913A2890E0A0E029
:10B1A000B0E0280F391F4A1F5B1F209337283093C8
:10B1B00038284093392850933A28209133283091E9
:10B1C00034284091352850913628280F391F4A1FBE
:10B1D0005B1F2093332830933428409335285093B5
:10B1E00036282091D7292223A1F020912F283091B1
:10B1F00030284091312850913228280F391F4A1F9A
:10B200005B1F20932F283093302840933128509390
:10B21000322808951F920F920FB60F920BB60F921D
:10B2200011242F933F934F935F936F937F938F934B
:10B230009F93AF93BF93EF93FF938091DA12909116
:10B24000DB1201969093DB128093DA128091DC126C
:10B250008F5F8093DC128091DC128038A9F4109209
:10B26000DC128091372890913828A0913928B0912C
:10B270003A280196A11DB11D809337289093382854
:10B28000A0933928B0933A288091D7298823F1F0E8
:10B290008091DD128F5F8093DD128091DD12803806
:10B2A000A9F41092DD1280912F2890913028A0915E
:10B2B0003128B09132280196A11DB11D80932F280D
:10B2C00090933028A0933128B09332280E94154BD8
:10B2D000009711F00E94154AFF91EF91BF91AF9135
:10B2E0009F918F917F916F915F914F913F912F919E
:10B2F0000F900BBE0F900FBE0F901F901895F894F3
:10B300001092B60016BC83EF87BD82E084BD94E046
:10B3100095BD95B395BB80936E0078940895209168
:10B32000DA123091DB128091DA129091DB12281739
:10B330003907A9F7C901089507C022E330E00000EA
:10B3400021503040E1F701970097B9F708950F9326
:10B350001F93CF93DF938C010E948F59EC010E94C1
:10B360008F598C1B9D0B80179107C8F3DF91CF91EC
:10B370001F910F9108950895209137283091382812
:10B380004091392850913A28809137289091382857
:10B39000A0913928B0913A28281739074A075B0746
:10B3A00059F7B901CA0108951F920F920FB60F9273
:10B3B0001124109202030F900FBE0F901F9018954A
:10B3C0001F920F920FB60F920BB60F9211242F936C
:10B3D0003F934F935F936F937F938F939F93AF931D
:10B3E000BF93EF93FF93E091F802F091F90280810F
:10B3F000E0910303F0910403309709F00995FF9160
:10B40000EF91BF91AF919F918F917F916F915F91DC
:10B410004F913F912F910F900BBE0F900FBE0F9049
:10B420001F9018951F920F920FB60F921124109231
:10B430000F030F900FBE0F901F9018951F920F9241
:10B440000FB60F920BB60F9211242F933F934F9389
:10B450005F936F937F938F939F93AF93BF93EF937C
:10B46000FF93E0910503F09106038081E0911003C2
:10B47000F0911103309709F00995FF91EF91BF9179
:10B48000AF919F918F917F916F915F914F913F917C
:10B490002F910F900BBE0F900FBE0F901F9018951D
:10B4A00090E02DE030E0829FF001839FF00D929FAD
:10B4B000F00D1124E850FD4FA281B3811C92A481AC
:10B4C000B5816C93A681B78188ED8C93A085B185F9
:10B4D0004C93128614861386089590E02DE030E098
:10B4E000829FF001839FF00D929FF00D1124E85090
:10B4F000FD4F81E08287A081B1816C933A96808173
:10B500008823E9F708951F93182F8A3031F480912A
:10B51000DE126DE00E946D5A02C08D3029F08091DC
:10B52000DE12612F0E946D5A80E090E01F91089515
:10B53000EF92FF921F93CF93DF93182FE62EE70130
:10B540007E01F72EE7010CC08A3021F4812F6DE0D7
:10B550000E946D5A69916D3019F0812F0E946D5AC9
:10B560008881882389F7DF91CF911F91FF90EF9019
:10B5700008950F931F93DF93CF93CDB7DEB7FE01EE
:10B580003A960FED12E1C80160E470E048855985F4
:10B590009F010E947C898F81B8010E94985ACF91A7
:10B5A000DF911F910F9108951F93CF93DF93182F71
:10B5B000EB0104C0812F0E946D5A2196FE01649117
:10B5C0006623C1F7DF91CF911F91089590E02DE0A0
:10B5D00030E0829FF001839FF00D929FF00D1124C7
:10B5E000E850FD4F748763870895682F80E00E94BC
:10B5F0006D5A08958093DE128AEE92E09093A43003
:10B600008093A330089584B7877F84BF88E10FB605
:10B61000F89480936000109260000FBE08952FE0B0
:10B6200088E190E00FB6F894A895809360000FBE73
:10B63000209360000895A895089588E10FB6F894C6
:10B6400080936000109260000FBE0895F89428E087
:10B6500088E190E00FB6F894A895809360000FBE43
:10B6600020936000FFCF80914A2890E0FC01EE0F0C
:10B67000FF1F9695982F882797958795E80FF91FB4
:10B68000E55BF74D10820895809142288091422811
:10B6900090E008958091390181FD0CC081E491E032
:10B6A0006FE140E00E941D61813039F021E030E01F
:10B6B000813129F020E030E002C021E030E0C90112
:10B6C00008958091390181FD12C081E491E06FE11C
:10B6D00040E00E941D61982F8151823050F09F31CF
:10B6E00041F0913041F081E0923031F402C081E0CC
:10B6F000089580E0089580E008950E94615B8823AA
:10B70000E1F3089581E491E06FE140E00E941D6162
:10B710000895E9E3F1E0808180818D7F80838DE071
:10B7200090E00197F1F782E491E06FE140E023E0DF
:10B730000E94276183E090E00197F1F708950E944D
:10B740007D5B1092D7290E94895B809139018260CC
:10B750008093390180915A2A8823E9F180919400DD
:10B760009091950020916B2A30916C2A8217930753
:10B77000A0F48091372A9091382AA091392AB0916B
:10B780003A2A8C57914EAF4FBF4F8093372A9093F0
:10B79000382AA093392AB0933A2A80919400909144
:10B7A0009500821B930BA0E0B0E02091372A3091E6
:10B7B000382A4091392A50913A2A820F931FA41FA8
:10B7C000B51F8093372A9093382AA093392AB093D3
:10B7D0003A2A10925A2A80915C2A8823E9F18091B2
:10B7E00094009091950020916F2A3091702A8217D1
:10B7F0009307A0F480913F2A9091402AA091412A7A
:10B80000B091422A8C57914EAF4FBF4F80933F2A41
:10B810009093402AA093412AB093422A80919400A9
:10B8200090919500821B930BA0E0B0E020913F2AFD
:10B830003091402A4091412A5091422A820F931F11
:10B84000A41FB51F80933F2A9093402AA093412ABA
:10B85000B093422A10925C2A08958091D7298823B8
:10B8600081F080911F13882321F40E94615B88235B
:10B8700031F481E08093A21321E030E004C00E9403
:10B880009F5B20E030E0C90108950F931F93182FAC
:10B89000883049F0863039F0893029F0863119F046
:10B8A000893109F041C08091390181FD40C00E9479
:10B8B0007D5B0E94825B082F181709F43BC018308B
:10B8C00019F40E94895B29C0193141F48631A9F429
:10B8D00082E491E06FE140E029E009C0163169F4AB
:10B8E000893159F482E491E06FE140E026E00E9462
:10B8F0002761E3E0F0E03197F1F782E491E06FE156
:10B9000040E0212F0E942761083019F4E9E6F1E0B8
:10B9100002C0E3E0F0E03197F1F70E94825B81170B
:10B9200049F023E430E008C022E430E005C024E41C
:10B9300030E002C020E430E0C9011F910F9108956A
:10B9400080919400909195009093702A80936F2A33
:10B9500021E020935C2A8091390181FF15C020935A
:10B96000D629809194009091950090936C2A8093B1
:10B970006B2A20935A2A809139018D7F8093390157
:10B980008091D6298823E1F786E10E94455C81E019
:10B990008093D72908958091D729882351F48091E5
:10B9A0001F13882321F081E08093A11302C00E941D
:10B9B000A05C81E090E008951F93DF93CF930F92F6
:10B9C000CDB7DEB78FB7898380911F13882331F5F8
:10B9D000F8948091D729882351F08091390181FD15
:10B9E0001BC00E94615B8823B9F080E003C00E9405
:10B9F000CB5C81E0909147019E3010F010E001C0D7
:10BA00001FEF882311F00E942D5C16FF05C089816D
:10BA10008FBF21E030E004C089818FBF20E030E09B
:10BA2000C9010F90CF91DF911F9108958091A113CB
:10BA3000882321F00E94A05C1092A1138091A21390
:10BA4000882321F00E949F5B1092A21310921F1373
:10BA50000895EF92FF92CF93DF93B82FA92FF62F7F
:10BA6000E72F81E080931F1320911B2A30911C2A1D
:10BA700040911D2A50911E2A2F5F3F4F4F4F5F4F1D
:10BA800020931B2A30931C2A40931D2A50931E2A70
:10BA9000862F8E5F87FF0CC08091D4299091D52985
:10BAA00001969093D5298093D429CFEFDFEF0BC077
:10BAB00020E233E1C9016B2F7A2F4F2F5E2F0E94B6
:10BAC0004188C0E0D0E00E94165DCE01DF91CF91A9
:10BAD000FF90EF9008959091390191FD0AC0282FB1
:10BAE000803108F02FE085E491E06FE040E00E94B3
:10BAF000276108958093A41308950E94825B825069
:10BB0000813130F4E82FF0E0E35CFC4F8081089550
:10BB100081E0089508958FEF80934E018CE691E0C7
:10BB200060EF44E022E00E9427618CE290E06EE04A
:10BB300041E025E00E94276180E880936F018091B9
:10BB4000460180936D0184E491E060E245E021E0EC
:10BB50000E9427610895CF93DF93CDEFD3E0CE010C
:10BB60000197F1F70E94136110924B281092CD2893
:10BB700010924F2910924A2810924928E9E3F1E0E7
:10BB800080818E7F808380818D7F80838DE090E0B7
:10BB90000197F1F780818160808382E491E06FE119
:10BBA00040E023E00E9427612197F1F780915D0139
:10BBB00080915E010E948B5D8FE193E060E070E018
:10BBC0000E944E480E94A05C81E090E0DF91CF91FE
:10BBD00008958091A3130895DF93CF930F92CDB76B
:10BBE000DEB789830E947D5B29812093A31388E4BB
:10BBF00091E06FE140E00E9427610F90CF91DF91CB
:10BC000008950E94EC5D86E00E94455C0895809353
:10BC1000620190936301609360017093610141152B
:10BC2000510531F1FA01819180936B01DA0111968E
:10BC30008C9180936A01DF01119681818093690163
:10BC4000FD01319611968C9180936801DF01119668
:10BC5000818180936701FD01319611968C91119736
:10BC60008093660181818093650182818093640164
:10BC700008958FE193E00E94714881E0809342280B
:10BC80008091432890914428019690934428809372
:10BC9000432881E090E00895EF92FF92CF93DF93E5
:10BCA00050914A28252F30E0F901EE0FFF1F3695FD
:10BCB000322F222737952795E20FF31FE55BF74DCB
:10BCC0004081442309F4CEC02091390121FDCAC02E
:10BCD0002091D729222309F4C5C047FF16C00E942E
:10BCE000335B80910B2A90910C2AA0910D2AB09180
:10BCF0000E2A0196A11DB11D80930B2A90930C2A48
:10BD0000A0930D2AB0930E2AADC04330B0F40E9428
:10BD1000335B8091072A9091082AA091092AB0915B
:10BD20000A2A0196A11DB11D8093072A9093082A23
:10BD3000A093092AB0930A2A95C0C42FD0E0229775
:10BD40006C177D07B0F40E94335B8091032A9091B9
:10BD5000042AA091052AB091062A0196A11DB11DC1
:10BD60008093032A9093042AA093052AB093062A6D
:10BD700079C0652F70E09B01220F331F7695762FD7
:10BD8000662777956795260F371F245B374DB901D6
:10BD900050E00E94418820914A28822F90E0FC01C7
:10BDA000EE0FFF1F9695982F882797958795E80F98
:10BDB000F91FE553F74D808180933B28822F90E057
:10BDC000FC01EE0FFF1F9695982F88279795879572
:10BDD000E80FF91FE55BF74D10822F5F20934A288B
:10BDE000233010F010924A2880914A2890E0FC01FC
:10BDF000EE0FFF1F9695982F882797958795E80F48
:10BE0000F91FE55BF74D8081882311F00E94395EB0
:10BE10006091470160933C2880914128882311F06C
:10BE2000681710F46093412884E070E00E940D5080
:10BE300060913B2883E070E00E940D5080911F2AA2
:10BE40009091202AA091212AB091222A0196A11D29
:10BE5000B11D80931F2A9093202AA093212AB0938A
:10BE6000222A02C0C0E0D0E0CE01DF91CF91FF9046
:10BE7000EF900895CF93DF93EC018881998100972B
:10BE800029F024E08B3F920739F505C08BEF94E051
:10BE90009983888325C0623819F5109242280E9440
:10BEA000874F0E94E44E60E870E00E944C5E1816D6
:10BEB000190644F40E94DF4EE091B003F091B10303
:10BEC0000995E4CF80913F28909140280196909366
:10BED000402880933F28DACF1982188283E001C07E
:10BEE00081E0DF91CF91089591E090931F130E941C
:10BEF0006B5D0E94165D08958091390181FD07C038
:10BF000085E491E06FE040E00E941D61089580E1CA
:10BF10000895CF92DF92EF92FF920F931F93CF93EA
:10BF2000DF93182F21E020931F130091D7298091D0
:10BF3000390181FF16C080919400909195009093F3
:10BF40006C2A80936B2A20935A2A2093D6298091B9
:10BF500039018D7F809339018091D6298823E1F7BB
:10BF600000E00E947D5B8091D729882309F441C0BD
:10BF700080915C2A8823E9F120919400309195000A
:10BF800080916F2A9091702A28173907A0F4209188
:10BF90003F2A3091402A4091412A5091422A2C5701
:10BFA000314E4F4F5F4F20933F2A3093402A4093AA
:10BFB000412A5093422A2091940030919500281BE9
:10BFC000390B40E050E0C0903F2AD090402AE090EA
:10BFD000412AF090422A2C0D3D1D4E1D5F1D2093DD
:10BFE0003F2A3093402A4093412A5093422A10928C
:10BFF0005C2A89E10E94455C86E00E941850009707
:10C0000051F00E947C5FC82F86E00E94185081503A
:10C010000E946B5D02C0C0E0D0E0809194009091DE
:10C02000950090936E2A80936D2A81E080935B2A1D
:10C03000F8948091390182608093390180913901AF
:10C040008D7F80933901612F6E5F80E293E10E94C2
:10C05000586178948091D1299091D229019690933A
:10C06000D2298093D1290E947D5B82E491E060EE29
:10C0700045E00E941D61182F86E00E94185000972D
:10C0800019F08C2F0E946B5D002319F00E94A05CB8
:10C0900002C00E949F5B80915B2A8823E9F1809116
:10C0A00094009091950040916D2A50916E2A8417CA
:10C0B0009507A0F480913B2A90913C2AA0913D2ABB
:10C0C000B0913E2A8C57914EAF4FBF4F80933B2A81
:10C0D00090933C2AA0933D2AB0933E2A209194004D
:10C0E00030919500241B350B40E050E080913B2AB5
:10C0F00090913C2AA0913D2AB0913E2A280F391FE9
:10C100004A1F5B1F20933B2A30933C2A40933D2AD1
:10C1100050933E2A10925B2A8091D729882361F0A0
:10C1200080919400909195009093702A80936F2A4B
:10C1300081E080935C2A07C082E491E06FE140E0F7
:10C1400023E00E9427610E94165D1130E1F0133058
:10C15000A9F48091132A9091142AA091152AB091E4
:10C16000162A0196A11DB11D8093132A9093142ABB
:10C17000A093152AB093162A12E00AC0153029F0B0
:10C18000173031F404C010E003C013E001C011E027
:10C19000812F90E0DF91CF911F910F91FF90EF9051
:10C1A000DF90CF900895CF93DF93EB010E94295D3C
:10C1B0009C01009731F4CE010E94895F9C01009799
:10C1C00049F08091D4299091D52901969093D52951
:10C1D0008093D429C901DF91CF9108950F931F93C4
:10C1E0008091D729882321F40E94CB5C11E001C003
:10C1F00010E00E94825B863111F0813119F40091C8
:10C20000470109C086E491E06FE140E00E941D61B2
:10C21000082F000F080F112311F00E942D5C802FB2
:10C220001F910F9108951092A6131092A513EFE697
:10C23000F0E08081806280830895FC018081862304
:10C2400090E002C0959587954A95E2F70895F89495
:10C25000FC019081862F8095892330E002C0220F57
:10C26000331F4A95E2F72623282B208378940895DC
:10C27000DC01119620917B01FC012083215030E0EC
:10C28000A9014F575E4FE0E8F1E061916D93E4172B
:10C29000F507D9F7FC01E058FF4F2F573E4FD90162
:10C2A0002C9120838F579F4F21E0FC01208308951C
:10C2B000FC016093800101966350860F911DA1E8F7
:10C2C000B1E021912D93E817F907D9F708951F924E
:10C2D0000F920FB60F920BB60F9211242F933F932C
:10C2E0004F935F936F937F938F939F93AF93BF937E
:10C2F000EF93FF938091470180933C282091492838
:10C3000030E0C901880F991F3695322F22273795C3
:10C310002795820F931F855B974D0E94386180910E
:10C3200049288F5F80934928833010F01092492864
:10C330000E94395EFF91EF91BF91AF919F918F91D4
:10C340007F916F915F914F913F912F910F900BBE15
:10C350000F900FBE0F901F9018951F920F920FB65F
:10C360000F9211240F900FBE0F901F9018951F92DF
:10C370000F920FB60F9211240F900FBE0F901F90C7
:10C3800018951F920F920FB60F9211240F900FBEA7
:10C390000F901F9018951F920F920FB60F921124B5
:10C3A0001092D6290F900FBE0F901F9018951F92D4
:10C3B0000F920FB60F9211241092D6290F900FBE34
:10C3C0000F901F9018951F920F920FB60F92112485
:10C3D0008F9381E0809342288F910F900FBE0F9032
:10C3E0001F9018951F920F920FB60F921124109262
:10C3F000D6290F900FBE0F901F9018951F920F9285
:10C400000FB60F9211248F939F938091A513909153
:10C41000A61301969093A6138093A5139F918F91D5
:10C420000F900FBE0F901F9018950F931F93CF93EF
:10C43000DF938091DF299091E029A091E129B091CB
:10C44000E2290196A11DB11D8093DF299093E02977
:10C45000A093E129B093E2290E94C664EC0187EA27
:10C4600093E10E9413490BC0D8011296ED91FC9103
:10C470001397309709F00995C8010E94D949082FF0
:10C48000192F0115110581F7209719F0CE010E948F
:10C490008346DF91CF911F910F9108950E94006A0A
:10C4A0000E94874F0E94D06281E993E09093DA293D
:10C4B0008093D9290E94C36482E090E060E074E038
:10C4C00040E05EE12FEF31E00E9484640895CF9256
:10C4D000DF92EF92FF920F931F93CF93DF936C0144
:10C4E000EB018A0187EA93E10E9413490CC0D7014E
:10C4F0001496ED91FC911597309711F0CE010995A6
:10C50000C7010E94D949E82EF92EE114F10479F708
:10C51000C601BE01A8010E948B46DF91CF911F91F9
:10C520000F91FF90EF90DF90CF900895BC0187EAC4
:10C5300093E10E949A490895BC0187EA93E10E9421
:10C5400061490895CF93DF93EC018091DB299091AD
:10C55000DC29A091DD29B091DE290196A11DB11D34
:10C560008093DB299093DC29A093DD29B093DE2909
:10C57000CE010E94DD64009769F00E94014FE091B6
:10C580009503F091960387E692E6BE01099521E0B6
:10C5900030E002C020E030E0C901DF91CF91089582
:10C5A00089EA93E10E940F4908950F93CF93DF9397
:10C5B000EC017B836A8318865F834E8389EA93E16B
:10C5C000BE010E949A49E091AB13F091AC133097F1
:10C5D00049F04C815D818A819B81688520E030E053
:10C5E00001E00995DF91CF910F910895BC0189EA8F
:10C5F00093E10E94614908950F93DC0118961C9203
:10C600001897E091AB13F091AC13309759F0129654
:10C610008D919C91139760E040E050E020E030E085
:10C6200000E009950F9108950F93DC01AB0114967A
:10C630002D913C91159781E018968C93189715963B
:10C640007C936E931497E091AB13F091AC133097F9
:10C6500039F012968D919C91139761E000E0099555
:10C660000F9108950F93DC01E091AB13F091AC139F
:10C67000309769F014962D913C91159712968D91F3
:10C680009C91139718966C91A90101E009950F915F
:10C690000895E091AD13F091AE13309709F009952C
:10C6A00008959093AE138093AD1308959093AC13B7
:10C6B0008093AB13089589EA93E10E94134908958A
:10C6C000EF92FF920F931F93CF93DF938C01EB01B7
:10C6D0007A0189EA93E10E94134915C0DC011296A0
:10C6E0002D913C9113972C173D0759F41696ED9117
:10C6F000FC911797309761F0B801AE019701099549
:10C7000007C00E94D949282F392FC901009731F756
:10C71000DF91CF911F910F91FF90EF9008950895B1
:10C72000AF92BF92CF92DF92EF92FF920F931F933F
:10C73000DF93CF9300D0CDB7DEB75B010E94E44E0C
:10C74000FC01008111811A8309830C30110518F452
:10C75000EE24FF242EC000D000D089E593E0EDB791
:10C76000FEB792838183148303830E94DC880F9039
:10C770000F900F900F9020C00E94E44EF701EE0F33
:10C78000FF1FEE0FFF1FE80FF91FC280D3800E942A
:10C79000E44E0894E11CF11CF701EE0FFF1FEE0FB1
:10C7A000FF1FE80FF91F40815181C501B6010E94AA
:10C7B0006063E016F10600F30F900F90CF91DF91C8
:10C7C0001F910F91FF90EF90DF90CF90BF90AF90AF
:10C7D0000895CF93DF93CAECD3E16091E013709199
:10C7E000E113CE014BE154E620E030E00E94D84B4B
:10C7F0000E94FD696091E0137091E1130E945582DF
:10C80000BC01CE01409740E354E620E030E00E94B6
:10C81000D84BDF91CF9108950F93013051F480915F
:10C82000DA139091DB139093E1138093E0130E944D
:10C83000E9630F9108958091E0139091E1132091A5
:10C84000DE133091DF13880F991F2817390708F47A
:10C85000C9019093E1138093E0130E94E963089566
:10C86000EF92FF92CF93DF930E94874F0E94E44E96
:10C87000E82EE7017E01F92EE701198218820E9455
:10C880005B6326C028813981F901EE0FFF1FEE0F8F
:10C89000FF1FEC0FFD1FDC0112964D915C91139769
:10C8A000538342832F5F3F4FF901EE0FFF1FEE0FBF
:10C8B000FF1FEC0FFD1F14964D915C91159751834E
:10C8C0004083398328830E94D949282F392FC901F1
:10C8D000009721F0FC0120852223A1F6888199810F
:10C8E000880F991F880F991F02960E94DF4E88813A
:10C8F0009981009721F08FEA93E10E945646DF91DB
:10C90000CF91FF90EF900895EF92FF920F931F93B6
:10C91000CF93DF93FC018B017A01E9018FEA93E168
:10C92000BF0146E753E00E9438461093DB130093A3
:10C93000DA13F092DD13E092DC13D093DF13C0938F
:10C94000DE138CE094E60E945663DF91CF911F9135
:10C950000F91FF90EF900895CF93DF93CAECD3E14E
:10C96000CE010E945F4CCE0140970E945F4CCE01E9
:10C970004B970E945346DF91CF9108958091E01329
:10C980009091E11308950E9497460895EF92FF92C7
:10C99000CF93DF93E0917A03F0917B030995EC014B
:10C9A000009729F06A817B8181E00E940D50CE01C1
:10C9B000DF91CF91FF90EF9008950F931F93CF9346
:10C9C000DF938C01E0917C03F0917D030995EC01EC
:10C9D000F8016281738181E00E940D5021E030E016
:10C9E000209711F420E030E0C901DF91CF911F9131
:10C9F0000F910895E0917E03F0917F0309950895CA
:10CA0000FC0120E030E004C08181280F311D329606
:10CA100080818823C9F7C9010895FC01818190E0D4
:10CA2000308120E0822B932B02C0880F991F6A95DA
:10CA3000E2F7892F9927FA01E058FC4F208130E076
:10CA40008223932328E030E0241B350B02C0969507
:10CA500087952A95E2F708956F927F928F929F9221
:10CA6000AF92BF92CF92DF92EF92FF920F931F93FC
:10CA7000CF93DF936C017B015A0189012830310586
:10CA800044F4CB01BA01A9010E940D65F60180832F
:10CA900041C0390133E0759467943A95E1F7411547
:10CAA000510521F04C01C0E0D0E016C0DB01FC01D3
:10CAB000C0E0D0E08D9181932196C615D705D4F3BF
:10CAC000A801477050704115510521F1C7018C0F25
:10CAD0009D1F60E070E019C0C7018C0F9D1FB5015C
:10CAE00048E050E00E940D65F40181934F012196CA
:10CAF000C615D7058CF3A801477050704115510534
:10CB000049F0C7018C0F9D1FB5010E940D65CC0D2A
:10CB1000DD1D8883DF91CF911F910F91FF90EF90E2
:10CB2000DF90CF90BF90AF909F908F907F906F904D
:10CB300008954F925F926F927F928F929F92AF92E1
:10CB4000BF92CF92DF92EF92FF920F931F93DF93EA
:10CB5000CF9300D000D0CDB7DEB70E94E44EE82ED0
:10CB6000092F82E090E00E94C04E009709F464C053
:10CB7000EE2DF02F918180E02081820F911D0E9487
:10CB8000AB467C01009709F459C00E94E44E3C0179
:10CB9000F7014681242F30E02770307081E090E06B
:10CBA0002115310511F480E090E0469546954695B3
:10CBB000840F911D0E94C04E0097F1F1F70104818E
:10CBC0001581CC24DD2453E0452E512C4C0E5D1EE6
:10CBD0004E010894811C911C2AC0F801A180BB243D
:10CBE000B60143E0759567954A95E1F7660D771DA7
:10CBF000A60147705070883150F0C40195010E9421
:10CC00002C65F8018081B4010E9421500CC01C8267
:10CC10001B82C20195010E942C656B817C81F80109
:10CC200080810E940D50CA0CDB1C0E5F1F4FF80163
:10CC30008081882391F602C0EE24FF24C7010F9063
:10CC40000F900F900F90CF91DF911F910F91FF9058
:10CC5000EF90DF90CF90BF90AF909F908F907F909C
:10CC60006F905F904F900895FC0150E080E190E05C
:10CC7000861B970B821B930B02C0440F551F8A958E
:10CC8000E2F78081852B80838181842B81830895C5
:10CC90006F927F928F929F92AF92BF92CF92DF92CC
:10CCA000EF92FF920F931F93CF93DF938C015B0161
:10CCB0006A0179012830310524F4C801FA01408164
:10CCC00056C0390163E0759467946A95E1F7A11441
:10CCD000B10421F04A01C0E0D0E021C0DA01F8013E
:10CCE00080E090E02D912193019686159705D4F36D
:10CCF00097012770307021153105D9F1F601E80F41
:10CD0000F91F408150E068E070E0621B730B02C0C5
:10CD1000559547956A95E2F7800F911F26C0F4015B
:10CD200041914F01C8018C0F9D1FB50128E030E0F3
:10CD30000E9434662196C615D7058CF3970127709B
:10CD4000307021153105A9F0F601EC0FFD1F40816F
:10CD500050E0C5010896821B930B02C0559547957C
:10CD60008A95E2F7C8018C0F9D1F60E070E00E9479
:10CD70003466DF91CF911F910F91FF90EF90DF907C
:10CD8000CF90BF90AF909F908F907F906F900895BD
:10CD90004F925F926F927F928F929F92AF92BF92CB
:10CDA000CF92DF92EF92FF920F931F93DF93CF9377
:10CDB00000D0CDB7DEB78C01DC0116964C911697EA
:10CDC000842F90E08770907021E030E0009711F49C
:10CDD00020E030E04695469546957901E40EF11C39
:10CDE000C70102960E944C4F009709F453C00E945D
:10CDF000EC4EFC01D80112968C9112978083139609
:10CE00008C9181830E94EC4EF2E06F2E712C680EA3
:10CE1000791EC30160E070E0A7010E944A88F80112
:10CE2000C480D58000E010E02E010894411C511C04
:10CE30002AC0D60111968C90119799247801E3E0CD
:10CE4000F594E794EA95E1F7E60CF71C77E0A72E56
:10CE5000B12CA022B122883130F00E942B50AC01BD
:10CE6000C701B50107C00E9418509A838983C70182
:10CE7000B501A20194010E944866080D191DE2E067
:10CE8000F0E0CE0EDF1ED6018C91882391F621E0D2
:10CE900030E002C020E030E0C9010F900F90CF9148
:10CEA000DF911F910F91FF90EF90DF90CF90BF9097
:10CEB000AF909F908F907F906F905F904F9008956C
:10CEC000E091AE03F091AF0309950895E091570307
:10CED000F091580309950895E091B203F091B303DE
:10CEE00009950895E091B403F091B503099508956B
:10CEF00080E090E008950895E0913903F0913A03BD
:10CF000009950895009731F0E0913903F0913A03C3
:10CF100009950895E0913B03F0913C03099508952C
:10CF200080E090E008950F931F93DF93CF93CDB7E8
:10CF3000DEB7E0970FB6F894DEBF0FBECDBF0E94FC
:10CF4000364F8C010E94E44E602FAE014F5F5F4F61
:10CF50000E94C66F882309F445C088A99801281B40
:10CF60003109C9010E94C04E0097E1F12E812223B0
:10CF700071F18A859B853BEA8D3C930721F03FEF59
:10CF80008F3F930779F5223041F088E090E007C0A9
:10CF9000019722912F3F41F00BC082E090E0FE010B
:10CFA000E80FF91F3C96F4CF181619068CF30FC042
:10CFB00089E1BE01645F7F4F0E94215089E10E9498
:10CFC0002B5068EE77E20E94E945009759F088E11E
:10CFD000BE016A5E7F4F0E942150E0919703F0915D
:10CFE00098030995E0960FB6F894DEBF0FBECDBF4B
:10CFF000CF91DF911F910F910895AF92BF92CF9281
:10D00000DF92EF92FF920F931F93DF93CF93CDB7F1
:10D01000DEB7E0970FB6F894DEBF0FBECDBF6C0150
:10D020008B01FE01319680E3DF011D928A95E9F7BD
:10D0300081E089838CE00E9418508C831D821F82BE
:10D040008091E41389878F5F8093E41383E0E82E57
:10D05000E8868DEC9BEA9B878A8789E10E942B50AA
:10D0600061E772E00E94E945009731F082E08E832B
:10D070008FEF8C878D8709C089E10E942B50BC01FE
:10D08000CE010C960E94E045EE828DEC9BEA9D8BD2
:10D090008C8BCE01469668EE77E20E94E0450E94B6
:10D0A000E44E9FA78EA70E94364F88AB7E0108945E
:10D0B000E11CF11CC7010E94BD6EA82E90E00E94E9
:10D0C0004C4F009741F10E94EC4EBC01C7014A2D24
:10D0D0000E94DB6EA0902F03B09030030E94EC4EB4
:10D0E0007C010E94404FBC01C701F5010995C114A4
:10D0F000D10489F0009721F08130910561F404C0DA
:10D10000C80160E070E003C0C80164E070E041E085
:10D1100050E0F6010995E0960FB6F894DEBF0FBE19
:10D12000CDBFCF91DF911F910F91FF90EF90DF90D6
:10D13000CF90BF90AF9008950E94FD698093E41353
:10D14000E0913903F0913A0309950895EF92FF9227
:10D15000CF93DF93E82EE7017E01F92EE70104C0AB
:10D1600060E070E00E944E48899199910097C1F764
:10D17000DF91CF91FF90EF900895EF92FF92CF93C0
:10D18000DF93E82EE7017E01F92EE70102C00E943D
:10D190009347899199910097D1F7DF91CF91FF90B3
:10D1A000EF900895CF93DF93EC017B836A830E9415
:10D1B0008F5999838883DF91CF910895FC018081F5
:10D1C000918122813381820F931F918380830895FF
:10D1D000CF93DF93EC010E948F5999838883DF916D
:10D1E000CF910895CF93DF93EC010E948F5928814E
:10D1F0003981821B930B019621E030E04A815B81EB
:10D200004817590710F020E030E0C901DF91CF91B5
:10D210000895EF92FF92CF93DF93FC01C281D381F7
:10D2200080819181C80FD91F0E948F59C81BD90BCB
:10D23000CE01DF91CF91FF90EF900895CF93DF93D0
:10D24000E1E6FAE2C3E2DAE2A5E5BAE2119211926E
:10D2500019921992199219921D928AE2E937F807E8
:10D26000A9F7DF91CF9108950F931F93CF93DF9389
:10D27000FC01DC01AB5AB54D8C91882339F100914A
:10D28000940010919500EF01CC0FDD1FCC0FDD1F36
:10D29000CD5DD54DDF01AA0FBB1FAF59B54D8D91A7
:10D2A0009C9111979801281B390B40E050E0688150
:10D2B00079818A819B81260F371F481F591F288338
:10D2C00039834A835B8311961C930E93EE0FFF1FE5
:10D2D000EE0FFF1FED5DF54D6081718182819381BD
:10D2E000DF91CF911F910F91089560E070E0CB0125
:10D2F0000895FC01EE0FFF1FEE0FFF1FED5DF54DD2
:10D3000040835183628373830895EF92FF920F935A
:10D310001F93CF93DF9325E53AE2C3E2DAE2E1E639
:10D32000FAE2D9018D919D018823C9F040919400C2
:10D3300050919500808191817A01E81AF90A00E004
:10D3400010E088819981AA81BB818E0D9F1DA01F4D
:10D35000B11F88839983AA83BB835183408324961A
:10D360003296BAE221363B07E1F6DF91CF911F9169
:10D370000F91FF90EF9008950E943A6E08950F93D9
:10D380001F93FC01CB014091E5135091E6133383C9
:10D3900022831583048371836083F093E613E09303
:10D3A000E5134115510511F40E94546E80E090E0A0
:10D3B0001F910F9108958091E5139091E6130097C6
:10D3C000C1F01092E6131092E513DC0114966D91F2
:10D3D0007C9115971296ED91FC9113970995E09128
:10D3E000E513F091E613309721F0808191810E943E
:10D3F000546E08950E94D48408950E94D0840895A4
:10D4000088EB93E00E94874880EC93E00E94874875
:10D410000895EF92FF92CF93DF930E94F34E00970F
:10D42000C9F080EC93E00E94A748E82EE7017E0156
:10D43000F92EE701209731F10E94364F99838883B6
:10D440000E94314F9B838A83C70104960E945F4EDE
:10D450008CAB18C088EB93E00E94A748EC017E01DA
:10D46000F92EE701209771F0C70102960E94764ECF
:10D4700099838883B7016E547F4FC7018E579F4FA2
:10D480000E94E34FCE01DF91CF91FF90EF9008957E
:10D49000BC016E547F4F8E579F4F0E94E34F0895FB
:10D4A000CF93DF93EC0188EB93E0BE010E94F2483A
:10D4B000009719F088EB93E009C080EC93E0BE017F
:10D4C0000E94F248009729F080EC93E0BE010E9490
:10D4D000CD48DF91CF910895EF92FF92CF93DF93E4
:10D4E000EC0188EB93E0BE010E94F248009779F0CE
:10D4F00068817981CE0102960E94B04FBE016E54C0
:10D500007F4FCE018E579F4F0E94F84F1BC080EC7B
:10D5100093E0BE010E94F2480097A1F00E94874F5D
:10D52000688179818A819B810E94B04F8CA990E0AB
:10D530000E944C4F0E94EC4E4CA92496BE0150E034
:10D540000E944188DF91CF91FF90EF900895EF9274
:10D55000FF92CF93DF93EC0188EB93E0BE010E9432
:10D56000F248009711F022960DC080EC93E0BE01C6
:10D570000E94F248009721F00A80DB81C02D02C092
:10D58000C0E0D0E0CE01DF91CF91FF90EF90089501
:10D59000FC0180819181089570E06F5B7F4F660F81
:10D5A000771F680F791FCB010895E62FF0E0EF5B3E
:10D5B000FF4FEE0FFF1FE80FF91F80819181089543
:10D5C00008958DE39AE10E94FD4A009721F08DE3D2
:10D5D0009AE10E94E84A0895E0914A1AF0914B1AA4
:10D5E000309711F00995089580E00895EF92FF9229
:10D5F0000F931F93CF93DF93EC018A018881998168
:10D60000009731F023E08C30920709F006C12BC05F
:10D6100080E00BC0E82FF0E0EE0FFF1FEE0FFF1FC2
:10D62000E55DF54E118210828F5F843098F3809310
:10D63000451A80916C1190916D1190933C1A8093D2
:10D640003B1A0E948C478093792A8DE39AE160E42B
:10D6500070E00E94D24A0E9455718CE093E0998359
:10D66000888381E0DDC0623009F4B9C0633030F4F2
:10D67000662309F489C0613081F79CC0673819F0CE
:10D68000683859F741C01092461A4BE2E42E4AE13D
:10D69000F42E18C0F701828193818017910749F415
:10D6A000808191810E949C72F70111821082138205
:10D6B000128284E090E0E80EF91E8091461A8F5F96
:10D6C0008093461A8091461A843020F3E9E8FFE2FD
:10D6D000848D958D8017910719F4158E148E118EF7
:10D6E000B09690E3E930F90799F7EFE1F0E381852F
:10D6F00092858017910711F4158214823D9620E3DC
:10D70000E13AF207A1F7A9CF8AE14D33580709F0B2
:10D71000A4CFCA010E94FD4A009709F49ECF10923F
:10D72000461A2DC0F0E035E0EE0FFF1F3A95E1F705
:10D73000E757F04D818D8823E9F08DE39AE10E944F
:10D74000E84A8091461A90E025E0880F991F2A95B3
:10D75000E1F78757904D9093882F8093872F82E031
:10D760000E94D07280917A2A90917B2A009711F0C2
:10D770000E94EC6A8091461A8F5F8093461AE0916E
:10D78000461AE43078F269CF4115510509F465CFA6
:10D790005093882F4093872F83E00E94D07280910E
:10D7A0007A2A90917B2A009711F00E94EC6A0E94DD
:10D7B000E16A53CF4115510509F44FCF5093842F9F
:10D7C0004093832F85E00E94D07280917A2A9091B5
:10D7D0007B2A009709F441CF0E94EC6A3ECF8091EA
:10D7E0007A2A90917B2A009709F437CF80918B2A6F
:10D7F000863031F48091A32A81FF02C00E94E16A41
:10D8000081E00E94D07280917A2A90917B2A0097C1
:10D8100009F423CF0E941F6D20CF1982188283E064
:10D82000DF91CF911F910F91FF90EF90089590930A
:10D830004B1A80934A1A089520916C1130916D1102
:10D8400060E0EBE2FAE113C04081518148175907CB
:10D8500061F4428153814217530739F46093491AA6
:10D86000118210820E949C72089534966F5F64301A
:10D8700058F36093491A089540E0EBE2FAE116C0CC
:10D88000542F5F5F208131812115310569F4409368
:10D89000481A9183808320916C1130916D113383EC
:10D8A00022830E94B67208953496452F443040F387
:10D8B0004093481A0895FC0180916C1190916D116C
:10D8C000958F848F778F668F0895FC0180916C11FE
:10D8D00090916D1192878187748763870895CF93A4
:10D8E000DF93EA010E941872FC01009741F08091D9
:10D8F0006C1190916D1192878187D487C387CF0176
:10D90000DF91CF9108950F931F93DF93CF9300D0B2
:10D9100000D0CDB7DEB78C01AB018FEF89838A834E
:10D920008B838C83CE010196B8010E946F6CFC0141
:10D93000009711F015830483CF010F900F900F9083
:10D940000F90CF91DF911F910F91089585ED93E096
:10D9500062E040E050E00E943F4810927B2A109223
:10D960007A2A0895AC0185ED93E061E00E941C489D
:10D970000895AC0185ED93E060E00E941C48089595
:10D980000F931F93CF93DF93EA010E948E718C0156
:10D99000009761F080916C1190916D11F801958F55
:10D9A000848FD78FC68FC8010E94B96CC801DF91E0
:10D9B000CF911F910F910895CF93DF93A091872F5F
:10D9C000B091882F109719F0ED016C9605C0C091A9
:10D9D000832FD091842F29968091822F86FF22C099
:10D9E0001092471A40E0EBE2FAE116C02081318143
:10D9F00014968D919C9115972817390759F48281B7
:10DA00009381009739F04093471A998388831B824A
:10DA10001A8206C034964F5F443040F34093471A51
:10DA20000E94E16A88819981009731F04A815B8187
:10DA30006091792A0E943F48DF91CF9108950F931A
:10DA40001F93CF93DF9380918B2A863009F074C0A7
:10DA500080917A2A90917B2A25E08030920709F004
:10DA60006BC0C4E9D2E0D0937B2AC0937A2A02E04B
:10DA70000093842A14E91093852A1092A72A109201
:10DA8000A62A0E944D71809590959093A72A809325
:10DA9000A62A10928D2A10928C2A0E943C718095A1
:10DAA000909590938D2A80938C2A0E94EC6AD09353
:10DAB0007B2AC0937A2A0093842A1093852A909116
:10DAC000852F8091862FE92FF82FDF01A459BD4FB4
:10DAD0008CE692E00D9001920197E1F78AE99AE2D3
:10DAE0006CE672E00E94E07080917E2A80939A2A10
:10DAF00080917F2A80939B2A8091802A80939C2A00
:10DB00008091812A80939D2A1092A72A1092A62A9A
:10DB10000E944D71809590959093A72A8093A62A94
:10DB200010928D2A10928C2A0E943C7180959095BB
:10DB300090938D2A80938C2A0E94EC6ADF91CF917A
:10DB40001F910F910895282F392FF90120E030E01F
:10DB500080E0A8E112C0419198E0542F5827B52FDA
:10DB6000B17050FD8A278695B13009F480689150D4
:10DB700011F04695F2CF2F5F3F4F2617370759F721
:10DB800008951F920F920FB60F920BB60F921124A9
:10DB90002F933F934F935F936F937F938F939F93B5
:10DBA000AF93BF93EF93FF93809194009091950072
:10DBB0009093662A8093652A81E08093572A80910A
:10DBC0007100807D809371000E94DB698091572AEB
:10DBD0008823E9F180919400909195002091652A25
:10DBE0003091662A82179307A0F480912B2A909196
:10DBF0002C2AA0912D2AB0912E2A8C57914EAF4FEE
:10DC0000BF4F80932B2A90932C2AA0932D2AB09358
:10DC10002E2A8091940090919500821B930BA0E096
:10DC2000B0E020912B2A30912C2A40912D2A50913E
:10DC30002E2A820F931FA41FB51F80932B2A909327
:10DC40002C2AA0932D2AB0932E2A1092572AFF91A6
:10DC5000EF91BF91AF919F918F917F916F915F9164
:10DC60004F913F912F910F900BBE0F900FBE0F90D1
:10DC70001F9018959FB7F894E1E7F0E08081807DD0
:10DC8000808388B38F6288BB10929000E1E9F0E056
:10DC90001082109292001092950010929400808150
:10DCA000856080839FBF08952FB7F8949093990063
:10DCB0008093980088B38F6288BBE1E7F0E08081B1
:10DCC000826080832FBF0895EF92FF92CF93DF93FE
:10DCD000FC01DB0185E0EB0119928A95E9F785816A
:10DCE00090E083709070009711F082E08C938781B0
:10DCF00090E083709070009721F082E012968C93F0
:10DD00001297858190E083709070009799F08781D9
:10DD100090E083709070009769F023893489818541
:10DD200092852817390731F481E0848312961C927A
:10DD3000129701C01482858183708250823030F442
:10DD4000C82FD0E0C152DC4F888101C080E011961D
:10DD50008C931197E781E370E250E23028F4F0E011
:10DD6000E152FC4F808101C080E013968C931397A1
:10DD7000DF91CF91FF90EF900895DF93CF9300D084
:10DD800000D00F92CDB7DEB7BE016F5F7F4F0E940C
:10DD9000646E89819A81890F8D5F9B81890F9C8137
:10DDA000890F9D81890F0F900F900F900F900F900A
:10DDB000CF91DF910895AF92BF92CF92DF92EF9211
:10DDC000FF920F931F93DF93CF9300D000D000D02A
:10DDD000CDB7DEB78C017B01BE016F5F7F4F4E83F5
:10DDE0000E94646EC9809A81A92EBB24DB808C813D
:10DDF000682F70E095012C0D311D2D5F3F4F2D0DCB
:10DE0000311D260F371F5D81250F311D4E8150E0DA
:10DE1000421753070CF4A8C0D80111964C911197E2
:10DE200050E041705070E3E0440F551FEA95E1F770
:10DE300012962C91129730E02170307054E0220F2E
:10DE4000331F5A95E1F7242B3C913770232B1396FF
:10DE50003C911397E32FF0E0E170F07045E0EE0F96
:10DE6000FF1F4A95E1F72E2B14963C911497E32F50
:10DE7000F0E0E170F07036E0EE0FFF1F3A95E1F749
:10DE80002E2BF701208315964C91159750E0437087
:10DE90005070440F551F440F551F16962C9116971E
:10DEA00030E02370307054E0220F331F5A95E1F7B1
:10DEB000242B17963C9117973295330F330F307CF4
:10DEC000322B318318962C9118972283FC2DF23037
:10DED00069F419962C91D70113962C931397F80196
:10DEE000228514962C93149745E001C043E0E92F56
:10DEF000F0E03B96E00FF11F542F0AC09701250F69
:10DF0000311DC290D901CC925F5F0894A108B1087D
:10DF1000A114B10499F7940FBD2DB23089F4F70123
:10DF2000E90FF11DD80153962C91539720839F5FE1
:10DF3000F701E90FF11D54962C91549720839F5FB0
:10DF4000E82FF0E07596E00FF11F292F08C0D701E8
:10DF5000A20FB11D32913C932F5F6150704061154B
:10DF60007105A9F7890F01C080E026960FB6F894D5
:10DF7000DEBF0FBECDBFCF91DF911F910F91FF90FC
:10DF8000EF90DF90CF90BF90AF900895BF92CF9267
:10DF9000DF92EF92FF920F931F93CF93DF937C0159
:10DFA000D62EEA01633008F4ADC0FC018081B82EA2
:10DFB000B294B694B694B3E0BB22F1E0BF22F7016D
:10DFC0009181292F269526952370C92EC294C69437
:10DFD000C694A3E0CA22382F37703883382F36957D
:10DFE0003695369531703983382F329531703A83B2
:10DFF0008295869581708B83BC822D83892F829533
:10E0000083708E83CF828281888787010D5F1F4F47
:10E01000222361F1F801918180E0F7013381830FC0
:10E02000911D9A87898787010B5F1F4F223081F4EA
:10E03000CA010B9661E772E00E94E045F801818118
:10E040008B87F70185818C878701095F1F4F16C079
:10E050002330A1F4F7013D96DA011B9682918D934E
:10E06000E017F107D9F7085F1F4F08C0CA010B96E8
:10E0700061E772E00E94E0451A861986CC2089F19A
:10E08000BB2059F4F801918180E02081820F911D1D
:10E090009C8B8B8B0E5F1F4F04C089859A859C8B50
:10E0A0008B8BFC2DF23071F4CE01459661E772E066
:10E0B0000E94E045F80181818D8B80818E8B0E5FFF
:10E0C0001F4F17C0FC2DF330A1F4085F1F4FD8017C
:10E0D000FE01759680E09E9191938F5F8830D9F70D
:10E0E00008C0CE01459661E772E00E94E0451C8AB7
:10E0F0001B8A802F8E199D2D981B9FA71EA70DA7E9
:10E10000D81608F480E0DF91CF911F910F91FF9016
:10E11000EF90DF90CF90BF9008959C014150504008
:10E12000460F571FDB0110C0FC91E0E011968C9167
:10E130001197BF01680F711D260F371F261737076C
:10E1400010F42F5F3F4F1296A417B50768F3A4177A
:10E15000B50749F49C9180E0280F391F281739072B
:10E1600010F42F5F3F4FC9010895CF93DF93909133
:10E17000852AC92FD0E064973091842A20E0C20F0D
:10E18000D31F9E01280F311DC9016EE87AE248E0D5
:10E1900050E00E948D7066E97AE2AE010E948D70B7
:10E1A000009719F0382F292F02C02FEF3FEFC90138
:10E1B000DF91CF91089590935B1A80935A1A089536
:10E1C000FC014381460F4093812A872F99272281A2
:10E1D000280F2093802AA181A0937F2A50815093F9
:10E1E0007E2A30E02817390748F48A2F8F5F809302
:10E1F0007F2A882319F45F5F50937E2A842F90E052
:10E2000070708617970798F48091802A8F5F8093AB
:10E21000802A882361F480917F2A8F5F80937F2AF0
:10E22000882329F480917E2A8F5F80937E2A089527
:10E23000BC018091872F9091882F08960E94E070F2
:10E24000E091872FF091882F80917E2A808780919E
:10E250007F2A81878091802A82878091812A838783
:10E2600008959C01AB0180E090E0B9010E948D709F
:10E27000382F292FC901089580E090E062E87AE202
:10E2800044E150E00E948D70009719F0382F292F3B
:10E2900002C02FEF3FEFC901089586E00E94B570DC
:10E2A000089581E10E94B570089580E009C0E82FCB
:10E2B000F0E0EE0FFF1FE75FFF4C118210828F5FCF
:10E2C0008430A8F380E00BC0E82FF0E095E0EE0F7B
:10E2D000FF1F9A95E1F7E757F04D118E8F5F84305D
:10E2E00098F380E094E090935D1A80935C1A40E08C
:10E2F0008DE090E00EC0242F30E0289FF001299F90
:10E30000F00D389FF00D1124E15EFF4C1582148250
:10E310004F5F4A3080F34093581A089520915C1A59
:10E3200030915D1A2F5F3F4F4DE72030340710F0DA
:10E3300020E030E1522F432FA0E013C0EA2FF0E09D
:10E34000B5E0EE0FFF1FBA95E1F7E757F04DB18D3D
:10E35000BB2331F00480F581E02DE417F50711F3BC
:10E36000AF5FA43059F730935D1A20935C1A109276
:10E37000581A20E0E0E0F0E01EC0A22FB0E035E047
:10E38000AA0FBB1F3A95E1F7A757B04D59963C919C
:10E390005997332321F42093581AFD0110C03730C8
:10E3A00049F4309731F05A964C915A97328D341780
:10E3B00008F4FD012F5F243000F32093581A3097A2
:10E3C000A9F122E0218F2091521A24872091531A1B
:10E3D00025872091541A26872091551A278728EDE2
:10E3E00034E0338B228B358B248B21E030E0318B72
:10E3F000208B138E21E0228F23E0208F168A20E1CC
:10E40000278B20915C1A30915D1A322723273227FF
:10E410003583248377836683DC012D913D914D9173
:10E420005C9113972083318342835383CF010895F6
:10E430000F931F93CF93DF9320915C1A30915D1A55
:10E440004DE050E02F5F3F4FADE720303A0710F02E
:10E4500020E030E1B22FA32F10E012C0C12FD0E096
:10E46000C49FF001C59FF00DD49FF00D1124E15E13
:10E47000FF4C0480F581E02DEA17FB0719F31F5FBD
:10E480001A3061F730935D1A20935C1A10E02DE08A
:10E4900030E01AC0012F0F5FC12FD0E0C29FF00102
:10E4A000C39FF00DD29FF00D1124E15EFF4CDF0100
:10E4B0001496448155814115510529F41093581A39
:10E4C000309749F433C0102F1A3020F31093581AA4
:10E4D000E0E0F0E02BC020915C1A30915D1A322709
:10E4E0002327322711963C932E93778366830097D8
:10E4F00029F4108211821282138209C0DC012D914D
:10E500003D914D915C9120833183428353838DE013
:10E5100090E0C89FD001C99FB00DD89FB00D1124C5
:10E52000A15EBF4C80E418968C931897CF01DF91C1
:10E53000CF911F910F91089540E013C0E42FF0E0B8
:10E54000542F5F5FEE0FFF1FE75FFF4C208131818B
:10E550002817390729F44093581A11821082089518
:10E56000452F443058F34093581A089540E013C0A3
:10E57000E42FF0E0542F5F5FEE0FFF1FE75FFF4CCB
:10E58000208131812115310529F44093581A918356
:10E5900080830895452F443058F34093581A0895C6
:10E5A000EF92FF920F931F93CF93DF93C091872F2A
:10E5B000D091882F843009F4F7C10AEA1AE2109347
:10E5C000862F0093852F10937D2A00937C2A833019
:10E5D00071F4898D90E08F7090708330910509F00F
:10E5E00074C088899989009709F02FC78DC082303F
:10E5F00009F08EC08091551A8F5F8093551A882339
:10E6000099F48091541A8F5F8093541A882361F48F
:10E610008091531A8F5F8093531A882329F4809135
:10E62000521A8F5F8093521A10927B2A10927A2A84
:10E6300010921E3010921D30898D873011F0853078
:10E6400041F48A8D8F5F8A8F843109F0FEC6198E5E
:10E65000FCC6882309F4F9C62889398921153105B2
:10E6600009F44EC09A8D292F21502A8F992309F041
:10E67000ECC69B8D983031F0282F2150223048F481
:10E68000953039F4198E80E88093822F0E94DC6CDB
:10E6900095C5953048F423E030E0092E02C0220FE2
:10E6A000331F0A94E2F701C020E32A8F9F5F9B8FFC
:10E6B00090E08F70907083309105E1F08430910587
:10E6C0004CF48130910509F461C38230910509F061
:10E6D000BCC60DC08630910509F40CC58830910583
:10E6E00009F408C58430910509F0AFC603C510923E
:10E6F000A32A4FC384E08093822F0E94DC6C90C5D4
:10E700008F70833009F0A1C688E08093822F4BC5BB
:10E71000853019F5E091832FF091842F84819581C4
:10E72000009709F492C61092882F1092872F0C50F0
:10E7300010401093862F0093852F10937D2A00930D
:10E740007C2A10921E3010921D3010927B2A10925B
:10E750007A2A88E08093822F25C108521040809148
:10E76000822A853409F071C69091842A80E0209134
:10E77000852A7C01E20EF11C80917A2A90917B2AF5
:10E780008E159F0508F461C6F0927B2AE0927A2AE2
:10E790008091882A90E08F739070009709F055C699
:10E7A0008091892A882309F050C680911930909170
:10E7B0001A30C091E503D091E6038C179D0759F4F8
:10E7C00040911B3050911C302091E7033091E803B9
:10E7D00042175307A1F02091922A3091932A2817CB
:10E7E000390709F032C62091942A3091952A8091F8
:10E7F0001B3090911C302817390709F026C60E945B
:10E800003C712FEF8F3F920709F01FC680918B2A32
:10E81000863009F431C18131E9F1813009F015C642
:10E820008091962A883009F010C61092962A80911D
:10E83000982A9091992A4FEF873F940710F00996F4
:10E8400001C008969093992A8093982A80918E2AE5
:10E8500090918F2AA091902AB091912A8093922A28
:10E860009093932AA093942AB093952A809119307B
:10E8700090911A30A0911B30B0911C3080938E2A59
:10E8800090938F2AA093902AB093912A80E4F80164
:10E890008087B8C5C7014C9790937B2A80937A2ACA
:10E8A0008EE99AE29093862F8093852F80919C2AFF
:10E8B00090919D2A009739F00E945171FFEF8F3F90
:10E8C0009F0709F0C2C52091982A3091992A2115F5
:10E8D000310509F4BAC58FE190E39093842F8093BA
:10E8E000832F6091E7037091E8034091E103509119
:10E8F000E2030091E3031091E40339C08481958120
:10E90000009781F12817390769F58681978100976B
:10E9100039F0A091962AB091972AA817B90711F556
:10E92000808191818C179D0729F4A281B381A6175C
:10E93000B70739F18417950729F4A281B381A0178D
:10E94000B107F9F0A0918E2AB0918F2AA817B907C4
:10E9500049F4A091902AB091912A82819381A817BD
:10E96000B90779F03D96F093842FE093832FE091DF
:10E97000832FF091842F80E3E13AF80708F4BECFAB
:10E9800064C51092882F1092872F82E08093822F87
:10E990008EE99AE290937D2A80937C2A10921E3011
:10E9A00010921D300E94DC6C80911D3090911E30C1
:10E9B000009709F44AC59C01245E3F4F30937B2A9F
:10E9C00020937A2A3093842A2093852AE091832FFA
:10E9D000F091842F208520938A2A21E120938B2A8D
:10E9E000089698278927982790939B2A80939A2A9C
:10E9F00010929D2A10929C2A848195819093972A47
:10EA00008093962A868197819093992A8093982A59
:10EA10008091193090911A30A0911B30B0911C3028
:10EA200080938E2A90938F2AA093902AB093912A54
:10EA300080819181A281B3818093922A9093932ABD
:10EA4000A093942AB093952A8AEA9AE29093862F0B
:10EA50008093852F0E9451718095909590939D2A67
:10EA600080939C2A009709F0CDC48FEF9FEF90937D
:10EA70009D2A80939C2AC6C40E944D71EFEF8F3F60
:10EA80009E0709F0E2C48091982A9091992A0097F4
:10EA900009F4DBC42091962A3091972A211531057B
:10EAA00009F4D3C4C9E8DFE2498D4423E9F06C815D
:10EAB0007D8186179707C1F46E817F8126173707FE
:10EAC00099F4E0918E2AF0918F2A68817981E61776
:10EAD000F70751F4E091902AF091912A6A817B81A5
:10EAE000E617F70709F46DC1A096F0E3C930DF0718
:10EAF000D9F62091A32A2F732230B9F49093571A94
:10EB00008093561A40E00DC0E42FF0E0EE0FFF1F97
:10EB1000E75FFF4C208131814F5F8217930709F433
:10EB20006EC0443088F34093581A8091A32A82FD26
:10EB30008CC484E1F80181A388E290E090937B2A61
:10EB400080937A2A80E580A380919D2A9091A12AC2
:10EB5000938F30919C2A9091A02A928F368F20918A
:10EB60009B2A90919F2A918F258F90919A2A90931A
:10EB7000581A40919E2A408F948F8F5F878F8823E9
:10EB800061F4832F8F5F868F882339F4822F8F5F04
:10EB9000858F882311F49F5F948F8091962A90919E
:10EBA000972A9093571A8093561A2091982A309159
:10EBB000992AF801358B248B978B868B80918E2A2E
:10EBC00090918F2AA091902AB091912A8093922AB5
:10EBD0009093932AA093942AB093952A8091193008
:10EBE00090911A30A0911B30B0911C3080938E2AE6
:10EBF00090938F2AA093902AB093912AE8C3109201
:10EC0000581A80E0C0E0D0E022C0E82FF0E075E0C4
:10EC1000EE0FFF1F7A95E1F7E757F04D918D99239D
:10EC200021F48093581AEF0116C0973079F4209799
:10EC300021F0228D9A8D921748F4C82FD0E065E01C
:10EC4000CC0FDD1F6A95E1F7C757D04D8F5F843039
:10EC5000E0F28093581A209709F4F7C3D093882FD5
:10EC6000C093872F83E08A8F888F1E8A84E08F8BE2
:10EC70001B8E8091982A9091992A9D838C838091F4
:10EC8000962A9091972A9F838E8380918E2A9091C5
:10EC90008F2AA091902AB091912A88839983AA8380
:10ECA000BB8381E0898F8091521A8C878091531A9F
:10ECB0008D878091541A8E878091551A8F8781E0B5
:10ECC00090E0998B888B80919D2A8B8780919C2ADC
:10ECD0008A8780919B2A898780919A2A888781E0F8
:10ECE00090E00E9418718091A22A282F30E0207FA6
:10ECF0003070213531050CF449C082958F7090E059
:10ED00000597880F991F880F991F5091591A40E055
:10ED100034C0F901EE57F54D50A5552329F4409321
:10ED2000581A1092591A32C0513011F44F5F25C051
:10ED30005230E1F461A56430C9F44093581A5093FD
:10ED4000591A32A520E083A590E0822B932B909353
:10ED5000571A8093561AF4E0893D9F0710F088ED0A
:10ED600094E09B8B8A8B9D8B8C8B10C02E57354DDE
:10ED7000F90121A5222331F0420F242F30E028177A
:10ED800039073CF24093581A5093591A80E1809306
:10ED9000A32A8091A32A82608093A32A82E0809391
:10EDA000AA2A84E08093AB2A8093AC2A88ED8093D2
:10EDB000AD2A8CE290E090937B2A80937A2A80E6B9
:10EDC000B3C2D093882FC093872F1092822F809147
:10EDD000A32A90E082FF03C0198E80E24EC22091E8
:10EDE000A22A22952F70220F220F2093581AB701C2
:10EDF000621B71099B012451304030937B2A209380
:10EE00007A2A50E04F7050704230510539F4AC010D
:10EE10004F7350704231510551F42AC041305105B1
:10EE200031F4AC014F7350704230510509F1211596
:10EE3000310531F49C012370307021153105C1F08A
:10EE400030919A2A2885321709F064C230919B2AA2
:10EE50002985321709F05EC230919C2A2A85321723
:10EE600009F058C230919D2A2B85321709F052C201
:10EE700084FF4AC0688979896115710509F444C025
:10EE8000CE010C960E94E07030919E2A80917E2ADD
:10EE90003817D1F520919F2A80917F2A2817A1F554
:10EEA0009091A02A8091802A981771F58091A12ACB
:10EEB0004091812A841741F53C872D879E878F8753
:10EEC0008B8D8823D1F42E89888D9A8D891B922F62
:10EED000969596959695891B280F2E8B87FD819583
:10EEE0009F89392F36953695931B980F9F8B822FCC
:10EEF000869586958695890F888F81E08093822FED
:10EF0000888D8A8F198A188A298D30E0C9018F70FF
:10EF100090708430910509F4B5C18530910564F491
:10EF200082309105C9F1833091050CF0B9C0813070
:10EF3000910509F08AC211C08630910509F4E2C139
:10EF4000863091050CF4BEC18730910509F4E2C109
:10EF50008830910509F079C28AC18091822F80FFA3
:10EF600014C083E0898F80E48093822F198A188AE5
:10EF700080917A2A90917B2A009709F410C122E4AB
:10EF80002093822F0E9418710AC18091A32A8F7347
:10EF9000823009F05AC2FACE8091822F80FF75C06C
:10EFA0008091A32A8F73823109F06FC08091A22AC9
:10EFB000282F30E0207F3070213531050CF449C016
:10EFC00082958F7090E00597880F991F880F991F81
:10EFD0005091591A40E034C0F901EE57F54D50A553
:10EFE000552329F44093581A1092591A32C05130BF
:10EFF00011F44F5F25C05230E1F461A56430C9F4CB
:10F000004093581A5093591A32A520E083A590E0F6
:10F01000822B932B9093571A8093561A74E0893D54
:10F02000970710F088ED94E09B8B8A8B9D8B8C8BDF
:10F0300010C02E57354DF90121A5222331F0420F82
:10F04000242F30E0281739073CF24093581A509388
:10F05000591A83E0898F80919A2A888780919B2A08
:10F06000898780919C2A8A8780919D2A8B8781E05D
:10F0700090E00E94187182E48093822F198A188A86
:10F0800010927B2A10927A2A8AC080E28093822F83
:10F090000E94DC6CE091872FF091882F118E45CD76
:10F0A0008091A32A80FF2AC024FD28C088899989DD
:10F0B000009709F0CAC180917A2A90917B2A019623
:10F0C0000E9418712091822F822F80618093822F5D
:10F0D00080917A2A90917B2A009719F022612093DF
:10F0E000822F0E94DC6C81E090E0998B888B88E015
:10F0F000898F1B8E81E18093A32A0FC185FF1CC0DD
:10F100005091A82A40E08091A92A90E0842B952B69
:10F110004091852F5091862F480F591F5093862F6D
:10F120004093852F40917A2A50917B2A481B590B96
:10F1300050937B2A40937A2A80917A2A90917B2A55
:10F14000009749F024FD07C02091822F2260209370
:10F15000822F0E9418719091A42A80E02091A52A04
:10F16000820F911D9093571A8093561A2C893D89CE
:10F170002817390710F0009721F43093571A20937D
:10F18000561A8091561A9091571A9B8B8A8B8091B0
:10F19000822F90E083709070009709F456C110920E
:10F1A0001E3010921D300E94DC6C8091822F85FFF2
:10F1B00007C010921E3010921D30198E84E19BCF33
:10F1C00084FF0AC010921E3010921D3081E090E042
:10F1D000998B888B84E08CCF20911D3030911E302C
:10F1E00021153105E1F080FF02C0198A188A88894B
:10F1F0009989009781F48A899B898217930720F463
:10F2000090931E3080931D3080911D3090911E3060
:10F21000998B888B04C090931E3080931D301B8E79
:10F2200080917C2A90917D2A9093862F8093852FC0
:10F2300080911D3090911E30009759F088899989EE
:10F24000009739F0889690937B2A80937A2A88E1F8
:10F250000BC08091822F81FFF8C088E290E09093EC
:10F260007B2A80937A2A80E18093A32A5CC08091D4
:10F27000822F80FFEAC0198E80E18093822F0E9446
:10F28000DC6CE3C080917A2A90917B2A009711F080
:10F290000E9418719091A32A8091822F90FF0BC039
:10F2A00080FF06C087E0898F1A8E198A188A19C0D4
:10F2B00086E0898F16C080FF1EC085E0898F198A7D
:10F2C000188AC3C080917A2A90917B2A009711F006
:10F2D0000E9418718091A32A80FF0DC087E0898F5A
:10F2E0001A8E81E090E00E94187180E18093822F55
:10F2F0000E94DC6C0FC080917A2A90917B2A009743
:10F3000049F4A3C08091822F80FF9FC087E0898F3E
:10F310001A8E9BC080E1F80181A388E290E090936F
:10F320007B2A80937A2A80E58093A22A888580931D
:10F330009E2A898580939F2A8A858093A02A8B851F
:10F340008093A12A8C8580939A2A8D8580939B2A0D
:10F350008E8580939C2A8F8580939D2A86E080935A
:10F360008B2A8C819D819093972A8093962A8E81F7
:10F370009F819093992A8093982A80911930909137
:10F380001A30A0911B30B0911C3080938E2A90933C
:10F390008F2AA093902AB093912A88819981AA817B
:10F3A000BB818093922A9093932AA093942AB0933E
:10F3B000952A898D84FF05C01092A52A1092A42A4F
:10F3C00006C084E08093A42A88ED8093A52A80E477
:10F3D00080938A2A80917A2A90917B2A9093842A1A
:10F3E0008093852A1092A92A1092A82A1092A72AFF
:10F3F0001092A62A0E944D71809590959093A72A0D
:10F400008093A62A85E48093822A1092832A109200
:10F41000892A1092882A80915A1A90915B1A019633
:10F4200090935B1A80935A1A9093862A8093872A26
:10F4300010928D2A10928C2A0E943C718095909592
:10F4400090938D2A80938C2A04C010927B2A10926C
:10F450007A2A1092822FDF91CF911F910F91FF9006
:10F46000EF900895382F292FC9010895382F292F9B
:10F4700040E050E076276727762780E090E0CB01D8
:10F4800077276627262B372B482B592BB901CA0122
:10F490000895AC01E0917C2AF0917D2A2227332740
:10F4A0002E1B3F0B2E57304D621773070CF49B0138
:10F4B0001216130664F420931D3030931E304E173D
:10F4C0005F0729F0CF01BA01A9010E944188089580
:10F4D0002F923F924F925F926F927F928F929F9264
:10F4E000AF92BF92CF92DF92EF92FF920F931F9352
:10F4F000CF93DF93CDB7DEB763970FB6F894DEBF37
:10F500000FBECDBF7C011B016A01FC011782168270
:10F51000838181FF66C3BE016F5F7F4F4B01F7019F
:10F520009381F10193FD859193FF81911F018823C0
:10F5300009F453C3853239F493FD859193FF81918A
:10F540001F01853239F4B70190E00E94AA88560164
:10F550006501E5CF10E0512C20E02032A0F48B3281
:10F5600069F030F4803259F0833269F420612CC0A4
:10F570008D3239F0803339F4216026C02260246056
:10F5800023C0286021C027FD27C030ED380F3A3056
:10F5900078F426FF06C0FAE01F9F300D1124132FC8
:10F5A00013C06AE0569E300D1124532E20620CC009
:10F5B0008E3221F426FD11C3206406C08C3611F46E
:10F5C000206802C0883641F4F10193FD859193FFD4
:10F5D00081911F018111C1CF9BEB980F933018F4DB
:10F5E0002061805E06C09BE9980F933008F0AAC1A5
:10F5F0002F7E26FF16E02F73722E853621F4F22F10
:10F60000F0647F2E08C0863621F4622F6068762E63
:10F6100002C01111115077FE07C01C3348F4442476
:10F620004394410E27E00BC0183030F4212F06C060
:10F6300027E04CE3442E03C027E017E0412C56019D
:10F6400074E0A70EB11CF601608171818281938103
:10F65000042DA4010E9449876C01098100FF02C0AA
:10F6600003FF06C071FC07C072FC08C0612C08C013
:10F670003DE2632E05C02BE2622E02C090E2692EAD
:10F68000802F8C7099F1662011F084E001C083E036
:10F69000851510F0512C0BC0581A73FC08C0B70127
:10F6A00080E290E00E94AA885A94C9F7F3CF6620BE
:10F6B00029F0B701862D90E00E94AA8803FD03C0BF
:10F6C0000EED1FE002C00AED1FE0F72DF0717F2E56
:10F6D000F8018491882309F476C271108052B70131
:10F6E00090E00E94AA880F5F1F4FF2CF77FE0FC0F5
:10F6F0004C0C04FF04C08A81813309F44A94141429
:10F7000074F5F8E0F41578F588E0482E2CC076FC06
:10F710002AC0812F90E08C159D059CF06CEFC616D9
:10F720006FEFD60674F0772D7068772E0AC0E2E08E
:10F73000F0E0EC0FFD1FE10FF11D8081803319F423
:10F7400011501111F4CF77FE0EC044244394410EA2
:10F75000812F90E0C816D9062CF41C1904C044244B
:10F76000439401C010E077FE07C01C141D043CF454
:10F7700096012F5F3F4F05C025E030E002C021E039
:10F7800030E0662011F02F5F3F4F112331F0412F01
:10F7900050E04F5F5F4F240F351F452D50E0241779
:10F7A000350714F4521A01C0512C872D897049F481
:10F7B000552039F0B70180E290E00E94AA885A945F
:10F7C000F7CF662029F0B701862D90E00E94AA8825
:10F7D00073FC09C0552039F0B70180E390E00E9426
:10F7E000AA885A94F7CF77FE5FC09C2D8D2DD7FE47
:10F7F00002C090E080E0692E782E40E050E0C60123
:10F80000841991099D878C87960126193709280D3F
:10F81000391D812F90E0EE27FF27E81BF90BFF87AA
:10F82000EE87FFEF6F167F0669F4B7018EE290E076
:10F830002B8B3A8B488B598B0E94AA88598948890F
:10F840003A892B89C614D70454F06C857D856615DA
:10F8500077052CF4F901E40FF51F818101C080E3E5
:10F8600071E0671A71084F5F5F4FEE85FF856E1676
:10F870007F066CF0B70190E02B8B3A8B488B598B4D
:10F880000E94AA882B893A8948895989CACF6C1461
:10F890007D0439F49A81963318F4953311F404FFFA
:10F8A00081E3B70190E04BC08A81813309F00F7E7C
:10F8B000B70190E00E94AA88111105C074FE18C01B
:10F8C00085E490E017C0B7018EE290E00E94AA881C
:10F8D00082E066246394680EF401E80FF11D8081D4
:10F8E000B70190E00E94AA88115041F3862DF1CF14
:10F8F00085E690E0B7010E94AA88D7FC05C0C11434
:10F90000D10439F404FF05C0D194C194D1088DE22B
:10F9100001C08BE2B70190E00E94AA8880E36AE010
:10F92000C616D1042CF08F5FFAE0CF1AD108F7CFBA
:10F93000B70190E00E94AA88B701C601C0960E9454
:10F94000AA8841C1833631F0833779F0833509F0D5
:10F9500058C021C0560172E0A70EB11CF60180818B
:10F96000898301E010E0640114C05601F2E0AF0E9B
:10F97000B11CF601C080D18026FF03C0612F70E06A
:10F9800002C06FEF7FEFC6012B8B0E9470888C0145
:10F990002B892F7715C05601F2E0AF0EB11CF6018E
:10F9A000C080D18026FF03C0612F70E002C06FEFDE
:10F9B0007FEFC6012B8B0E9432888C012B89206837
:10F9C000722E23FD1AC0852D90E008171907A8F4A0
:10F9D000B70180E290E00E94AA885A94F4CFF60121
:10F9E00077FC859177FE81916F01B70190E00E94CD
:10F9F000AA8851105A94015011090115110579F77F
:10FA0000E2C0843611F0893651F5560127FF09C04E
:10FA1000F4E0AF0EB11CF6016081718182819381A7
:10FA20000AC0F2E0AF0EB11CF60160817181882737
:10FA300077FD8095982F022F0F7697FF08C090953D
:10FA40008095709561957F4F8F4F9F4F00682AE09A
:10FA500030E0A4010E94B589C82EC8183EC0022F0C
:10FA6000853721F40F7E2AE030E01DC0097F8F36F4
:10FA700091F018F4883559F0B0C0803719F0883704
:10FA800011F0ABC0006104FF09C0046007C024FF8F
:10FA900008C0066006C028E030E005C020E130E084
:10FAA00002C020E132E0560107FF09C0F4E0AF0ECA
:10FAB000B11CF601608171818281938108C0F2E0FE
:10FAC000AF0EB11CF6016081718180E090E0A4016D
:10FAD0000E94B589C82EC8180F7706FF0BC0202FCB
:10FAE0002E7FC11650F404FF0AC002FD08C0202F6B
:10FAF0002E7E05C0DC2C202F03C0DC2C01C0D12EB3
:10FB000024FF0DC0FE01EC0DF11D8081803311F446
:10FB1000297E09C022FF06C0D394D39404C0822F4B
:10FB2000867809F0D39423FD13C020FF06C01C2D56
:10FB3000D51418F4150D1D19D52CD51468F4B7017A
:10FB400080E290E02B8B0E94AA88D3942B89F5CF7A
:10FB5000D51410F45D1801C0512C24FF12C0B70158
:10FB600080E390E02B8B0E94AA882B8922FF17C08C
:10FB700021FF03C088E590E002C088E790E0B7016C
:10FB80000CC0822F867859F021FD02C080E201C0AE
:10FB90008BE227FD8DE2B70190E00E94AA88C11692
:10FBA00038F4B70180E390E00E94AA881150F7CFA3
:10FBB000CA94F401EC0DF11D8081B70190E00E9420
:10FBC000AA88C110F5CF552009F4C2CCB70180E254
:10FBD00090E00E94AA885A94F6CFF7018681978117
:10FBE00002C08FEF9FEF63960FB6F894DEBF0FBE93
:10FBF000CDBFDF91CF911F910F91FF90EF90DF90DC
:10FC0000CF90BF90AF909F908F907F906F905F90BC
:10FC10004F903F902F9008955058BB27AA270ED0A1
:10FC20004EC23FD230F044D220F031F49F3F11F465
:10FC30001EF4FFC10EF4E095E7FBF5C1E92F50D2A9
:10FC400080F3BA17620773078407950718F071F4F9
:10FC50009EF568C20EF4E0950B2EBA2FA02D0B0175
:10FC6000B90190010C01CA01A0011124FF27591B01
:10FC700099F0593F50F4503E68F11A16F040A22F07
:10FC8000232F342F4427585FF3CF46953795279578
:10FC9000A795F0405395C9F77EF41F16BA0B620B77
:10FCA000730B840BBAF09150A1F0FF0FBB1F661FBE
:10FCB000771F881FC2F70EC0BA0F621F731F841F01
:10FCC00048F4879577956795B795F7959E3F08F027
:10FCD000B3CF9395880F08F09927EE0F97958795E6
:10FCE0000895DFD158F080E891E009F49EEFE0D16B
:10FCF00028F040E851E059F45EEF09C09AC112C201
:10FD0000E92FE078EDD168F3092E052AC1F3261713
:10FD100037074807590738F00E2E07F8E02569F035
:10FD2000E025E0640AC0EF6307F8009407FADB01FE
:10FD3000B9019D01DC01CA01AD01EF9347D0BFD1EC
:10FD40000AD05F91552331F02BED3FE049E450FD9F
:10FD500049EC63CF0895DF93DD27B92FBF7740E8E3
:10FD60005FE31616170648075B0710F4D92FE1D199
:10FD70009F938F937F936F9346D3E0E2F1E06CD132
:10FD80009ED12F913F914F915F919AD2DD2349F0FF
:10FD90009058A2EA2AED3FE049EC5FE3D0785D2776
:10FDA0004DDFDF918CC11BD108F481E008950CD0A8
:10FDB00086C17ED140F075D130F021F45F3F19F05B
:10FDC00032C15111B0C135C18BD198F39923C9F318
:10FDD0005523B1F3951B550BBB27AA276217730751
:10FDE000840738F09F5F5F4F220F331F441FAA1F05
:10FDF000A9F333D00E2E3AF0E0E830D091505040C5
:10FE0000E695001CCAF729D0FE2F27D0660F771F72
:10FE1000881FBB1F261737074807AB07B0E809F054
:10FE2000BB0B802DBF01FF2793585F4F2AF09E3FE9
:10FE3000510568F0F8C077C15F3FECF3983EDCF302
:10FE4000869577956795B795F7959F5FC9F7880F62
:10FE5000911D9695879597F90895E1E0660F771FB4
:10FE6000881FBB1F621773078407BA0720F0621B45
:10FE7000730B840BBA0BEE1F88F7E095089519F405
:10FE80000EF0D1C04FC1D5C033D1C8F39638C0F7FA
:10FE900007F80F92E8942BE33AEA48EB5FE712D2B7
:10FEA0000F920F920F924DB75EB70F92CAD1EDE449
:10FEB000F1E0D2D04F915F91EF91FF91E595EE1F68
:10FEC000FF1F49F0FE57E0684427EE0F441FFA95E4
:10FED000E1F74195550B36D10F9007FE2AC10895E1
:10FEE00097FB0EF4A9D03EC0E89409C097FB3EF4FE
:10FEF00090958095709561957F4F8F4F9F4F992377
:10FF0000A9F0F92F96E9BB279395F69587957795F4
:10FF10006795B795F111F8CFFAF4BB0F11F460FFB4
:10FF20001BC06F5F7F4F8F4F9F4F16C0882311F00C
:10FF300096E911C0772321F09EE8872F762F05C020
:10FF4000662371F096E8862F70E060E02AF09A95BB
:10FF5000660F771F881FDAF7880F9695879597F9B0
:10FF60000895E894F92F96EBFF2381F012161306FB
:10FF70001406440B9395F695879577956795579555
:10FF80004040FF23B9F71BC099270895882351F4F7
:10FF90009850D2F7872B762F652F542F432F322F6F
:10FFA00020E0B1F3121613061406440B88233AF02E
:10FFB0009A95440F551F661F771F881FCAF7552350
:10FFC0004AF4440F551F11F460FF04C06F5F7F4F68
:10FFD0008F4F9F4F880F9695879597F90895990FA2
:10FFE0000008550FAA0BE0E8FEEF16161706E80703
:10FFF000F907C0F012161306E407F50798F0621B24
:020000021000EC
:10000000730B840B950B39F40A2661F0232B242BF8
:10001000252B21F408950A2609F4A140A6958FEF17
:10002000811D811D089597F99F6780E870E060E069
:1000300008959FEF80EC0895909580957095609558
:1000400050954095309521953F4F4F4F5F4F6F4FE3
:100050007F4F8F4F9F4F0895DF93CF931F930F9341
:10006000FF92EF92DF927B018C01689405C0DA2E3B
:10007000EF0126D1FE01E894A59125913591459196
:100080005591AEF3EF01DADDFE019701A801DA9494
:1000900079F7DF90EF90FF900F911F91CF91DF9153
:1000A000089500240A9416161706180609060895DE
:1000B00000240A9412161306140605060895092E44
:1000C0000394000C11F4882352F0BB0F40F4BF2BB3
:1000D00011F460FF04C06F5F7F4F8F4F9F4F0895F3
:1000E00057FD9058440F551F59F05F3F71F04795E9
:1000F000880F97FB991F61F09F3F79F087950895CE
:10010000121613061406551FF2CF4695F1DF08C0EC
:10011000161617061806991FF1CF86957105610509
:1001200008940895E894BB2766277727CB0197F9B1
:1001300008959B01AC0160E070E080E89FE337CE5A
:1001400072CF64C1D5DFE8F39923D9F3940F511D21
:10015000BBF39150504094F059F0882332F0660F71
:10016000771F881F91505040C1F79E3F510544F7BB
:10017000880F911D9695879597F908955F3FACF08C
:10018000983E9CF0BB27869577956795B79508F4C0
:10019000B1609395C1F7BB0F58F711F460FFE8CF3A
:1001A0006F5F7F4F8F4F9F4FE3CFBDCF0AD029EDB9
:1001B0003BE54EED5EE378C00EF028C13ACF68947F
:1001C00032CF96DFC8F39923D1F3C6F3DF93CF93F1
:1001D0001F930F93FF92C92FDD2788232AF02197C1
:1001E000660F771F881FDAF720E030E040E85FEB0A
:1001F0009FE3883920F0803E30F021968F770DDD27
:10020000E5E7F1E003C009DDE2EAF1E025DF8B017B
:10021000BE01EC01FB2E6F5771097595771F880B96
:10022000990B64DE28E132E741E35FE349D0AF2D6B
:100230009801AE01FF900F911F91CF91DF91FEDCED
:100240003ECFFA01DC01AA0FBB1F9B01AC01BF57D7
:1002500028F422273327442750781FC0B75188F449
:10026000AB2F0024469537952795011CA395D2F313
:10027000002069F0220F331F441FB395DAF30DD02D
:10028000CBCC61307105A0E88A07B94630F49B01F8
:10029000AC016627772788279078309621F0208355
:1002A00031834283538308950BD009CFFADE28F0BF
:1002B000FFDE18F0952309F0B6CEBBCE112433CF64
:1002C0000FDFA0F3959FD1F3950F50E0551F629F6C
:1002D000F001729FBB27F00DB11D639FAA27F00D9F
:1002E000B11DAA1F649F6627B00DA11D661F829FC6
:1002F0002227B00DA11D621F739FB00DA11D621FAB
:10030000839FA00D611D221F749F3327A00D611DC7
:10031000231F849F600D211D822F762F6A2F1124A9
:100320009F5750408AF0E1F088234AF0EE0FFF1FFC
:10033000BB1F661F771F881F91505040A9F79E3F33
:10034000510570F070CEEFCE5F3FECF3983EDCF3DA
:10035000869577956795B795F795E7959F5FC1F770
:10036000FE2B880F911D9695879597F90895FA01B0
:10037000EE0FFF1F30962105310599F161157105CA
:1003800061F48038BFE39B0749F168949038810598
:1003900061F08038BFEF9B0741F0992342F5FF3FA2
:1003A000E1053105210511F1E8940894E795D9019B
:1003B000AA2329F4AB2FBE2FF85FD0F310C0FF5F44
:1003C00070F4A695E0F7F73950F019F0FF3A38F4D9
:1003D0009F779F930CD00F9007FC905808953EF0A4
:1003E00028CE60E070E080E89FE308954FE79F77B4
:1003F0005F934F933F932F93E4DE2F913F914F9163
:100400005F9152DF41CD9B01AC014ECF9F3F31F058
:10041000915020F4879577956795B795880F911D32
:100420009695879597F908950E941C82332312F4BC
:100430008A1B9B0B0C942D82A29FB001B39FC0011D
:10044000A39F700D811D1124911DB29F700D811D00
:100450001124911D08950E941C82B7FF0895821BEC
:10046000930B08950E941C82A59F900DB49F900D40
:10047000A49F800D911D11240895B7FF0C94328222
:100480000E943282821B930B0895DB018F939F930E
:100490000E943282BF91AF91A29F800D911DA39FB8
:1004A000900DB29F900D11240895AA1BBB1B51E122
:1004B00007C0AA1FBB1FA617B70710F0A61BB70BD4
:1004C000881F991F5A95A9F780959095BC01CD0179
:1004D000089597FB072E16F4009407D077FD09D0F6
:1004E0000E94558207FC05D03EF4909581959F4F60
:1004F0000895709561957F4F0895A1E21A2EAA1B69
:10050000BB1BFD010DC0AA1FBB1FEE1FFF1FA217C3
:10051000B307E407F50720F0A21BB30BE40BF50BC0
:10052000661F771F881F991F1A9469F76095709549
:10053000809590959B01AC01BD01CF010895052EDA
:1005400097FB1EF400940E94CA8357FD07D00E94B7
:100550007D8207FC03D04EF40C94CA8350954095DD
:10056000309521953F4F4F4F5F4F0895689401C0DC
:10057000E894F92FF12B12F00C94EA82A0E0B0E09D
:10058000E4ECF2E80C94E883092E059422F40E942E
:10059000D283112392F4F0E80F26FFEFE094F09459
:1005A00000951095B094C094D094A194BF0ACF0A3E
:1005B000DF0AEF0AFF0A0F0B1F0B0E94798307FC6B
:1005C0000E94D283CDB7DEB7ECE00C94048468942B
:1005D00001C0E8948F929F92CF93DF930E9479831A
:1005E000DF91CF919F908F900895DF93CF931F93CA
:1005F0000F939A9DF02D219FF00D8B9DF00D8A9DFC
:10060000E02DF10D039FF00D029FE00DF11D4E9DB9
:10061000E00DF11D5E9DF00D4F9DF00D7F936F93EA
:10062000BF92AF925F934F93D5010E941C828B01C2
:10063000AC01D7010E941C82EB01E80FF91FD60123
:100640000E9445832F913F91D6010E941C82C60FC4
:10065000D71FE81FF91FAF91BF910E9445832F91CB
:100660003F910E941C82C60FD71FE81FF91FD601B9
:100670000E941C82E60FF71F9801BE01CF011124D2
:100680000F911F91CF91DF9108950E941C82460F18
:10069000571FC81FD91F08F431960895E894DF93B7
:1006A000CF93FC01DB010E941C827F936F93E901D1
:1006B0009A01AC01BF93AF933F932F93DF010E9448
:1006C0001C8226F46C1B7D0B820B930B9E01EB01AD
:1006D000FC010E944583AF91BF912F913F910E94F1
:1006E0004583BE01CF01F9012F913F91CF91DF9159
:1006F000089588249924F401E401B0E49F93AA2783
:100700009A158B049C04ED05FE05CF05D007A107C3
:1007100098F4AD2FDC2FCF2FFE2FE92D982C892EAA
:10072000982F872F762F652F542F432F322F222774
:10073000B85031F7BF9127C01B2EBF91BB27220FA6
:10074000331F441F551F661F771F881F991F881C62
:10075000991CEE1FFF1FCC1FDD1FAA1FBB1F8A1491
:100760009B04EC05FD05CE05DF05A007B10748F0A9
:100770008A189B08EC09FD09CE09DF09A00BB10B13
:1007800021601A94E1F62EF49401AF01BE01CD016F
:10079000000C089590958095709561957F4F8F4FCF
:1007A0009F4F0895609570958095909530954095F0
:1007B000509521953F4F4F4F5F4F6F4F7F4F8F4F5A
:1007C0009F4F08952F923F924F925F926F927F9228
:1007D0008F929F92AF92BF92CF92DF92EF92FF9251
:1007E0000F931F93CF93DF93CDB7DEB7CA1BDB0BFD
:1007F0000FB6F894DEBF0FBECDBF09942A883988A2
:1008000048885F846E847D848C849B84AA84B984A8
:10081000C884DF80EE80FD800C811B81AA81B981B4
:10082000CE0FD11D0FB6F894DEBF0FBECDBFED01C8
:1008300008950F93083090F0982F872F762F652F0B
:10084000542F432F322F22270850F4CF220F331F6B
:10085000441F551F661F771F881F991F0A95B2F7FF
:100860000F91089597FB10F8169400080F93083025
:1008700098F00850232F342F452F562F672F782FAD
:10088000892F902DF4CF0594979587957795679547
:1008900057954795379527950A95AAF70F9108958B
:1008A0002A0D3B1D4C1D5D1D6E1D7F1D801F911F60
:1008B00008950024A7FD00942A0F301D401D501DEF
:1008C000601D701D801D901D08952A193B094C095B
:1008D0005D096E097F09800B910B08952A153B0570
:1008E0004C055D056E057F0580079107089500247E
:1008F000A7FD00942A1730054005500560057005D6
:100900008005900508958F929F92AF92BF92CF92EB
:10091000DF92EF92FF92CF93DF93EC0168817981B0
:100920008A819B81611571058105910521F464E23D
:1009300079ED8BE597E02DE133EF41E050E00E9447
:100940009F8249015A019B01AC01A7EAB1E40E94D0
:1009500032826B017C01ACEEB4EFA50194010E94E0
:100960004082C60ED71EE81EF91EF7FE06C081E0C3
:10097000C81AD108E10880E8F80AC882D982EA8258
:10098000FB82C6019F77DF91CF91FF90EF90DF90C0
:10099000CF90BF90AF909F908F9008950C948384D8
:1009A00089EE93E00C948384A0E0B0E08093E903A7
:1009B0009093EA03A093EB03B093EC0308952F9276
:1009C0003F925F926F927F928F929F92AF92BF926F
:1009D000CF92DF92EF92FF920F931F93CF93DF930B
:1009E0008B01EA016115710521F0DB018C931196F1
:1009F0009C93209739F09E01225031092332310512
:100A000008F0FBC07C016701BFEFCB1ADB0A56017F
:100A1000F7016080862D90E00E942188892B11F0DB
:100A20007601F1CFFDE26F120AC0570182E0A80EF5
:100A3000B11CD70111966C90772473940BC0BBE264
:100A40006B1207C05701E2E0AE0EB11CD701119640
:100A50006C90712CCE018F7E892B89F4B0E36B12E0
:100A600022C0F50180818F7D883541F56180F2E0FB
:100A7000AF0EB11C872D8260782EC0E1D0E0C83067
:100A8000D105F1F04CF4C230D10511F5C12CD12CB7
:100A9000E12CB0E4FB2E2FC0CA30D10531F0C031BB
:100AA000D10521F115C0209751F7CAE0D0E0ACEC98
:100AB000CA2EDC2CEC2CACE0FA2E1DC02097F9F6E7
:100AC000C8E0D0E0C12CD12CE12CF0E1FF2E13C006
:100AD00060E070E080E090E89E01442737FD40959B
:100AE000542F0E947D8269017A0105C0C12CD12C4E
:100AF000E12CE8E0FE2EF50160E020E030E0A90105
:100B00004E01AA2497FCA094BA2C1F0170ED572E19
:100B1000560CA9E0A51570F48FEB860D8A3118F4F8
:100B200099EC592E06C08FE9860D8A3130F589EA95
:100B3000582E560C852D90E08C179D07F4F467FD18
:100B400018C0C216D306E406F50680F0C501B4014C
:100B50000E9445829B01AC01250D311D411D511D97
:100B6000213031054105B0E85B0710F06FEF01C09F
:100B700061E03196D1016C90C8CF872D817001154D
:100B8000110571F0662329F03197D801ED93FC939C
:100B900007C071FE19C03297D801ED93FC9314C0C1
:100BA00067FF12C0882329F020E030E040E050E8E1
:100BB00004C02FEF3FEF4FEF5FE782E290E09093AA
:100BC000A8308093A73016C0882341F050954095F7
:100BD000309521953F4F4F4F5F4F0CC057FF0AC0D4
:100BE00082E290E09093A8308093A7302FEF3FEF00
:100BF0004FEF5FE7B901CA0104C060E070E080E038
:100C000090E0DF91CF911F910F91FF90EF90DF90D7
:100C1000CF90BF90AF909F908F907F906F905F909C
:100C20003F902F9008952F923F925F926F927F9204
:100C30008F929F92AF92BF92CF92DF92EF92FF92EC
:100C40000F931F93CF93DF938B01EA016115710519
:100C500021F0DB018C9311969C93209739F09E0133
:100C6000225031092332310508F0D8C07C016701D8
:100C7000BFEFCB1ADB0A5601F7016080862D90E0AA
:100C80000E942188892B11F07601F1CFFDE26F12CD
:100C90000AC0570182E0A80EB11CD70111966C90D2
:100CA000772473940BC0BBE26B1207C05701E2E0DC
:100CB000AE0EB11CD70111966C90712CCE018F7EB7
:100CC000892B89F4B0E36B1237C0F50180818F7DE9
:100CD0008835D1F46180F2E0AF0EB11C872D8260BF
:100CE000782EC0E1D0E0CA30D10551F1C031D10534
:100CF00021F0C830D10599F409C0CC24CA94DC2C69
:100D0000EC2CAFE0FA2E22C0209769F7C8E0D0E0C3
:100D1000CC24CA94DC2CEC2CFFE1FF2E17C06FEF23
:100D20007FEFCB019E01442737FD4095542F0E9451
:100D30007D8269017A010AC02097A9F6CAE0D0E055
:100D4000E9E9CE2EDC2CEC2CE9E1FE2EF50160E089
:100D500020E030E0A9014E01AA2497FCA094BA2C0F
:100D60001F0170ED572E560CA9E0A51570F48FEBFE
:100D7000860D8A3118F499EC592E06C08FE9860D3C
:100D80008A3148F589EA582E560C852D90E08C174B
:100D90009D070CF56F3FD9F0C216D306E406F506A1
:100DA00098F0C501B4010E9445829B01AC01852DDC
:100DB00090E0A0E0B0E0280F391F4A1F5B1F281702
:100DC00039074A075B0710F46FEF01C061E0319605
:100DD000D1016C90C5CF0115110551F0662311F0BA
:100DE000319703C071FE04C03297D801ED93FC9394
:100DF00070FE07C050954095309521953F4F4F4F5D
:100E00005F4F67FF10C082E290E09093A83080931C
:100E1000A7306FEF7FEF8FEF9FEF07C060E070E0CC
:100E200080E090E002C0B901CA01DF91CF911F912B
:100E30000F91FF90EF90DF90CF90BF90AF909F9079
:100E40008F907F906F905F903F902F9008956627CE
:100E500077270C944E8AFC0188279927E8942191E2
:100E60002032E9F3293010F02E30C8F32B3241F054
:100E70002D3239F4689404C00E94A288820F911D1B
:100E8000219120532A30C0F31EF4909581959F4FF5
:100E90000895283008F027E03327DA01990F311D33
:100EA00087FD916000966105710539F432602E5F0F
:100EB0003D9330E32A95E1F708959F3F30F0803865
:100EC0007105610509F03C5F3C5F3D93913008F08E
:100ED0008068911DDF93CF931F930F93FF92EF9242
:100EE000192F987F9695E92F96959695E90FFF27EC
:100EF000E45CFF4E99273327EE24FF24A701E70186
:100F000005900894079428F4360FE71EF81E491F31
:100F1000511D660F771F881F991F0694A1F7059032
:100F2000079428F4E70EF81E491F561FC11D770FBE
:100F3000881F991F661F0694A1F70590079428F44F
:100F4000F80E491F561FC71FD11D880F991F661F16
:100F5000771F0694A1F70590079420F4490F561FB8
:100F6000C71FD81F990F661F771F881F0694A9F700
:100F700084911095177041F0D695C7955795479570
:100F8000F794E7941A95C1F7E2EEFFE068941590A4
:100F9000159135916591959105907FE27395E118D2
:100FA000F10A430B560BC90BD009C0F7E10CF11E37
:100FB000431F561FC91FD01D7EF4703311F48A954C
:100FC000E6CFE894015030F0080F0AF4002702172A
:100FD00008F4202F2395022F7A3328F079E37D93AC
:100FE0002A95E9F710C07D932A9589F6069497957E
:100FF0006795379517951794E118F10A430B560B2F
:10100000C90BD00998F023957E9173957A3308F037
:1010100070E37C932013B8F77E9170617D9330F07C
:10102000839571E37D9370E32A95E1F71124EF90A6
:10103000FF900F911F91CF91DF91992787FD909598
:1010400008959111A8C3803219F089508550D0F7C6
:101050000895FB01DC018D91059080190110D9F3F1
:10106000990B0895FC010590615070400110D8F76C
:10107000809590958E0F9F1F08954EE55AE10C9430
:101080007B88FB01DC0102C001900D924150504071
:10109000D8F70895DC0101C06D9341505040E0F74E
:1010A0000895FB01DC018D91019080190110D9F3A5
:1010B000990B0895FB01DC0101900D920020E1F7EE
:1010C0000895FB01DC014150504048F001900D9221
:1010D0000020C9F701C01D9241505040E0F708952B
:1010E000FC016150704001900110D8F780959095F7
:1010F0008E0F9F1F0895FA01A191B081009719F4F6
:101100001097E1F0CD01DC01CD010D90002011F42C
:10111000C00113C0FB012191222319F02015D9F73A
:10112000F3CFFB012191201519F41E92119606C0F0
:101130002223C1F70D900020A1F7D001FA01A1935D
:10114000B08308957AE0979F902D879F802D910D11
:10115000112408950F931F93CF93DF93182F092F16
:10116000EB018B8181FD03C08FEF9FEF20C082FFD9
:1011700010C04E815F812C813D81421753077CF462
:10118000E881F9819F012F5F3F4F398328831083C6
:1011900006C0E885F985812F0995892B29F72E81CD
:1011A0003F812F5F3F4F3F832E83812F902FDF9111
:1011B000CF911F910F910895CF93DF93CDB7DEB7F5
:1011C000FE01359661917191AF018091A3309091AC
:1011D000A4300E94687ADF91CF9108950F931F93F6
:1011E000CF93DF93CDB7DEB7FE0137966191719152
:1011F00003EA10E3D8018D919C91DC0113962C91A8
:101200001397286013962C93AF010E94687AD80137
:10121000ED91FC912381277F2383DF91CF911F9153
:101220000F9108950F931F93CF93DF93E091A33015
:10123000F091A430238121FF1BC0EC0100E010E0FD
:1012400089916091A3307091A430DB011896ED91E3
:10125000FC911997882331F00995892B89F30FEFB9
:101260001FEFEECF8AE00995892B11F4C80102C067
:101270008FEF9FEFDF91CF911F910F9108950F9303
:101280001F93CF93DF93CDB7DEB72E970FB6F894A9
:10129000DEBF0FBECDBF0D891E898F89988D26E0D8
:1012A0002C831A83098397FF02C080E090E801979E
:1012B0009E838D83AE01455E5F4F698D7A8DCE0131
:1012C00001960E94687A4D815E8157FD0AC02F8188
:1012D0003885421753070CF49A01F801E20FF31F07
:1012E00010822E960FB6F894DEBF0FBECDBFDF91F1
:1012F000CF911F910F9108950F931F93CF93DF9379
:10130000CDB7DEB72E970FB6F894DEBF0FBECDBFB8
:101310008C01CA0146E04C831A83098377FF02C01F
:1013200060E070E8615071097E836D83A901BC01A2
:10133000CE0101960E94687A4D815E8157FD0AC0F8
:101340002F813885421753070CF49A01F801E20FF8
:10135000F31F10822E960FB6F894DEBF0FBECDBFDE
:10136000DF91CF911F910F910895FA01AA2728309C
:1013700051F1203181F1E8946F936E7F6E5F7F4F62
:101380008F4F9F4FAF4FB1E03ED0B4E03CD0670FDE
:10139000781F891F9A1FA11D680F791F8A1F911D31
:1013A000A11D6A0F711D811D911DA11D20D009F481
:1013B00068943F912AE0269F11243019305D3193C3
:1013C000DEF6CF010895462F4770405D4193B3E0AC
:1013D0000FD0C9F7F6CF462F4F70405D4A3318F053
:1013E000495D31FD4052419302D0A9F7EACFB4E004
:1013F000A6959795879577956795BA95C9F70097BC
:101400006105710508959B01AC010A2E069457955C
:10141000479537952795BA95C9F7620F731F841FB3
:10142000951FA01D0895DC01CB01FC01F999FECFA9
:1014300006C0F2BDE1BDF89A319600B40D9241505C
:101440005040B8F70895F999FECF92BD81BDF89A42
:10145000992780B50895A8E1B0E042E050E00C94EF
:10146000158ADC01CB0103C02D910E943C8A4150BA
:101470005040D0F70895262FF999FECF1FBA92BD9C
:1014800081BD20BD0FB6F894FA9AF99A0FBE019665
:1014900008950E943B8A272F0C943C8A4F925F92BA
:1014A0006F927F928F929F92AF92BF92CF92DF9274
:1014B000EF92FF920F931F93CF93DF938B016115F0
:1014C000710521F0DB018C9311969C93EC015E0178
:1014D000BFEFAB1ABB0A7501C8808C2D90E00E944B
:1014E0002188892B11F0E501F2CFEDE2CE1208C080
:1014F0007E01F2E0EF0EF11CC980DD24D39409C017
:101500002BE2C21205C07E0142E0E40EF11CC9804C
:10151000D12CE701219743E050E064EE70E1CE0169
:101520000E94CE8B892BD1F4E701229645E050E052
:101530006FED70E1CE010E94CE8B892B11F4E70193
:1015400027960115110519F0D801CD93DC93D11020
:1015500008C160E070E080E89FE70CC143E050E024
:101560006CED70E1CE010E94CE8B892B59F40115F0
:10157000110509F4FBC0B2E0EB0EF11CF801F18299
:10158000E082F4C0F70160E070E0CB01C0E0D0E0A1
:101590007F01A0EDAA2EAC0C29E02A1530F14D2DCB
:1015A0004260B42E2D2D2870D2FE04C0211125C01A
:1015B000219623C021112197A5E0B0E09B01AC0149
:1015C0000E943282660F771F881F991F6A0D711D56
:1015D000811D911D6839A9E97A078A07A9E19A074F
:1015E00060F0BD2DB660BB2E08C02EEFA2120AC05F
:1015F000D3FC50C04D2D4860B42E3196D701CC900D
:10160000DB2CC6CF2C2D2F7D253409F043C0A081C3
:10161000AD3241F4BD2DB061DB2E7F0122E0E20E40
:10162000F11C0CC07F01AB3231F04FEFE41AF40A29
:1016300021E030E006C0A2E0EA0EF11CA18122E028
:1016400030E0A053AA3018F0E21AF30A23C0F701E1
:1016500020E030E02038BCE03B075CF4A901440FF7
:10166000551F440F551F240F351F220F331F2A0FFC
:10167000311DAF014F5F5F4F7A01A081A053AA30A7
:1016800010F4FA01E7CFD4FE03C03195219531095A
:10169000C20FD31FD1FE09C00115110531F0E1E0E1
:1016A000EE1AF108D801ED92FC920E94747F2D2D64
:1016B0002370233019F06B017C0106C06B017C01A3
:1016C000F7FAF094F7F8F09420E030E0A901C701B0
:1016D000B6010E94D37E882309F440C0D7FF06C01C
:1016E000D195C195D1090BEF10E102C003E111E1E1
:1016F0004801B8E18B1A910890E2A92EB12CF801AB
:101700004590559065907490CA15DB055CF0A30177
:101710009201C701B6010E9454816B017C01CA1974
:10172000DB09F2CF04501109B594A79408151905E7
:1017300031F78E2D880F8F2D881F8F3F49F020E0C5
:1017400030E0A901C701B6010E94D37E811106C015
:1017500082E290E09093A8308093A730C701B60151
:1017600009C060E070E080E89FEF04C060E070E0D6
:1017700080EC9FE7DF91CF911F910F91FF90EF9049
:10178000DF90CF90BF90AF909F908F907F906F90A1
:101790005F904F900895992788270895FB01DC01F9
:1017A0004150504088F08D9181341CF08B350CF401
:1017B000805E659161341CF06B350CF4605E861BB5
:1017C000611171F3990B0895881BFCCFF894FFCF3A
:1017D000010010001F004000261166090000D50816
:1017E000E715000000000000E608FB0E0000000006
:1017F0000000F408953800000000000006090F0EF4
:101800000000000000001409D837000000000F1A83
:101810000A403C003C003C004D80040000000000F9
:101820006162636465666768696A6B6C6D6E6F7030
:1018300020091A22FFCC3B22FFCC3BD734EF3C01DE
:101840000000000F460346181000000000457665B2
:101850006E742074696D65720000007D021A4A0082
:101860000000004374696D65722070726F63657368
:10187000730000009302584B0000000002030607AB
:101880000A0B0E0F020306070A0B0E0F284329202E
:1018900032303132204865726A756C660055747654
:1018A00065636B6C696E6720202020202000436FE9
:1018B0006E74696B6920322E350000000002000052
:1018C0000000835A00000000C600C500C400C1002B
:1018D000C200000000CE00CD00CC00C900CA00004C
:1018E000000052463233302064726976657200001F
:1018F0000012033A5F00000000AB5D295D895FD3F1
:10190000604C5EDC5C4A5B445BCB5C2D5C0001019F
:1019100001010101010101010101010101005269FF
:101920006D65004E034E62156261646174612E6ED6
:10193000756D20776179206F7574207468657265A4
:101940003A2025640A0090638F639965C866006534
:101950000080C0E0F0F8FCFEFF6E756C6C6D61639A
:101960000089037B67606766676C67726778677377
:101970006963736C6F776D6163009F039C68FD679B
:1019800093677C6782679067BA000800E713EF13DC
:1019900035000200BF19C1195443502F495020731C
:1019A0007461636B000000C803F66A000000000267
:1019B00008FFFFFFFF0000000001000000BC430023
:1019C0000034022A0220020C021602000054696D43
:1019D000656F757420414444523D252D642E252D9C
:1019E00064205345513D252D6420525353493D25D4
:1019F0002D75204C51493D252D750A0028457874D8
:101A00005077722900415432344D414300484948CF
:101A10003631333000424D50303835004144584C57
:101A200033343500484D4335383833004C33473470
:101A300032303044005348543258004D4350333410
:101A40003258004D5335363131004E484443303220
:101A500031360065756936343D00253032780073C3
:101A60006E3D00413A202564202564202564200A2B
:101A700000433A20256420256420256420613D250B
:101A8000352E31660A0073687432785F7365726947
:101A9000616C3D253032782530327825303278251A
:101AA000303278253032782530327825303278253A
:101AB0003032780A007374617475733D3078253064
:101AC00032780A20006669726D776172653D533223
:101AD0002D352E372D323031342D30392D32340022
:101AE0006F7065720072785F6C6564720074785F05
:101AF0006C65647900706B74006F77006C656400CE
:101B00006576656E740070305F6C6564720070316C
:101B10005F6C6564790061657300705F7077720057
:101B20007072657300616363656C00636F6D7061F3
:101B300073730072656C61795F6C656479007478A9
:101B4000740065363400696400743100745F6D633D
:101B50007500765F6D63750070300070305F7400E3
:101B600070305F6C73740070310070315F7400709E
:101B7000315F6C737400757074696D650072680014
:101B8000616800745F64657700745F686561745FA5
:101B900069647800765F696E0061310061320061CE
:101BA0003300616431006164320061643300616458
:101BB0003400706100745F73687432780072685F1B
:101BC000736874327800705F6D7335363131006F31
:101BD0006E006F666600656570726F6D007265738A
:101BE0006574006E6F6E6500737461747300747851
:101BF000743D25730A00636820706B74730025328E
:101C00007520252D3130750A006175746F00666C82
